:020000040800F2
:1000000000000220F9A700083FA8000841A8000846
:1000100043A8000845A8000847A800080000000001
:1000200000000000000000000000000049A80008D7
:100030004BA80008000000004DA80008114B000864
:1000400053A8000855A8000857A8000859A8000898
:100050005BA800085DA800085FA8000861A8000868
:1000600063A8000865A8000867A8000869A8000838
:100070006BA800086DA800086FA800080599000883
:1000800073A8000875A8000877A8000879A80008D8
:100090007BA800087DA800087FA8000881A80008A8
:1000A00083A8000885A8000887A8000889A8000878
:1000B000BD6900088DA800088FA8000891A8000855
:1000C00093A8000895A8000897A8000899A8000818
:1000D0009BA80008DD4E0008ED68000855A5000843
:1000E000A3A80008A5A80008A7A80008A9A80008B8
:1000F000ABA80008ADA80008AFA80008B1A8000888
:10010000B3A80008B5A80008B7A80008B9A8000857
:10011000BBA80008BDA80008BFA80008C1A8000827
:10012000C3A80008C5A80008C7A80008C9A80008F7
:10013000CBA80008CDA80008CFA80008D1A80008C7
:10014000D3A80008D5A80008D7A80008D9A8000897
:10015000DBA80008DDA80008DFA80008E1A8000867
:10016000E3A80008E5A80008E7A80008E9A8000837
:10017000EBA80008EDA80008EFA80008F1A8000807
:10018000F3A80008F5A8000810B5054C237833B98A
:10019000044B13B10448AFF300800123237010BD5A
:1001A0002C0100200000000074D30008084B10B59B
:1001B0001BB108490848AFF300800848036803B939
:1001C00010BD074B002BFBD0BDE81040184700BF07
:1001D000000000003001002074D300082C01002032
:1001E00000000000154B002B08BF134B9D46A3F5E4
:1001F000803A00218B460F461348144A121A0AF01F
:100200006FFC0F4B002B00D098470E4B002B00D0FB
:1002100098470020002104000D000D48002802D05E
:100220000C48AFF300800AF02DFC2000290000F0FC
:1002300013F80AF069FB00BF00000800000002206C
:1002400000000000000000002C010020504A0020A7
:1002500000000000000000002DE98048BBB005F060
:1002600095F8924A9249936803F00C03042B03D04B
:10027000082B03D08F4B18E08F4B16E05068536863
:1002800010F4800F03F03F03506814BF8A4A894A74
:10029000B2FBF3F3854A5268C2F30142C0F38810FF
:1002A000013243435200B3FBF2F3804E0B60B3685C
:1002B000824A834C834FDFF844A2C3F3031304F153
:1002C0002C00D25C0B68D3400B6012237E49E38084
:1002D0000AF083FE7D4904F16C000AF07EFE09F00D
:1002E000D1F97B4806F060FB7A4806F05DFB7A485E
:1002F00006F05AFB774806F057FB784806F054FBA7
:10030000744806F051FB06F047FB1BA804F07EFE84
:10031000336B43F00403002533631BA94FF4806360
:1003200038461B938DF870508DF871508DF87250CF
:100330008DF8735004F073FE694806F035FB65488C
:1003400006F032FB06F028FB1BA804F05FFE336BBF
:1003500043F004031BA933634FF001084FF480738B
:1003600038461B938DF871508DF870808DF872505F
:100370008DF8735004F053FE5A4806F015FB5548AB
:1003800006F012FB584806F00FFB524806F00CFB33
:1003900006F002FB05F002FA544806F005FB4D4852
:1003A00006F002FB06F0F8FA09F074FC504806F07B
:1003B000FBFA484806F0F8FA06F0EEFA1BA804F03B
:1003C00025FE336B43EA080333631BA94FF0200972
:1003D0005046CDF86C908DF871508DF870808DF886
:1003E00072508DF8735004F01AFE4248AAF81A9021
:1003F00006F0DAFA374806F0D7FA06F0CDFA1BA86D
:1004000004F004FE336B43F0040333631BA94FF481
:10041000005338461B938DF870508DF8735004F0DC
:10042000FEFD3B690A9713F4005F71D1AAF818909A
:1004300009F028F909F0A2FE2F4B1B68B3F5E13F44
:1004400001D009F00FFE2D4C102580266583322047
:10045000668304F063F926834FF4FA7004F05EF9C2
:100460002583274D274E2C46336833B11BA809F04E
:10047000D3FE10B11B9808F021F82B68002BF3D0A5
:10048000214B224819684A1CB2F5807F405C1A60F3
:1004900004BF00221A60C0B272B62368013B236019
:1004A00062B61B900AF0ACF8DEE700BF00380240ED
:1004B000B80000200024F40000127A00240000207C
:1004C000D446002000080240E3B70008EDB700085A
:1004D000F4B700082EBD000813B8000830B80008B3
:1004E0003DB800084BB800085FB800086BB80008BA
:1004F00079B800089DB8000840250020000002409F
:10050000281000202410002018020020640E002073
:10051000984806F049FA984806F046FA06F03CFA80
:10052000ADF87450ADF86E508DF87650336C4FF0D6
:10053000804743F0010333643B8823F45C731B045E
:100540001B0C3B806423FB6241233B85A7F814808E
:10055000BB899BB243F00103BB811C238DF85C3047
:1005600017A80F238DF85D308DF85E308DF85F8011
:1005700009F0D2FA3B8881489BB243F001033B80EB
:1005800006F012FA7C487E4F06F00EFA06F004FAE6
:100590001BA804F03BFD336B43F0040333631BA93A
:1005A0000A98CDF86C908DF870508DF8738004F037
:1005B00036FD744806F0F8F906F0EEF9724806F0D8
:1005C000F3F96D4806F0F0F9704806F0EDF96A4865
:1005D00006F0EAF906F0E0F96D4806F0E5F966483C
:1005E00006F0E2F913A804F0CDFC169B009313A9C2
:1005F0000EC9684806F064FF06F0CEF9664804F0BC
:100600009DFF65480AF08EF83B680BB1634800E037
:100610006348644D06F0C8F9574806F0C5F92B68E1
:100620000BB1614800E0614806F0BEF9524806F09F
:10063000BBF93B680BB12B680BBB5D4806F0B4F906
:100640004D4806F0B1F94CF2503004F077FF4CF20F
:1006500050300AF067F83B680BB1564800E0564846
:1006600006F0A2F9444806F09FF92B680BB15348F5
:1006700000E0534806F098F93F4806F095F9514ECE
:1006800005F02AFB0023336008F06EFA03F0ACFC9F
:100690002B68B046002B00F0FD804B4EDFF8389100
:1006A00033684B4500F0F6804946484806F008FF9D
:1006B000C6F8009004F098FF10B9454808F024FAF5
:1006C0002B68002B01F0608405F020FF05F0F8FE98
:1006D00005F0E6FE05F0D4FE05F0C2FE05F0B0FE22
:1006E00005F09EFE05F084FE05F068FE05F056FE5E
:1006F00005F044FE05F032FE05F020FE4FF0000943
:10070000484609F1010905F0F9FDB9F1400FF7D1AB
:100710004FF00009484609F1010905F0D3FDB9F190
:10072000100FF7D14FF00009484609F1010905F013
:10073000A5FDB9F1100FF7D105F08CFD05F076FDA0
:1007400005F062FD0622234940F2A57009F0A2FFE0
:100750002B68002B42D005F0CFF84FF00009D8F8F5
:10076000003099453DD2484605F088F809F1010965
:10077000F5E700BF8BB800082EBD00089AB8000846
:10078000A4000020ACB80008B6B80008BEB8000845
:10079000D4B80008E5B80008A086010005B9000833
:1007A00013B900083825002022B9000839B900081B
:1007B00051B9000875B9000887B900089BB900084D
:1007C000B0B900089012002034000020C6B900081B
:1007D000ECB900088446002000090200B54808F082
:1007E00093F92B68002B01F0ED831022B249AA2067
:1007F00009F050FF002801F0E58304F0B5FC002863
:1008000001F0E08305F022FA10B9AC4808F07CF959
:1008100004F006FB10B9AA4808F076F904F09EFD32
:1008200010B9A84808F070F904F038FE10B9A648CD
:1008300008F06AF907F068FE10B9A44808F064F9F6
:1008400009F0F2F810B9A24808F05EF92B68002B05
:1008500001F0BD8303F0FEFE03F0E8FE03F0D2FEDC
:1008600003F0C0FE03F0AEFE03F09CFE08F060F95A
:1008700010B9984808F048F908F07AFE10B996487F
:1008800008F042F9954806F08FF8954806F08CF884
:10089000944B3360944D2E68002E48D1DFF860826F
:1008A00011A804F0B3FB8DF87060D8F830308F4891
:1008B00043F00403C8F830301023119311A9032327
:1008C0008DF848308DF84B6004F0A9FBD8F844301F
:1008D000874A43F48073C8F844304FF48033189348
:1008E00019961A965168834B0B4043F4803353603A
:1008F000814B8DF870605A6822F0407222F4807249
:100900005A6099687D4A0A409A60DA6A22F4700255
:10091000DA62DA6822F4E042DA605A6B22F01F02EF
:1009200042F00E025A639A6842F001029A60744ED5
:100930004FF001081BA8C5F8008004F067FB336B7B
:100940006A4843F00403336300254FF400631BA996
:100950001B938DF871508DF870508DF8735004F022
:100960005EFB1BA804F052FB336B604843F00403AA
:1009700033634FF480591BA9CDF86C908DF87150FA
:100980008DF870808DF872508DF8735004F047FB2D
:100990000A9BA3F8189005F045F85A4B1A68B2F56F
:1009A000165F77D04FF4165917A84FF00C0AC3F80A
:1009B000009004F02BFBCDF86C90ADF87050ADF8C2
:1009C0007250ADF87450ADF876A0ADF87850336B36
:1009D00043F002033363336B43F002033363736CFE
:1009E00043F010037364A6F550563046336A23F083
:1009F00070633362336A43F0E0633362336A23F037
:100A000070433362336A43F0E043336202238DF86C
:100A1000603003238DF8613017A9402317938DF8B8
:100A200062508DF8638004F0FAFA3046A6F57446F9
:100A3000802317A9179304F0F2FAB3896FEA4343AE
:100A40006FEA53439BB2B38130461BA9CDF86C903B
:100A5000ADF87050ADF87250ADF87450ADF87850F4
:100A6000ADF876A009F0AAF8B389274A9BB243F4FF
:100A70000053B381136843F02003136011A82523AA
:100A80008DF844308DF845508DF846508DF84780EC
:100A900009F042F81D4805F087FF00210C2003F003
:100AA000E9FD1B4B01221A601A4B1E681D460336D6
:100AB00032E000BF20BE000868000020F5B9000841
:100AC0000EBA000827BA000841BA000853BA000855
:100AD00065BA00087BBA0008B5C50008A0BA0008CE
:100AE0002EBD0008000902005C0E00200008024034
:100AF00000230140E030FCFF00200140FDF7FFC073
:100B000000380240880F00200C100140A5BA0008F0
:100B10002C1000204C0100202B689E420CD917A8F5
:100B200007F076FD0028F7D017A807F071FD04F054
:100B3000A7FD08B104F058FD914B1A6882BB012251
:100B40001A6008F09FFD8F4805F02EFF09F016FB94
:100B50008D4B1B68B3F5E13F01D009F083FA8B4D53
:100B6000DFF8848280266E83322003F0D7FD2E8347
:100B700046460023DFF87492C8F800303225D9F8D1
:100B800000301BB93368002BF9D005E01BA809F031
:100B900043FB0028F6D0ECE70023013D3360EED1A3
:100BA0007B4B1B680BB104F0CFFF3B680BB104F02B
:100BB000A9FC3B6813B308F0F3FDF8B1E269A3693F
:100BC00060692569E668A768216A02F26C720133E0
:100BD000C4F8B020C4F8B430C4F8B800C4F8AC10FD
:100BE000C4F8BC50C4F8C060C4F8C4708DE8E1001B
:100BF000684850F82110684806F062FC05F054FE81
:100C0000664C674EFF2304930693002307930B93D0
:100C100005932546634BD3F80080634BC3F80080EF
:100C2000059B002B3CD00B9BC3EB0803052B1CD969
:100C30000A9B1F6917F4005717D15C4805F0B4FEF2
:100C40005B4805F0B1FE5B4B5B4A5F6083F83C702C
:100C50005A495B4B1BA80AF075F9012239461BA8BB
:100C600007F0C2FECDF82C801AE0079BC3EB080307
:100C7000052B15D90A9B1F6917F0200710D1514881
:100C800005F092FE4A4805F08FFE4A4B4E485F60E1
:100C90000122394683F83C7007F0A6FECDF81C808F
:100CA00001F0DCFAE36A002B48D0A36B002B45D19E
:100CB000E369002B42D0454FB81C04F0DBF8002854
:100CC0003CD07B88B7F804E0F888734538BFA7F8B4
:100CD00002E07B88834284BF3C4B5880864514D217
:100CE0007A883A49CEEB02025201CEEB000392FB26
:100CF000F3F33A781F2B28BF1F23934201D9013207
:100D000001E004D2013A0A7001E01F233B70304A2F
:100D10007988136801F110009842C1F05D811033A9
:100D2000994201F259812B493B780A68581C90423C
:100D3000C1F05D810132934201F25981059B53B9A3
:100D40001C4B1B68002B54D0234805F02DFE18487F
:100D500005F02AFE11E0214B1A6872B9154A526853
:100D60000127002A44D01E481F6005F01DFE1048D0
:100D700005F01AFE1B4B1F603AE00123059338E093
:100D800060010020B7BA00084025002000000240A2
:100D90003C1C00207CBE0008C8BA00081444002097
:100DA000380000204C01002000020020F4BA0008A6
:100DB0002EBD0008980F002038BB000842BB000879
:100DC0002DBB00084FBB00087FBB000818000020A7
:100DD000400000203C00002083BB0008780F00206A
:100DE00092BB0008D0010020B80100202410002090
:100DF0000597834A1368002B5DD0824B824F1B6896
:100E000082496433FB61824B1B68013BBB61814BB0
:100E10001B687B610B68072B4FF0000318BF096844
:100E2000BB6208BF194639627B49136009683961A2
:100E30007A4B7B491B680968F9600F21B9600BB1D7
:100E400009F09CF8D7F8BC103A696F4B914204D175
:100E5000D3F8C020DB689A4206D0724B5B680BB1B6
:100E600008F03CFE04233360FA69BB697869D7F85F
:100E700010E0396AD7F80CC0D7F8088002F26C721B
:100E80000133C7F8B020C7F8B430C7F8B800C7F8C6
:100E9000AC10C7F8BCE0C7F8C0C0C7F8C4808DE884
:100EA00001406148CDF80C8050F82110CDF808C001
:100EB0005E4806F005FB5E4B1B68002B3DD0574B90
:100EC0001B68002B36D008F06BFC98B34E49D1F864
:100ED000BC300869834204D1D1F8C020CB689A4263
:100EE00001D004233360CA698B690F6AD1F814E01A
:100EF000D1F80CC0D1F8088002F26C720133C1F84D
:100F0000B020C1F8B430C1F8B8E0C1F8AC70C1F895
:100F1000BC00C1F8C0C0C1F8C48043490190CDF8FD
:100F20000C80CDF808C0CDF800E051F827104148FA
:100F300006F0C6FA3E4B00221A60E36A7BB1A16B51
:100F400069B9E3695BB13C4A136843B13B488368C4
:100F500043F0804383603A4B116001201860394FA1
:100F60003B6883B12F4B5B683BB137490B7801225B
:100F700003B91946354807F037FD00233B60344B71
:100F800040F6D8621A60334B1A68002A00F09F803E
:100F90001D4F00221A60D7F8B030A3F26C73FB61CA
:100FA000D7F8B430013BBB61D7F8B8307B61D7F8D4
:100FB000BC303B61D7F8C030FB60D7F8C430BB60B1
:100FC000D7F8AC303B62174B5B680BB108F086FD7D
:100FD000D7F8AC20D5F83080D7F8BC30D7F8C0109F
:100FE0003C2000FB03134146002004F0EDFD0028E7
:100FF00046D0B8F1000F2FD0012100202EE000BF15
:10100000240200203C020020D44600206C0F002067
:10101000A8010020B4010020640F0020A4000020DB
:101020008C0F0020980F00207CBE0008A5BB000894
:101030002C100020C8BA00085C01002000200140EC
:10104000840F0020D001002068000020CEBB0008E3
:1010500010000020500100204146012007F030FD23
:10106000DFF8A0E23060296BA448D7F8BC20D7F89D
:10107000C030002914BF71460146A14806F020FA8D
:10108000D7F8AC20D5F83480D7F8BC30D7F8C010EA
:101090003C2000FB03134146012004F095FD90B174
:1010A000B8FA88F0400907F049F9D7F8BC2093480E
:1010B000616BD7F8C030934F002914BF3946014601
:1010C000914806F0FDF933680BB9042333608F4B68
:1010D0001A68002A65D000271F602B6B002B60D098
:1010E0008B4B196840F6BA62914204D91968894855
:1010F00006F0E6F955E0884BDFF82892D3F8B410F3
:10110000D3F8B820D3F8B00002EB0128834A116865
:10111000884292460BD1824BD9F800901B68089305
:101120000023804ADFF8F0A19C46194612E0D3F86C
:10113000B0301360D9F800309F42ECD23846DAF86C
:10114000001004F045FB0137F4E7176CF80704D4EE
:10115000013144324945F8D11FE0DAF8C0B0D2F885
:1011600008E0BBFBFEF70EFB17B7002FF0D1576965
:1011700027B1B845ECD3506C8045E9D8F44508D385
:10118000E6D1002F089818BF0846089018BF012321
:10119000DEE70891F4460123DAE713B1604B089AC1
:1011A0001A60614BDFF888811A681AB300271F6044
:1011B0005E4B1B68F3B1D8F8009004F0F9FBC8B19E
:1011C000552004F0A9FB08F041FF442004F0A4FBE3
:1011D000B9F1000F0ED043F2154904F0BDFB013701
:1011E00010B94F45F9D103E043F215439F4201D1B5
:1011F00004F0DEFBD8F80030F3B14D4B00221A604A
:101200004A4B1B68B3B104F09FFC4A4B069010F0A8
:10121000010F494A4FEA500108BF1A46474806F0F5
:101220004FF9474B5B683BB1464B1720596808F0B4
:101230003BFC01E0FF230693434B1A68E2B1434FA6
:1012400000221A603B68ABB104F05CF9394B0490A2
:1012500010F0010F384A4FEA500108BF1A463C48C7
:1012600006F02EF9364B5B6833B1B968152008F0EB
:101270001BFC01E0FF230493294FDFF8EC90396851
:10128000DFF8E8A01F2900F2E68026484FF0440866
:1012900008FB010383465B68013B082B00F2D88002
:1012A000DFE803F0052666708C96A57E910008FBAA
:1012B00001011C31274806F003F93868264A08FB6B
:1012C00000F80BEB08011C3151F8103C2348042BAB
:1012D00098BF0523C2F8083C09F0C2F93B684FF0FB
:1012E000440808FB03B81E4BD8F80C201A60AFE086
:1012F0000123C9F800301B483EE000BFC2BD000812
:10130000D3BB0008FAC70008F2BB00085801002050
:10131000100000201BBC0008D4460020380200202A
:101320000400002090120020740F00203C1C0020BC
:10133000900F002030BD0008E0B700084BBC00084B
:10134000980F00208000002030100020A400002012
:1013500067BC00087FBC00085002002091BC000858
:101360001C0200209DBC0008C0010020940F00203A
:1013700001239D48CAF8003005F016FB9B4805F094
:1013800013FB65E0002008F0F7FA3B6898484FF03F
:10139000440808FB03B8974BD8F80C201A60EBE719
:1013A000012008F0E9FA3B6893484FF0440808FB35
:1013B00003B8904BD8F80C201A60DDE7022008F043
:1013C000DBFA8E48D8E7032008F0D6FA8C48D3E73A
:1013D00008FB01011C318B4806F072F8386808FBE5
:1013E00000B01C3008F09EFD0423336030E008FBA1
:1013F000010808F11C082F21404609F0D6FD09908C
:1014000010B3814BD3F8BC10D3F8C0303C2000FBA4
:1014100001334046089309F073FA099A8346501C39
:1014200009F06EFA089B8046184609F0CBF978B1AE
:1014300059464246754806F043F848EA0B2189B2FE
:101440000F2003F017F903E04146714806F038F821
:1014500020233B6015E06F4B1A6892B1511C08D1F4
:10146000AA6A72B9E26A62B16B4A126805321A60FE
:1014700007E0694909688A429FBF00221A60042375
:101480003360DAF80030BBB1644B00221A60069B6F
:10149000FF2B09D02B6B13B1069809F06BF95D4B4C
:1014A0004FF0FF321A6007E0049BFF2B04D02B6B38
:1014B000002BF4D00498F0E7D9F80030002B40D08E
:1014C000574BDFF89081504F0020186018F8013F0B
:1014D00093B31B2830DC592B1ED006D8442B0CD0DC
:1014E0004D2B1ED1BA69013208E06D2B0CD0792B3F
:1014F0000FD0642B15D17A6911E07A6949491BAB89
:10150000184409F01FFD13E00D2811DCBA690132FF
:1015100005E0FA69643AF1E7FA6902F26C7242494D
:10152000EDE73AAA104400F87C3C002300F87B3C2D
:101530001BA809F05AFDC9E71BA808F0F3FC042317
:1015400033603268394F002A35D06B682968013B17
:10155000994227D1364B1B6863B104F0F5FA354B3D
:10156000354A10F0010F80464FEA500108BF1A4675
:1015700032480EE0324B186870B103F0C3FF2D4BB8
:101580002D4A10F0010F80464FEA50012D4808BF48
:101590001A4605F095FF00E080463A68A8F114016C
:1015A000002004E0184BD3F8BC00D3F8C01005F0BD
:1015B00001F900233B60244B1A68002A00F0DC810B
:1015C00000211960214B1B681B78002B44D0204A56
:1015D000D5F86C021368013383421360C0F0CC81EC
:1015E000116006F063FEC7E1AABC00082EBD00082A
:1015F000BEBC00081C020020D3BC0008F1BC0008DF
:1016000001BD00081ABD0008D446002031BD000805
:101610004ABD0008700F002000020020940F002037
:10162000C0010020A2CD0008D3C00008380000206F
:101630003C1C002030BD0008E0B700086CBD00086D
:10164000A400002091BD0008F8010020B400002093
:101650004802002083460020AA6B002A79D0226B22
:10166000002A00F08981DFF8A4828DF86C30D8F868
:1016700000708DF86D308DF86E30002F3DD1DFF8A1
:10168000AC92BA4607F809A038461BA9013708F002
:1016900023FCB7F5806FF5D1954F02F003FD3B6851
:1016A000944AC3F120035B0813607B68924AC3F13C
:1016B00020035B0807F58160136009F096FC8F4BEF
:1016C000186007F6080009F090FC8D4B8D4A1860F1
:1016D000D7F8083C042B9CBF0523C7F8083CD7F873
:1016E000083C03F18063013B9B011360864B0022A1
:1016F0001A600123C8F800303EE1834B1F680137B0
:10170000FA071F601BD57F2F01D87B0806E07D4BB1
:101710001B68DB1B7F2B00F22F815B082A6905EB1E
:101720008202D2F8EC2108929A4280F06F84734BC7
:101730001B68002B40F06B8401E002F0B3FC714B9E
:101740001B689F42C0F01881704A00231360A36396
:1017500012E1636A0D2B20D8226B1AB9A26A0AB96A
:10176000E26AF2B9AA6A1AB1142202FB034312E038
:10177000E76AB7B9042B02D1D4F8A8300CE0644969
:10178000142000FB03430A68D86D013282420A60CC
:10179000C0F0F2800F609B6D9847EB6A002B00F061
:1017A000EB80EB68012B48D15A4AD4F880111368BA
:1017B0000133B3EB411F13604DD35748002313602F
:1017C0000368013B052B00F2A784DFE803F0030A5E
:1017D0001118222C95F849303E2B00F29D840133DC
:1017E00013E095F84830002B00F09684013B16E09A
:1017F00095F84A303E2B00F28F84013319E095F8BA
:101800004930002B00F08884013B84F8493000F017
:101810007FBC95F848303E2B00F27E84013384F87B
:10182000483000F075BC95F84A30002B00F0748405
:10183000013B84F84A3000F06BBC022B0BD1374AD5
:10184000374BD2F8BC001968884204D0D2F8BC20CB
:101850001A6004F0AFFEAB68032B69D1314AD4F8AB
:10186000D01113680133B3EB411F13606ED32E48C0
:10187000002313600368013B052B00F27084DFE84E
:1018800003F0030A1118222C95F84C303E2B00F27D
:101890006684013313E095F84B30002B00F05F8431
:1018A000013B16E095F84D303E2B00F25884013391
:1018B00019E095F84C30002B00F05184013B84F87E
:1018C0004C3000F06CBC95F84B303E2B00F2478456
:1018D000013384F84B3000F062BC95F84D30002B9A
:1018E00000F03D84013B84F84D3000F058BC00BF4F
:1018F00050020020BC0100207C0F0020C801002005
:10190000AC0100202C0200204C020020B00100207D
:10191000680F0020600E002014020020D446002032
:101920001400002064010020480100201440002021
:10193000042B0BD1A84AA94BD2F8BC0019688842E5
:1019400004D0D2F8BC201A6004F0DEFE2B6B9BB9E9
:10195000D4F83480B8F1000F0ED1A14F3B685BB1D1
:10196000A04BA1484FF480725A8305F01DF89F48A0
:1019700005F01AF8C7F800809D4B1A68002A00F09D
:101980000B81002119609B4B1F68A368013B012B51
:1019900000F20281636C984A9F4228BF0F46136889
:1019A000BB42964B4BD019606B6917600F2B28BF59
:1019B0000F2305EB83039249D3F82C2211A802F0E0
:1019C000EDFA904A9DF844309DF845109DF846E0A8
:1019D00012F813008C4B12F8111012F81E20187018
:1019E00059709A702B6A1B072CD51423DFF820C27C
:1019F000B0FBF3FEBEF1000F01D14FF0010ECCF8A9
:101A000000E0B1FBF3F3DFF80CE203B90123CEF8F9
:101A100000301423DFF800E2B2FBF3F303B9012333
:101A2000CEF80030794B4FF0000E83F800E083F8D9
:101A300001E083F802E0D87019715A7102E01A6867
:101A400001321A602B6A180735D57048704A6E4902
:101A5000D2F800C003780A7863449342D4BF03707D
:101A6000027043786B48694AD0F800E0487889787A
:101A700073448342D4BF53705070644B66489A7865
:101A8000006802448A42C8BF9970D978D8BF9A705A
:101A9000B1EB0C015D4A48BF0021D1701A795B4956
:101AA0005B79B2EB0E0248BF00220A711B1A574A3B
:101AB00048BF00235371AB68012B42D1002006F0D0
:101AC0002DFCD4F8B831990725D5636C3C2B22D175
:101AD000236A4C4A13F0040F12D0504B197832F895
:101AE00011108DF86C10597832F811108DF86D10B6
:101AF0009B7832F813308DF86E304FF0000801E01B
:101B0000474BEBE740461BA908F1050808F0C0F970
:101B1000B8F13C0FF6D12B6A1A0729D5002FBBBFAD
:101B2000606C3A493949C019A8BF384608F0B0F985
:101B3000781E45BF6B6C3B493A49C01808F0A8F9BC
:101B400026E0254BD3F8C080002006F0E7FB18F014
:101B5000010810D1474506D040462B4908F098F9B6
:101B600008F10108F6E72B6A1B0701D5274900E0B9
:101B700025493846E2E7236A180707D52949384638
:101B800008F086F96B6C01379F4201D21E49F6E7D7
:101B90006B6B0BB102F03CFA234B1A680AB10022BE
:101BA0001A601BA806F034FD002843D01F4A1368B2
:101BB000013313601E4A9DF87130116821B9D907AD
:101BC00002D50123136035E003F0010314211BA8A3
:101BD000136003F035FD2EE0D446002020000020E5
:101BE0006400002000080240B2BD00082EBD0008BD
:101BF0001002002040020020800F0020540100202D
:101C00005F440020B6BE0008080200203002002019
:101C10000C020020C4010020040200204400002027
:101C20000800002033020020F401002044020020BC
:101C300020020020FF20132800F20281DFE810F0CC
:101C4000140000011D0022002D0039003F00490052
:101C500055005F0090009F00A700AF00B900C100D1
:101C6000D800E800CB00FD00206BB0FA80F0012125
:101C7000400906F025FF3060E2E0206800B96068A6
:101C8000013806E094E80900013B984234BF013076
:101C90000020012104F024FC09E0636A0BB90D2344
:101CA00000E0013B636203F0FDF904F0E9FB04236B
:101CB0009CE0636A0C2B94BF01330023F2E7B54B21
:101CC000D3F8BC201AB1D3F8BC20013A0AE017229D
:101CD00008E0B04BD3F8BC20162A96BFD3F8BC203E
:101CE00000220132C3F8BC2014E0AA4BD3F8C02074
:101CF0001AB1D3F8C020013A0AE03B2208E0A54B14
:101D0000D3F8C0203A2A96BFD3F8C020002201326F
:101D1000C3F8C0200022C3F8C420042333609E4BC4
:101D20001B68002B00F08C809A4AD2F8B030A3F2E6
:101D30006C73D361D2F8B430013B9361D2F8B83000
:101D40005361D2F8BC301361D2F8C030D360D2F8FE
:101D5000C4309360D2F8AC30136208F00FF96FE032
:101D600094F84830002B40D0012B0CBF0023023BDD
:101D700084F8483004F000FC07F0AAFE35E094F83F
:101D800048303E2B31D80CBF3F230233F0E794F8A4
:101D9000493053B3012B0CBF0023023B06E094F8FB
:101DA00049303E2B21D80CBF3F23023384F8493001
:101DB000E0E794F84A30C3B1012B0CBF0023023B8B
:101DC00006E094F84A303E2B0FD80CBF3F23023375
:101DD00084F84A30CEE7E069704BB0FA80F0FF2219
:101DE000012140091A6004F05FFC0223336027E000
:101DF000E36943B1694BFF22012100201A6004F01E
:101E000053FC022333602B69002BEED0013B0EE024
:101E1000E36943B1614BFF22012100201A6004F005
:101E200043FC022333602B690E2BDED80133236180
:101E300004F0A2FB03F03EF9D7E7594B01221A60E8
:101E4000DFF874A102F078FCDAF80030002B3EF4E1
:101E5000E1AE544B1A683AB9012253481A6004F0B3
:101E6000A3FD524804F0A0FDDFF82881DFF850916F
:101E7000D8F8C020D9F800309A423EF4CBAED8F85A
:101E8000BC20D8F8C0304A493C2000FB0230D8F8CA
:101E9000AC20002751F8373013F0800F4FEAC70EFF
:101EA00007F1010738D08E44DEF804E0704533D1E5
:101EB000C3F3C20E03F007039E4506D1CEEB020E1C
:101EC000DEF1000343EB0E0318E00BD2724506D39C
:101ED0009A428CBF4FF0000E4FF0010E0DE04FF014
:101EE000000E0AE09A4206D9724534BF4FF0000E48
:101EF0004FF0010E01E04FF0010E734663B1D8F8C8
:101F0000AC102C48D8F8BC20D8F8C030009705F0A9
:101F1000D7FA47F440711DE0082FBBD1DAF814A0BE
:101F2000254FBAF1000F29D008F04CFC30B3BAF1BC
:101F3000010F40F05481D8F8C020164B7AB9D3F87D
:101F4000BC20D3F8BC100B2A00F23081FF2915D039
:101F500041F4807189B20F2002F08CFB0EE0D3F8BF
:101F6000C0200F2A00F02981D3F8C0201E2A00F0DB
:101F70002A81D3F8C0302D2B00F02B81D8F8C03047
:101F8000C9F80030FEF746BE0C4806F0BDFDFEF76E
:101F9000DFBB00BFD4460020A40000203C0000208E
:101FA000940F0020FC010020C6BD00082EBD0008D3
:101FB00068010020D9BD0008D40100200ABE000835
:101FC0000C000020934806F09FFDFEF71BBC9248D2
:101FD00006F09AFDFEF74ABC904B11605B68002B3F
:101FE0003EF4A1AE102007F05FFDFEF79CBE2A690B
:101FF0000B605B08934205D00F2B88BF0F23236132
:1020000004F0BAFA02233360FEF798BE0893BB08C7
:102010004FF00008DFF840B20C93CDF82480DBF8D5
:1020200000209045BFF489AB099B03F10809D9440E
:102030009A46099BDBF80420C3EB0A03934262D261
:10204000774A1268524505D999F80024402A01D9E7
:10205000413A00E00022734909688A4505D299F89F
:102060000018402901D9413901E04FF6FF710C9861
:10207000884238D20C99914240D3089A002A32D033
:1020800099F8002068480D93303A02EB420281181B
:10209000825C8DF83C204A788DF83D208A788DF856
:1020A0003E200FA9089A10A807F030FF5F4A9DF85C
:1020B00040100D9B32F811108DF844109DF841101E
:1020C00032F811108DF845109DF8421032F81120A9
:1020D0008DF84620564A1068564A1268404402EB72
:1020E000401011A907E0524A1068524A1268404451
:1020F00002EB40101BA9184407F0EEFE0AF1010A9A
:1021000009F1010995E708F10108CDF824A086E757
:1021100004F032FAFFF79FBB474B1A680132072AD7
:1021200000D101221A601B680360444844490268D8
:1021300001320D2A026004D10133072B0CD1012397
:102140000AE00E2A7FF487AB013B08BF06230B6031
:1021500000230360FFF77FBB0B60FFF77CBB394BAD
:102160001A680132072A00D101221A601B68036035
:1021700035483649026801320D2A026004D1013324
:10218000072B10D101230EE00E2A7FF4DFAB013BB9
:1021900008BF06230B6000230360FFF7D7BB04F0E2
:1021A00055FAFFF7D3BB0B60FFF7D0BB0C293FF408
:1021B000CFAED3F8BC100C39C8E6BB69D9077FF5A0
:1021C000DDAE0D21C4E6BB699A077FF5D7AE0E21BF
:1021D000BEE6BB695B077FF5D1AE0F21B8E6BAF169
:1021E000020F7FF4CBAEFB69002B3FF4C7AED8F8EB
:1021F000C010B1FBF3F203FB12131548002B7FF460
:10220000BDAED0F8BC10D0F8C020124805F058F987
:10221000B4E600BF36BE00084FBE0008980F00208D
:10222000C8010020AC01002098BE0008B6BE00081E
:10223000BC0100207C0F00202802002000000020AC
:1022400014020020CC01002048000020480100209A
:10225000D4460020F7BD0008500200202DE9F04FC1
:102260009BB007F0F5FF031F0790122B01F2478682
:10227000DFE813F0540A450E450EC009450E130061
:10228000870C9D0C450E450E450ED10C450E450E96
:10229000450E450E450E920CB70CB64C94F84C30DA
:1022A0004F2B00F0398515D8442B00F03C8407D81B
:1022B000412B00F0C184432B00F0E98401F01FBEE4
:1022C0004D2B00F0FE8400F2F780472B00F02886AB
:1022D00001F015BE612B00F0F38509D8532B00F0F7
:1022E000EB82542B00F09A83522B41F008862BE0AE
:1022F0006E2B00F08382742B00F0BF856C2B41F0B5
:10230000FE85022104F14D0002F00CFC022106467C
:1023100004F14F0002F006FC0221054604F15100D1
:1023200002F000FC0221074604F1530002F0FAFB20
:10233000914B03EBC60205EB0725556043F83600C9
:1023400002F06EFD01F0DBBD022104F14D0002F050
:10235000E9FB092801F2D385DFE800F00525454EA9
:10236000535898A99DA2854A936843F0804393608F
:10237000834B01221A600A2412A802F07BFD28B9BF
:102380000A2002F0CBF9013CF6D105E07D4BBDF807
:1023900048209A8006F0B8F87A4B1120998807F007
:1023A00083FB01F0ACBD754A936843F080439360B2
:1023B000734B01221A600A2412A802F05BFD28B9AF
:1023C0000A2002F0ABF9013CF6D105E06D4BBDF8F7
:1023D0004820DA8006F098F86A4B1220D98807F076
:1023E00063FB01F08CBD03F04BF9002801F08785F9
:1023F00003F0FAF801F083BD634B01221A6001F08B
:102400007EBD624B01221A6001F079BD604D01244E
:10241000604B14F0010F196814BF4FF0390E4FF0E4
:10242000000E14F0020F14BF3927002740F668523F
:1024300014F0040F14BF392600260023514303EB88
:1024400043020A44A8180133B3F58F6F05F802E080
:1024500047708670F3D101F0DBFD4FF47A7002F023
:102460005DF94FF47A7002F059F901344FF47A7043
:1024700002F054F9082CCBD1002001F0FBFE04F04F
:10248000E5F8454B04221A6001F039BD022007F03F
:1024900073FA01F034BD032007F06EFA01F02FBD8E
:1024A0003E4B00221A6007F063F801F028BD3C4B58
:1024B00001221A6001F023BD022104F14D0002F057
:1024C00031FB0221054604F14F0002F02BFB0221F3
:1024D000064604F1510002F025FB6B1E46EA00247B
:1024E0002D2B00F27481DFE813F00A0D0A0D2E0087
:1024F0005F0072016D008A00A6007201B200C40084
:10250000DA00E600F00000010A0D0A0D0A0D0F01C5
:102510000A0D0A0D26010A0D2F01720172017201C6
:1025200072010A0D3B003A010A0D72014601540185
:102530005A01600166016C0172017201720172013F
:1025400079017F018301174B1B6B9C4201F0D784FB
:102550000121204606F0B4FA0F4B186001F0CFBC01
:10256000104B5B6B9C4201F0CA84204605F0E6FEEE
:1025700001F0C5BC980F0020680100200020014038
:10258000840F002018000020D0010020940F0020AC
:10259000442500203C250020380000203400002085
:1025A000C001002014440020B34B1B689C4201F082
:1025B000A6840021204603F093FFB04B04221A604A
:1025C00001F09DBCAC4BDA691D4632B1AC4B002129
:1025D000FF2208461A6004F067F82A69A64B944265
:1025E00008D00F2C86BF0F221A611C6103F0C4FFB4
:1025F00003F026FFA14B02221A6001F080BC9E4D21
:10260000AB68033B012B04F0020605D926B12B6A07
:102610009F0701D403F092FF04F09AF82C620EB9E0
:1026200004F0B4F80123AB6203F03AFF934B0422A9
:102630001A6001F064BC924BFF221A6014B10021B1
:10264000012001E02146204604F02EF8D2E78A4B13
:102650005A6A944201F053840D2C02D85C6203F054
:102660000FFF884B00221A60844B04221A6001F08D
:1026700046BC814B9A68944201F04184042C09D8ED
:102680009C601B6A9C0701D404F080F804F060F899
:1026900003F074FE794B04221A6001F030BC772CF1
:1026A000754B8ABF78225C645A6404F0FDF803F02D
:1026B00055FE01F024BC762C6F4B8ABF00221C64AF
:1026C0001A6403F03BFE01F01ABC6B4D6B699C422F
:1026D00090D00F2C86BF0F236B616C6103F0B6FFA7
:1026E0006B69AB6103F05AFE84E7634BDA6894428E
:1026F00001F00584022C01F20284DC6003F07EFF0D
:1027000003F0AEFE01F0FBBBE005E5B248BF6D4251
:1027100029465D4804F0D4FE05F10C03182B01F2A4
:10272000EE835A4B5A69954201F0E9835D6102F0EC
:102730001BFD01F0E4BB564B5C6002F0AFFE554B55
:1027400001221A6001F0DBBB534B1C6002F006FE55
:10275000524A01231360524A136001F0D0BB102C7F
:10276000454B8ABF1022C3F86C42C3F86C2203F0B9
:102770004BFD01F0C4BB4B4B4B489C60214604F021
:102780009FFEA1B2062001F075FF01F063FF01F08A
:10279000B6BB444BDC6001F049FF01F0B0BB414BDC
:1027A0001C6101F02FFF01F0AABB3E4B5C6101F000
:1027B00019FF01F0A4BB3B4B9C6101F003FF01F04A
:1027C0009EBB384BDC6101F0EDFE01F098BB224668
:1027D0002946364804F074FE01F091BBA1B20F20E7
:1027E00001F048FF01F08BBB314B1C6001F087BB4F
:1027F000304B1C6003F080F801F081BB022104F132
:102800004D0002F08FF90221064604F14F0002F05C
:1028100089F90221054604F1510002F083F91EB145
:10282000012E15D001F06BBB3F2D01F268830F28FC
:1028300001F26583104B03EB8505C5F8EC0103F04D
:1028400009FD03F099FE0D4B02221A6001F057BBFF
:102850003F2D01F254830F2801F25183064B03EB05
:102860008505C5F82C0203F0E1FC03F0EFFE034BF5
:1028700002221A6001F043BB1444002038000020FB
:102880003C000020F801002043BF00086800002041
:10289000A40000203010002080000020740F0020D1
:1028A000900F0020D401002056BF000870BF000820
:1028B0000400002090120020022104F14D0002F0DB
:1028C00031F90B2801F21B83DFE810F01200190B1D
:1028D000190B190B1A002A0037000F000C007B009F
:1028E00084009600C54B2E2152E0C44B2E2136E0C9
:1028F000C34807F017FBC34B04221A6001F0FFBA6C
:10290000BF49C14808F069FBC04B1B68002B01F0B0
:10291000F6821022BC49AA2007F0BCFE01F0EFBAF3
:102920002022B749BA4808F07DFB2022B84940F27E
:10293000471007F0AFFE01F0E2BA2022B049B548D7
:1029400008F070FBB14B1B68002B01F0D8822022ED
:10295000B04940F2671007F09DFE01F0D0BA13F8BD
:10296000012F1AB12C2A08BF1970F8E70822A449D0
:10297000A94808F057FBA54B1B68002B01F0BF824C
:102980000822A54940F2871007F084FE01F0B7BA8B
:1029900013F8012F1AB12C2A08BF1970F8E7082282
:1029A00097499E4808F03EFB984B1B68002B01F0AE
:1029B000A6820822994940F28F1007F06BFE01F0C1
:1029C0009EBA3F228E49964808F02CFB06F0A2F8EA
:1029D00001F095BA3F228A49924808F023FB8B4BBD
:1029E0001B68002B01F08B8240228E4940F23F2071
:1029F00007F050FE01F083BA052281498A4808F0A9
:102A000011FB8A49002381F87532062201F51C71F9
:102A100040F2A57007F03EFE01F071BA022104F108
:102A20004D0002F07FF8002841F0698294F84F20B1
:102A30007F4DA2F1300394F850206421303A4A438C
:102A40004FF47A7101FB032294F851100A233039B4
:102A500003FB012194F85220303A0A4494F85310B1
:102A6000EA61A1F1300094F85410303903FB0011F1
:102A700094F85500A961A0F1300694F8560030385A
:102A800003FB060094F857606861A6F1300794F8DC
:102A90005860303E03FB07662E6194F85960A6F13A
:102AA000300794F85A60303E03FB0766EE6094F8F6
:102AB0005B6094F85C40303E303C03FB064302F21E
:102AC0006C720131AB6002F051F85A4B28621B68FE
:102AD0002C460BB107F052FAD4F8BC102269544BC3
:102AE000914204D1D3F8C010DB68994202D0454B23
:102AF00004211960E36903F26C73C4F8B030A36970
:102B00000133C4F8B4306369C4F8B830236AC4F838
:102B1000AC30E368C4F8BC20C4F8C030A368C4F883
:102B2000C43001F0ECB9022104F14E0001F0FAFFCB
:102B300094F84D50432D074641F0E181022104F104
:102B4000500001F0EFFF0221C5B204F1520001F084
:102B5000E9FF0221C6B204F1540001F0E3FFC0B264
:102B6000AFB93F2D28BF3F253F2E304B28BF3F2612
:102B70003F2828BF3F2083F8485083F8496083F8F6
:102B80004A0003F0F9FC03F0C1FC01F0B8B9012FD1
:102B90001BD13F2D28BF3F253F2E244B28BF3F266A
:102BA0003F2828BF3F2083F84B5083F84C6083F8C0
:102BB0004D0083F84E5083F84F6083F8500003F0C7
:102BC00045FD03F015FC01F09AB9022F41F0978101
:102BD0003F2D28BF3F253F2E144B28BF3F263F28BF
:102BE00028BF3F2083F8515083F8526083F8530088
:102BF00003F01AFD03F0E2FB01F081B9E60F0020BB
:102C0000E70F002038000020680000203825002051
:102C1000D0240020F1240020122500201B250020B4
:102C20000047002040470020844600201444002034
:102C3000D4460020A4000020022104F14E0001F03F
:102C400071FF94F84D60442E054611D0462E41F098
:102C50005681022104F1500001F064FFAA4A1423B6
:102C600003FB05235866284603F048FB01F047B9EB
:102C7000022104F1500001F055FFA34A142303FB85
:102C80000523D865284603F039FB01F038B9022145
:102C900004F14E0001F046FF94F84D60442E0546C5
:102CA00041F02D81022104F1500001F03BFF964BD1
:102CB00003EB0513C3F87001284603F003FB01F092
:102CC0001EB9022104F14E0001F02CFF94F84D6072
:102CD000442E054611D0462E41F01181022104F107
:102CE000500001F01FFF884B03EB0513C3F8A80148
:102CF000284603F0C3FA01F002B9022104F15000A2
:102D000001F010FF804B03EB0513C3F8A001284628
:102D100003F0B4FA01F0F3B804F14E00022194F884
:102D20004D5001F0FFFEA5F143030446162B01F2BE
:102D3000E680DFE813F044003500E4088700E4088B
:102D4000E4082600E408E408E408E4087400E40861
:102D5000E408E408E40853001700E408E408E40881
:102D6000E40862000221694801F0DCFE684A136849
:102D70009C4281F0C480442303FB0424606001F082
:102D8000BEB80221614801F0CDFE614A13689C4241
:102D900081F0B580442303FB0424A06001F0AFB8A8
:102DA00002215A4801F0BEFE594A13689C4281F044
:102DB000A680442303FB0424E06001F0A0B80221B4
:102DC000524801F0AFFE524A13689C4281F097804E
:102DD000442303FB0424206101F091B804214B48F3
:102DE00001F0A0FE4A4A13689C4281F08880442387
:102DF00003FB0424606101F082B80221434801F022
:102E000091FE434A13689C4281F079804423002854
:102E100003FB042408BF0120A06101F070B83C4D01
:102E20002B68984281F06B8044235C432819202250
:102E300036491C302C4408F0F5F8002384F83C3067
:102E400001F05DB8324D3148022101F06BFE2B6874
:102E50009C4206D2442303FB04531864204602F02C
:102E60000DFD2C4BD3F8B0102B689C4281F04780AD
:102E7000204602F0ADFC01F042B8022104F14D0001
:102E800001F050FE0221064604F14F0001F04AFE17
:102E90000221054604F1510001F044FE02210746DB
:102EA00004F1530001F03EFE1B4B03EBC60205EBA1
:102EB0000725556043F8360002F0C8FE01F01FB840
:102EC000022104F14D0001F02DFE0221064604F11D
:102ED0004F0001F027FE0221054604F1510001F0E8
:102EE00021FE0221074604F1530001F01BFE0B4BAB
:102EF00003EBC60205EB0725556043F8360002F0E8
:102F0000A5FE00F0FCBF00BF14440020E80F002025
:102F100090120020D4460020FC1B0020641C0020DE
:102F200094F84D30532B00F0F381542B40F0E78799
:102F300094F84E30732B40F0E287DFF80C83BF4FDC
:102F4000BF4E0025D8F81020BE4C79190AA806F00B
:102F5000DDFF9DF8282034F81220AA559DF829207D
:102F6000AB1934F812205A709DF82A20033534F832
:102F700012209A70152DE5D1B34BB4491A690AA8ED
:102F800006F0C4FF9DF82820B14B34F812201A70C7
:102F90009DF8292034F812205A709DF82A2034F820
:102FA00012209A70AB4B00241C705C709C70204601
:102FB000A849013406F090FFB4F5806FF7D140F2D4
:102FC000EA3440F2F5362046A149013406F084FF88
:102FD000B442F8D1A04E00274FF07C08A5F10B00B9
:102FE00037607760B7609A4906F076FF86F8008010
:102FF0002846974906F070FF203540F215439D4260
:1030000086F80B804FF0000406F10C06E6D1934ED3
:10301000934D32680723B2FBF3F3C3EBC303D31A18
:10302000904A85E81800D35C0120C3F10202AA602F
:10303000C3F10C03022293FBF2F3EB6002F000F900
:10304000322304930123039402930896A94601F0C6
:1030500029F8854D002607F0FBF809280ED195F8D0
:103060004C30472B0AD195F84D30542B06D17E4B6E
:1030700093F84E30712B00F03B8107E00A2001F0FD
:103080004DFB049B01369E42E5D140E06D2B35D0CF
:1030900007D8642B2FD06C2B39D1714EF568013DC8
:1030A00007E0722B02D0752B0FD030E06C4EF56824
:1030B00001352A46B168706802F08AF80028C6D047
:1030C000002002F0BDF8F56011E0654B5D68DA683C
:1030D0009968032D14BF01350025284602F078F8C1
:1030E0000028B4D0002002F0ABF85D4B5D600120F9
:1030F00002F0A6F8ABE702F0DFF8A8E702F0DCF890
:1031000028B100F0CFFF322001F008FBF6E702F013
:10311000D3F800289BD1524A4F4FD36811680693C9
:103120005368966803EB810301F1010B4F490C22B0
:1031300001EB830A02FB06F35FFA8BFB05934FF06A
:103140000108069BC518059B591908FA00FE394469
:1031500000231AF803C01CEA0E0F0AD006EB030C7A
:10316000BCF11F0F05D80B2D9CBF02FB03FC01F81F
:103170000CB00133042BECD101300428E1D100263E
:103180001E2501273946284602F010F8002846D0AF
:1031900001370B2FF6D1364B4FF00C0808FB0533E7
:1031A0006F01059307F10B0301360693A846B8F1AA
:1031B000000F27D0DDF818A0DDF814B001271BF8A8
:1031C000012F8BF80C2039464046099201F0EEFFA2
:1031D00030B1099A1A4B013A02EB4201194400E05E
:1031E0001C495046013706F077FE0B2F0AF1010A01
:1031F000E5D1059B0C3B0593069B203B08F1FF386E
:103200000693D4E70B27144B12493B44384603F886
:103210000A8C013706F060FE152FF4D1013515F147
:10322000FF35AED2002E3ED0022E05D0032E21D087
:10323000012E22D1282322E0642320E0D9C00008F7
:10324000DC1B0020B6BE00081444002036BF000876
:1032500040100020611C0020101100204C010020B3
:10326000441C00203CBF0008980F002031C8000813
:10327000041100204FF4967301E04FF49663029A14
:1032800003FB0244039B3344092B039309D9029B9C
:1032900001330293049B092B84BF053B0493002355
:1032A000039300F0FFFE089B1A680723B2FBF3F3B9
:1032B000C3EBC303D31A0022C9F80420B24AC9F8E9
:1032C0000030D35C0120C3F10202C9F80820C3F129
:1032D0000C03022293FBF2F3C9F80C3001F0B0FFAB
:1032E00009F1040007C801F073FF00287FF4AFAEB6
:1032F000C82001F013FA2246A44912A807F022FEC2
:1033000012A806F00FFEA24B04221A6000F0F7BDCF
:10331000A04B93F84E30732B40F0F1859E4D9F4E9D
:103320009F4932699F4CDFF8A0A2284606F0EEFDC7
:103330002A789D4B34F812201A706A789B4934F829
:1033400012205A70AA789A4D34F812209A702846A2
:10335000326906F0DBFD2A78964B34F812201A7099
:103360006A78954934F812205A70AA7834F81220F5
:103370009A70924A0023137053709370904A0B60B6
:103380001E2313608F4B02920120186088469946D5
:10339000D3460023FF20002203EB0A0188540132A8
:1033A000202AFBD12033B3F5806FF4D1864B864AB7
:1033B000002483F86240FE2382F84230834B0322CC
:1033C0001A70834B02251D70824B20461D6001F050
:1033D00089FF012001F086FF284601F083FF204687
:1033E0007649013406F078FDB4F5806FF7D10326F5
:1033F000764B1C78764B1D7823462F465A01D01900
:1034000069490493039206F067FD039A049B5244B2
:10341000D25D032A0AD8DFE802F002040608013B65
:1034200004E0013302E0013F00E0013758010BEBFB
:103430000002D25DFE2AE1D138445B4906F04CFD22
:10344000654A664B002717F802E0F85C5949049278
:1034500000EB4E100137039306F03EFD032F039B54
:10346000049AF0D100F01EFE0027029B1A689742D2
:1034700031D206F0EDFE09281BD1464B93F84C20C3
:10348000472A16D193F84D20532A12D193F84E3083
:10349000712B00F0158504D8642B17D06C2B0DD040
:1034A00019E0722B0DD0752B15D1711E4E424E4175
:1034B00011E00A2001F032F90137D6E7032E15D1C9
:1034C0001AE0022E00F0DB84032615E0002E00F047
:1034D000F784012608E0022E09D0032E0CD0012E1D
:1034E00002D0013C621C04E0013406E00226013DEA
:1034F0006B1C00F0E58400E001351F2C00F3E08434
:103500001F2D00F3DD840AEB44125319525DFF2A8C
:1035100040F0D6842D4A14702D4A022E157006D024
:10352000032E06D0012E14BF0122002202E0032246
:1035300000E002221A700020274B1B5C9C4204D141
:10354000264B1B5CAB4200F09D8401300328F3D175
:1035500062010BEB02035B5D032B0BD8DFE803F08A
:1035600002040608013C05E0013403E06B1E02E0A2
:103570006B1C00E02B4660010BEB0001CF18C95C0F
:10358000FE292DD01D46E3E73CBF000896BF00088A
:1035900038000020980F0020641000201444002000
:1035A000D6C00008B6BE00083810002039BF000899
:1035B00043100020581000204C1000206C100020F8
:1035C0007810002050100020A81C00207D10002042
:1035D0007C1000205C100020F81B00208C1B0020B9
:1035E0005A44FF243C7018445155444906F074FC79
:1035F00000F055BC0A220AA9414807F07DFC414B66
:10360000414A5B6902444FF461611AAC01FB032338
:1036100044F8203D204607F08BF90369DA1E052A9D
:10362000054640F24384022B0CD18269C3689B1A81
:10363000182B14DD002A40F039848368012B00F335
:1036400035840CE0092B0AD18269C3689B1A182BB8
:1036500040F32C841AB98368022B40F327842B4C47
:103660006B69E3612B69A361EB68636129696A692E
:10367000E86802F26C72013101F078FA20622B6A7C
:10368000A362AB6823616B68E3602B68A360204B87
:103690001B680BB106F072FCD4F8BC1022691B4BFE
:1036A000914204D1D3F8C020DB689A4204D006F0DE
:1036B00015FA184B04221A60E369174A03F26C7377
:1036C000C4F8B030A3690133C4F8B4306369C4F8F6
:1036D000B830236AC4F8AC302369C4F8BC30E3685E
:1036E000C4F8C030A368C4F8C430D4F8C430C3F5FB
:1036F0006E630C33136000F002BC00BF6C1000203E
:10370000E40F0020680000208081557CD446002012
:10371000A40000203800002010000020B24AB34965
:10372000B34DB44CB44E0AA807F00CFCAE49B348F4
:1037300003F0C6FE03F030F90021084606F0B4F9A4
:10374000AF4B0120196806F0AFF9AE4B1D20D988A8
:1037500006F0AAF92968022006F0A6F9216B0320D9
:1037600006F0A2F9616B1E2006F09EF92168042084
:1037700006F09AF901F09EFC216A072006F094F900
:10378000E169082006F090F901F08CFCA1680B209B
:1037900006F08AF9616C0C2006F086F9216C0D2088
:1037A00006F082F961690E2006F07EF9E1680F20CB
:1037B00006F07AF97188102006F076F9B1881120A8
:1037C00006F072F9F188122006F06EF98E4B5969F5
:1037D0000029BDBF494289B241F4807189B21320EA
:1037E00006F062F9894B1420196806F05DF9A968A2
:1037F000152006F059F96968854D162006F054F930
:103800006968172006F050F929687A4D182006F0EB
:103810004BF9D4F86C121F2006F046F97D490120BF
:1038200006F032F97749022006F02EF97649042095
:1038300006F02AF97849052006F026F9774906208E
:1038400006F022F97649072006F01EF9754908208E
:1038500006F01AF97449092006F016F973490A208E
:1038600006F012F972490B2006F00EF906F036F94F
:1038700006F02EF96F49012001F03EFC6E4902204E
:1038800001F03AFC2E460024726D6C48214601F08E
:1038900047FCF26D6A48214601F054FC326E6948DB
:1038A000214601F04FFC726E67482146013401F059
:1038B00049FC0E2C06F11406E6D14E4E0024D6F833
:1038C0006C216248214601F02BFCD6F8702160483B
:1038D000214601F037FCD6F874215E48214601F0FC
:1038E00031FCD6F878215C482146013401F02AFCED
:1038F000032C06F11006E2D10024D5F89C2157488C
:10390000214601F00DFCD5F8A0215548214601F0D3
:1039100019FCD5F8A4215348214601F013FCD5F831
:10392000A82151482146013401F00CFC052C05F179
:103930001005E2D14D4E35462E2055F81C1B06F0E1
:10394000B3F80024374633689C4280F0A38055F8D2
:10395000182C4748214601F0F5FB3B689C4205D2F4
:1039600055F8142C4348214601F0ECFB33689C4287
:1039700005D255F8102C4048214601F0E3FB33688E
:103980009C4205D255F80C2C3C48214601F0DAFB4C
:1039900033689C420BD235F8083C0093384A3949C9
:1039A000234612A807F0CEFA12A801F08BFB336869
:1039B0009C4205D255F8042C3348214601F0C2FB45
:1039C00033689C4204D22A462146304801F0A8FBC5
:1039D00033689C4204D26A6A2D48214601F0B2FB4A
:1039E00001344435AFE700BFD40F0020A2BF000868
:1039F000A40000201444002018000020A8BF0008E4
:103A000038250020D4460020680000203C1C0020FF
:103A100080000020B6B80008D0240020F124002047
:103A2000122500201B2500200047002040470020D1
:103A3000844600205F44002065440020C0BF000889
:103A4000C3BF0008C6BF0008C9BF0008CCBF00083C
:103A5000CFBF0008D2BF0008D5BF0008D8BF0008FC
:103A6000DBBF0008DEBF0008E1BF000890120020A5
:103A7000E4BF0008E7BF0008EABF0008EDBF000888
:103A8000F0BF0008F3BF0008FEBF000801C0000837
:103A900004C00008B74D002405EBC40355F83420DA
:103AA0005B680192C3F307220092DBB22246B2495F
:103AB00012A807F047FA013412A801F003FB082C02
:103AC000EAD1AE4D002405EBC40355F834205B6801
:103AD0000192C3F307220092DBB22246A84912A842
:103AE00007F030FA013412A801F0ECFA082CEAD100
:103AF000A44CA549A54D002006F090FAA449012048
:103B000006F08CFA2168202005F0CEFF61682120A4
:103B100005F0CAFFA168222005F0C6FFE168232056
:103B200005F0C2FF2169242005F0BEFF6169252050
:103B300005F0BAFFA169262005F0B6FFE16927204C
:103B400005F0B2FF002405EBC40355F834205B6890
:103B50000192C3F307220092DBB222468D4912A8DC
:103B600007F0F0F9013412A801F0ACFA082CEAD100
:103B700002F012FF0AA806F0D5F9874B04221A605A
:103B8000BDE18649864803F09BFC844806F0CAF9EB
:103B9000814B04221A60B2E18049824803F090FC14
:103BA0007E4806F0BFF97C4B04221A60A7E17E4BE9
:103BB0007E4893F84C2093F84D308DF8493012A987
:103BC00000238DF848208DF84A3003F079FC784BBB
:103BD00078481A68784B12A9C3F8082C06F040FD03
:103BE0008DE1714B754893F84C2093F84D308DF86A
:103BF000493012A900238DF848208DF84A3003F08F
:103C00005FFC6B4B6B481A686B4B12A9C3F8082C0E
:103C100006F026FD73E16A4D0295D5F80080694CE7
:103C2000DFF8C8B1DFF8C8A1674DB8F1000F0DD0BB
:103C3000D4F80090DBF80070DAF80060574CDFF839
:103C40009CA1DFF8A0B1DFF8708149E00221534860
:103C5000594E00F067FF0221814630605B4800F05A
:103C600061FF042107467060594800F05BFF0421A2
:103C70002060584800F056FF0421CBF80000564859
:103C800000F050FF554B564AC3F80080554BCAF818
:103C9000000007FB09F11160C5F80080C3F800803F
:103CA000B9F1000F00F0CE80002F00F0CD8000228F
:103CB0004D48114604F098FE0120C6E02A684A45A6
:103CC00012DAB2F5806F0ADA3F4B0392511C196089
:103CD0002046022100F026FF039A4244107202346B
:103CE0002278002AEAD127E0DAF80020BA420FDA77
:103CF000B2F5806FF3DA511CCAF800102046022199
:103D0000039200F00FFF039A424482F80804E6E7AA
:103D1000DBF80020B242E2DAB2F5806FDFDA511C44
:103D2000CBF8001020460221039200F0FBFE039A1C
:103D3000424482F80808D2E7184B9C420AD0274A2E
:103D4000296812681144274A12684F443E440A44C5
:103D50009642ACD122492A680868174C00210E46C9
:103D6000904247DDB2F5806F44DA01321119CE710D
:103D70000121F5E7FC1B002007C00008641C00209F
:103D800019C00008D401002000460020680100206E
:103D9000404600202BC0000838000020E40F00201F
:103DA0003DC0000852C00008980F002070C00008F5
:103DB0001C02002088C000085002002097C00008A4
:103DC000741000205410002070100020E60F002016
:103DD000E80F0020EC0F0020F00F002068100020FA
:103DE0003410002048100020CEBC00083C100020F9
:103DF0006010002001B12A60434A444C136800213E
:103E00000E46984208DDB3F5806F05DA01331919C3
:103E100081F807640121F4E701B113603C4A3B4C8F
:103E2000136800210E46984208DDB3F5806F05DA6D
:103E30000133191981F807680121F4E701B1136012
:103E4000022002E0484600E03846029B029A1B68C6
:103E50000133136030B92F4802F0A6FD2E4802F05E
:103E6000A3FD4CE002284AD12C4B01229A632C4B33
:103E70001A682C4B1B6813442B4A13603FE0002642
:103E8000FFF72FBBD8F80020D9F800301344274A99
:103E9000C8F8003013680133136001F023FA234B94
:103EA0001B68B3F57F7F7FF6A3AA19E0129B20461B
:103EB00003F56163129306F03BFD0546FFF7CFBBA8
:103EC000C82000F02BFCD8F80020194912A807F0F0
:103ED00039F812A806F026F8164B04221A600EE0F4
:103EE000029B1B680A2B7FF654AAD9F800200132E6
:103EF000C9F80020104A0A3B1360FFF74ABA079836
:103F00001BB0BDE8F08F00BF6810002050020020F9
:103F100048100020B8C000082EBD0008144400203E
:103F2000000200201C020020700F00205C10002006
:103F3000CBC00008380000207810002010B50B49D5
:103F40000B680A4A002BFBD0094B0A4C1868411C2D
:103F50002029205C196004BF00211960C0B272B62C
:103F60001368013B136062B610BD00BFD010002083
:103F7000AC100020E4100020074A02F5806112F81E
:103F8000013F98074CBF43F0080323F008038A421F
:103F90001370F4D1704700BF134000200B7810B5A8
:103FA00053430F24B3FBF4F3DBB203700C7814B16A
:103FB0000BB9012303704B780F245343B3FBF4F385
:103FC000DBB243704C7814B10BB9012343708B788A
:103FD0005A430F23B2FBF3F2D2B282708B7813B143
:103FE0000AB90123837010BD084B10B503F580603A
:103FF000012413F8011F01F00201002901F0FF0262
:1040000018BF224683421A70F3D110BD134000201E
:10401000034B5B6B1BB14FF48F6005F005BC704721
:1040200014440020F0B40E4B0E4E1C6840F668524B
:104030004FF48063544303EB430222440778B754A0
:10404000B51842786A7001338278AA70B3F58F6F21
:10405000F1D111B1F0BCFFF7DBBFF0BC704700BF7E
:104060003C2500204425002007B50C4A0C4B117854
:1040700033F811108DF804105178927833F811103C
:104080008DF8051033F812308DF80630014601A87E
:10409000FFF7C8FF03B05DF804FB00BF88000020F5
:1040A000B6BE00084FF4806005F0BEBB30B568496D
:1040B0008B6A85B03BB300238B62CB62654B66484D
:1040C0001C781422B4FBF2F20AB904B10122026096
:1040D000624D58781422B0FBF2F20AB900B1012205
:1040E0002A609A785E4D1423B2FBF3F30BB902B148
:1040F00001232B605B4B00251D705D709D705A4B3A
:104100001C7058709A70CC6A002C40F09E80524B04
:104110001A68BAB1544803789A4202D89B1A0370BD
:1041200001E00BB1047001234E484A4C0578247815
:104130002A44A24201D8027002E0A54203D00470D2
:10414000012300E01346454A1268BAB1464C607834
:10415000824202D8801A607002E010B100236370BE
:10416000012340483B4C457864782A44A24201D858
:10417000427002E0A54201D044700123384A12681F
:10418000BAB1394CA078824202D8801AA07002E0FD
:1041900010B10023A370012332482E4C8578A478F7
:1041A0002A44A24201D8827007E0A54201D084705F
:1041B00003E013B90123CB6247E0264A2B4B117869
:1041C0002B4D33F811108DF804105178927833F894
:1041D000111033F812208DF80620224A8DF80510B0
:1041E000117833F811108DF808105178927833F85F
:1041F000111033F812208DF80A201B4A8DF809108F
:10420000117833F811108DF80C105178927833F83A
:10421000111033F812308DF80D108DF80E30002487
:10422000635D022B01D102A906E0012B01D103A994
:1042300002E0032B03D101A9204605F04DFE013415
:10424000B4F5806FECD1FFF72DFF05B030BD00BF96
:104250001444002044000020B41000200C11002061
:10426000E0100020CC10002004110020B6BE000891
:104270001440002073B5224B1A6806460AB901267D
:104280001E60204A204B1178204D33F811108DF814
:1042900004105178927833F8111033F812308DF8F9
:1042A000051000248DF806308DF800408DF801408F
:1042B0008DF8024015F8013F9B0707D501A920465C
:1042C00005F00AFE2B7843F0010306E0694620461C
:1042D00005F002FE2B7823F001030134B4F5806F62
:1042E0002B70E7D10A4C2EB1A3681BB90120FFF750
:1042F000BBFE01E0FFF7D6FE0123E36202B070BD12
:104300008010002044000020B6BE000813400020AA
:104310001444002010B5054CA36A1BB10020A06214
:10432000FFF7A8FF0123E36210BD00BF1444002083
:1043300073B5154A154B1178154E33F811108DF8D9
:1043400004105178927833F8111033F812308DF848
:104350000510002405468DF806308DF800408DF8D4
:1043600001408DF80240A35D2B4214BF01A96946AC
:104370002046013405F0B0FDB4F5806FF3D1FFF7AE
:1043800091FE02B070BD00BF44000020B6BE000820
:1043900014400020F8B57B4C7B4DA36A5BB106F05E
:1043A00053FC7A4B0340002BBEBF03F1FF3363F095
:1043B000030301332B602B68032B00F2E280DFE85C
:1043C00003F0023772A6A36A6E4A23B100239362F8
:1043D000D3626F4A1360E26A002A40F0D2806C4BCD
:1043E00018681F2856D86B4E471C1F60B646931995
:1043F0000021151A6C188F42744404D814F8014C2B
:1044000014F0010F02E0E47F14F0020F1C7801F1B8
:10441000010114BF44F0080424F0080420291C7092
:1044200003F10103E6D12032B2F5806FDFD12CE039
:10443000A36A544A23B100239362D362564A13609D
:10444000E26A002A40F09D80534B18681F2821D84B
:10445000461C504F1E602130D419234631461F2977
:104460001BD8655C15F0010F1D7801F1010114BF27
:1044700045F0080525F0080581421D7003F1010390
:10448000EDD12032B2F5806FE6D10820BDE8F840CA
:10449000FFF74EBF0123E362F8BD651815F8205CF5
:1044A00015F0020FE0E7A36A364A23B100239362B6
:1044B000D3623A4A1360E26A002A62D1374B1D6820
:1044C000B5F5806FE6D205F1200632481E6002F194
:1044D0002004131827189642A3EB050104D811F8FD
:1044E000201C11F0010F03E091F8E01311F0020F0E
:1044F000197814BF41F0080121F008011970013347
:10450000BB42E8D1B4F5806F2246E0D1BDE7A36A93
:104510001C4A23B100239362D362214A1360E36AE9
:104520007BBB1F4B1868B0F5806FB3D200F120023F
:10453000184C1A60A0F5806E2022A2F120030EEB29
:1045400002012344214417191618B6F5806F04D2CE
:1045500091F8005415F0010F02E00D7815F0020FEC
:104560001D7814BF45F0080525F008051D700133BE
:104570009F4201F10101E8D12032B2F5846FDCD114
:1045800083E7F8BD14440020B01000200300008031
:10459000C010002014400020C8100020DC100020B3
:1045A0000811002007B5064B02A9DB6901F8043D9C
:1045B000012240F2872006F06DF803B05DF804FB9D
:1045C000D401002007B5064B02A99B6901F8043D00
:1045D000012240F2862006F05DF803B05DF804FB8E
:1045E000D401002007B5064B02A95B6901F8043D20
:1045F000012240F2852006F04DF803B05DF804FB7F
:10460000D401002007B5084B1B698DF80430022245
:104610001B0A01A940F283208DF8053006F03AF814
:1046200003B05DF804FB00BFD401002007B5084BC0
:10463000DB688DF8043002221B0A01A940F28120B8
:104640008DF8053006F026F803B05DF804FB00BFD6
:10465000D401002007B5064B02A99B6801F8043D70
:1046600001224FF4207006F015F803B05DF804FB4A
:10467000D40100202DE9FF417E238DF80430FF2373
:104680008DF8053006230A0A8DF8063000238DF8D0
:1046900009208DF807008DF808308DF80A100122E6
:1046A00001AD515D01320B44072A9BB2F9D15B4247
:1046B0009BB21A0A8DF80C30144E1549DFF858E0F9
:1046C00014488DF80B20EF238DF80D30002334466D
:1046D0009C4615F8038032681F2AFCD80F687A1CA4
:1046E0001F2A0A600EF8078088BFC1F800C072B6A2
:1046F00022680132226062B60268013342F0800211
:104700000A2B0260E5D104B0BDE8F081D41000208E
:10471000C41000200C10014085100020044B1B68C1
:104720005843044B18601A68002AFCD1704700BF38
:10473000A0000020F41B0020F0B58C4B1B68092B57
:1047400085B05BD9FFF7FAFBC0B27E288DF8040074
:1047500054D1FFF7F3FB8DF80500FFF7EFFBC0B274
:1047600006288DF8060049D1032401ADFFF7E6FBCA
:10477000285501340A2CF9D100230122A95C013209
:104780000B44072A9BB2F9D19DF80B109DF80C2021
:104790005B429BB242EA0122934202D0744802F08B
:1047A0008FFE9DF80D30EF2B28D19DF807309DF836
:1047B00009109DF80A206F4E6F4D70483D2B42EA5C
:1047C00001241DD17768052F05D12F683D2F17D102
:1047D0000768BC4214D1FF232B604FF6FF730360C0
:1047E000674D684B2C781A78A24240F26A814FF4E8
:1047F00000710F200134FFF73DFF2C70002062E1B3
:104800002B603A3B0460132B00F21681DFE813F0B3
:10481000140023002C002F003200350055006700E3
:1048200069006D007000850095009B009E00A1004E
:10483000A400A700AA001001012C01D1524802E0F7
:10484000022C06D1514802F0AFF8514802F0ACF802
:10485000F2E05048F7E7012C01D14F48F3E7022C72
:104860000CBF4E484E48EEE721464E48E2E0214656
:104870004D48DFE021464D48DCE00CB94C48E2E70A
:10488000E00705D54B4802F08FF8414802F08CF85C
:10489000A10705D5484802F087F83D4802F084F8A2
:1048A000620705D5454802F07FF8394802F07CF8E8
:1048B000230740F1C1804248C5E7062C0DD8DFE848
:1048C00004F00406080C0C0C0A003E48BBE73E4806
:1048D000B9E73E48B7E73E48B5E73E4802E03E4804
:1048E000B1E73E4802F0ECFDA6E021463C48A1E0DD
:1048F000052C10D8DFE804F0030507090B0D394833
:10490000A1E739489FE739489DE739489BE739488F
:1049100099E7394897E7394895E7032C0BD8DFE842
:1049200004F00204060836488DE736488BE736481F
:1049300089E7364887E7364885E72146354802F05B
:10494000BFFD746078E02146334873E02146334868
:1049500070E0214632486DE0214632486AE0214647
:10496000314867E02146314864E000BFD0100020A4
:10497000EEC00008D40100205C0000206000002090
:1049800084100020B810002009C1000826C10008CA
:104990002EBD000841C1000863C100087FC10008A6
:1049A00099C10008C3C10008EFC1000819C200087E
:1049B00041C200085BC2000876C200088FC200082E
:1049C000A9C20008C0C20008D9C20008F9C2000884
:1049D00016C300082FC3000858C300086AC30008A4
:1049E00087C300089DC30008B1C30008C2C3000804
:1049F000D4C30008E6C30008FBC300080DC40008C8
:104A000022C4000841C4000860C400087FC4000834
:104A10009EC40008BEC40008D7C40008F4C400083F
:104A200013C500082EC5000845C5000862C500086A
:104A30002648214602F044FD3568254F0124002D0B
:104A40003DD124483C6001F0AFFF234801F0ACFFAA
:104A500029464620FFF70EFE6420FFF75FFEFFF7B2
:104A60006BFE02211D4802F02BFD02210920FFF7F9
:104A700001FE6420FFF752FEFFF75EFE294618484C
:104A800002F01EFD29460720FFF7F4FD6420FFF722
:104A900045FEFFF751FEBD681248294602F010FDA1
:104AA000A9B20620FFF7E6FD6420FFF737FEFFF707
:104AB00043FE0D4801F078FF074801F075FF2046DE
:104AC00001E00020187005B0F0BD00BF81C50008EE
:104AD000D40100209CC500082EBD0008BDC50008FB
:104AE000DFC5000856BF0008F5C50008064B1A6868
:104AF000064B012A18BFB0FBF2F0013018601A68AB
:104B0000002AFCD1704700BFB0000020F41B002039
:104B1000034B1A6812B11A68013A1A60704700BF55
:104B2000F41B002030B50446054600202B1BDBB2E9
:104B300099421AD92378C3B115F8013BA3F1300289
:104B4000D2B2092A0DD9A3F14102052A01D8373B77
:104B500004E0A3F16102052A02D8573BDAB200E073
:104B6000002202EB001398B2E0E730BD022910B535
:104B7000D4BF1446941E4FF01703204403FB01F1E9
:104B80004FF0090391FBF3F1084400F10400D8BF92
:104B900002F1FF32042392FBF3F318446FF0630336
:104BA00092FBF3F318444FF4C87392FBF3F2024400
:104BB000072092FBF0F0C0EBC000101A10BD0000FF
:104BC000F0B52C4FC0F30725C4B24FF4C87664206B
:104BD000002A20DD6B1E012D144457F823300DD11F
:104BE0008A073DD191FBF0F200FB121222B991FB32
:104BF000F6F206FB12129ABB013331E09C422DDD26
:104C000001350C2DA4EB030303F1FF32C4BF0131C6
:104C100001250124DCE7174F64204FF4C876EAB180
:104C20002244002A22DC013D08BF0C2505F1FF3398
:104C300008BF01F1FF31012D57F82340EFD18B0759
:104C4000EDD191FBF0F300FB13132BB991FBF6F3BD
:104C500006FB1313002BE2D10134E0E7224605E006
:104C6000A342FBDAE21A013A0225D2E742EA052022
:104C7000F0BD00BF20CB0008F8B5654B1A68824232
:104C8000054600F0C480634918606422132395FB35
:104C9000F2F2614C95FBF4F41444014090FBF3FEF6
:104CA000261D03FB1E0ED200072095FBF0F796FB96
:104CB000F0F0C0EBC000361A02F10D00192290FB93
:104CC000F2F2A21A1E200F32002992FBF0F34FF0ED
:104CD000130400FB1323B8BF01F1FF3104FB0E33B3
:104CE000B8BF61F0030193FBF0F200FB1233B8BFD1
:104CF0000131C7EBC7071D2BA5EB070706D01C2BFF
:104D000005D1BEF10B0FA8BF1B2300E01C2303EB52
:104D1000430201EB4701114406EB4106072196FBD4
:104D2000F1F1C1EBC101761A3344163303241F2B72
:104D300002DD1F3B0134FAE7384E43EA042440F217
:104D4000011373604FF48373B36040F20153F36057
:104D500040F6032340F6194733616FF02F0240F607
:104D60001A4329462046B3617761FFF729FF6FF0A8
:104D70000102F06129462046FFF722FF002230623F
:104D800029462046FFF71CFF012270622946204673
:104D9000FFF716FF2722B06229462046FFF710FFD3
:104DA0003122F06229462046FFF70AFF32223063A3
:104DB00029462046FFF704FF3C227063294620461F
:104DC000FFF7FEFE2A46B0630C211920FFF7CEFE46
:104DD0006FF014020446121A29463846FFF7F0FE17
:104DE0006FF00D02F063121B29463846FFF7E8FE0C
:104DF0006FF006023064121B29463846FFF7E0FECA
:104E00006242706429463846FFF7DAFEB064F8BDA6
:104E1000D81000200300008070FEFFFF901B0020D0
:104E200030B5124B186887B0E8B1114D0DF1010291
:104E300000233C2059195C5902F8014C4C68B4FB22
:104E4000F0F108331170402B00FB1141517002F159
:104E50000302EFD1182269464FF4227005F01AFCC4
:104E6000003018BF012007B030BD00BF382500203A
:104E700068010020074A136823B107490B6813F043
:104E8000020301D118467047CB6C038000231360E6
:104E900001207047840F002000200140012310B53D
:104EA000C1F3421401F01F029C4203FA02F201D145
:104EB000838903E0022C0CBF038A838A9BB21340D0
:104EC000028892B243B10123090A03FA01F10A42AE
:104ED00014BF1846002010BD184610BD70B5214CF7
:104EE00040F225512046FFF7D9FFB8B14FF6DF73E6
:104EF00023801D4BA28819681F2992B20ED81B4926
:104F00001B4E0D68D2B2681C72551F2888BF002244
:104F1000086088BF0A601A6801321A60114D40F2B9
:104F200027712846FFF7BAFFD8B14FF67F73114AB1
:104F30002B80136883B11049104D0B68581C202832
:104F40000860EB5C04BF002008601168DBB2013927
:104F50009BB21160A38070BD094A136823F08003DF
:104F6000136070BD00100140D0100020A810002078
:104F7000E4100020D4100020BC1000208510002078
:104F80000C10014010B51D4A936803F00C03042B6C
:104F900003D0082B03D01A4B18E01A4B16E05168C7
:104FA000536811F4800F03F03F03516814BF154A92
:104FB000134AB2FBF3F3114A5268C2F30142C1F340
:104FC000881101324B435200B3FBF2F30B4A0360EA
:104FD00093680D49C3F30313CC5C0368E34043605B
:104FE0009468C4F382240C5D23FA04F4846092680C
:104FF000C2F342328A5CD340C36010BD0038024025
:105000000024F40000127A004C0000204FF6FF73D9
:1050100003600023037143718371C3717047F0B55E
:105020000023012703260A6807FA03FC3CEA020270
:1050300033D15A00056806FA02F4E44325400560BE
:1050400091F804E005680EFA02FE4EEA05050560D7
:105050000D79013D012D14D885682C40846091F8AC
:1050600005E085680EFA02FE4EEA05058560446893
:1050700024EA0C0444608C7945689C40A4B22C431B
:105080004460C46806FA02F524EA0504C460CD79D8
:10509000C46805FA02F22243C2600133102BC2D168
:1050A000F0BD0000024B0A20596A04F0FDBC00BFAD
:1050B00014440020024B0620196904F0F5BC00BF1F
:1050C0001444002010B50446084805F0BFFA2046F5
:1050D00005F0BCFA064805F0B9FA064A1368002B39
:1050E000FCD1FDF7BBF80128FBD110BD04C60008B8
:1050F0002EBD0008A820002000B58BB08A780B7860
:1051000001924A7800920549024602A805F01AFF6A
:1051100002A8FFF7D7FF0BB05DF804FB09C6000833
:1051200000B593B00B4600920549024602A805F06F
:1051300009FF02A8FFF7C6FF13B05DF804FB00BF2C
:105140001EC6000800B58BB00B460092054902460A
:1051500002A805F0F7FE02A8FFF7B4FF0BB05DF858
:1051600004FB00BF27C6000807B50E4B5B69002B88
:10517000B8BF5B428DF805300B4B1868ABBF2B22D4
:105180002D228DF804208DF8042038B1022201A9C7
:10519000BA2005F07FFA003018BF012003B05DF897
:1051A00004FB00BF68000020382500201E280AD814
:1051B0000A2908D8054B0C2202FB0030405C003065
:1051C00018BF012070470020704700BF1011002059
:1051D0002DE9F74F184B1C6800EB8400C1EB8004ED
:1051E000164888461746044400264FF0010901F18D
:1051F000040A09FA06F3454607F1FF3B625D1A42CD
:105200000BD01E2D01930CDCBBF1090F09D83946D8
:105210002846FFF7CBFF019B18B901355545EDD165
:1052200001E0002005E00136042E07F10107E0D17E
:10523000012003B0BDE8F08F441C002031C80008F5
:105240002DE9F047DFF86890DFF868800746002610
:10525000CA46D9F8084034441F2C04DD0136042E18
:10526000F7D1BDE8F08764010A3400259AE80A0006
:1052700003EB810308EB83039B5D2B41DB070FD519
:10528000D9F80C0043190B2B0ADC2044284427B121
:10529000054B01EB4101194400E0044904F01CFEF8
:1052A0000135042DE2D1D9E7DC1B0020611C002070
:1052B000441C002031C8000838B5094CA568E268D4
:1052C000606801352946FFF783FF38B10020FFF7FA
:1052D000B7FF0120A560FFF7B3FF012038BD00BF75
:1052E000441C00202DE9F041184E194DDFF868806C
:1052F000FF2333542B54074605F0A6FC154C0440FD
:10530000002CBEBF04F1FF3464F01F04013405F02B
:105310009BFC104B0340002BBEBF03F1FF3363F037
:105320001F03013308EB4412D25CFF2AE4D10022B0
:10533000B15C8C4202D1A95C8B42DDD00132032AE0
:10534000F6D1F455EB55BDE8F08100BFF81B002005
:105350008C1B00201F000080A81C002007B5094BF3
:105360001B688DF80730084B186840B101220DF119
:105370000701DF2005F08EF9003018BF012003B0CF
:105380005DF804FB80000020382500203D4AD2F85B
:10539000883043F47003C2F888303B4B1A68002110
:1053A00042F001021A6099601A6822F0847222F4B5
:1053B00080321A60354A5A601A6882B022F480221C
:1053C0001A60D960009101911A6842F480321A6023
:1053D0001A6802F400320192009A01320092019A96
:1053E0001AB9009AB2F5C06FF2D1274B1B6813F4BB
:1053F000003318BF01230193019B012B3BD1224BAA
:1054000023491A6C42F080521A640A6842F48042BE
:105410000A609A689A609A689A609A6842F4805220
:105420009A601A6822F080721A601968164A880118
:10543000FBD4184B5360136843F0807313601168FA
:10544000114B8901FBD5144A40F2037111601268B7
:1054500002F00702032A00D0FEE79A6822F0030256
:105460009A609A6842F002029A609A6802F00C020E
:10547000082AFAD100E0FEE7024B4FF000629A6082
:1054800002B0704700ED00E0003802401030002408
:105490000070004004194007003C024007B5094B6A
:1054A0005B688DF80730084B186840B101220DF198
:1054B0000701DE2005F0EEF8003018BF012003B030
:1054C0005DF804FBA40000203825002007B50B463A
:1054D000009201460022D02003F0E2F9B0FA80F0F9
:1054E000400903B05DF804FB07B50B460092014686
:1054F0000022D02003F006FAB0FA80F0400903B091
:105500005DF804FB13B50C4C236883B1022201A99A
:105510001120FFF7E9FF58B19DF805009DF8043010
:10552000C0F3400040EA43006368C01A00E0FF2077
:10553000A06002B010BD00BFA400002037B5284B0A
:105540001B68984201D003F0BBF801220DF107015E
:105550003F20FFF7C9FF012205460DF1070138B3CF
:105560000720FFF7C1FF08B9002435E09DF8073098
:1055700043B1002301220DF1070107208DF8073008
:10558000FFF7A4FF01220DF107010020FFF7ACFF98
:1055900004460028E8D09DF807301A0619D503F014
:1055A0007F038DF8073001220DF1070100200EE086
:1055B0000E20FFF799FF04460028D5D09DF807304C
:1055C0003BB18DF8075001220DF107010E20FFF7C6
:1055D0007DFF044B01221A60204603B030BD00BF9E
:1055E000A41C0020A400002073B5134B186800B35E
:1055F000124D0024062606FB04F304EB84005A5DDA
:105600008DF800202B446946B3F801208DF8012065
:10561000120A8DF80220B3F803308DF8033005220A
:105620001B0A043001348DF8043005F033F8142CD3
:10563000E1D102B070BD00BF38250020141B00204E
:10564000F0B50E4C002306258B4214D005FB03F267
:105650000778165DB7420CD12244B0F80170B2F859
:105660000160B74205D1B0F80360B2F8032096425A
:1056700002D00133E8E7FF231846F0BD141B0020D9
:1056800073B52F4E2F4C0025204604F04BFC2046CE
:1056900001F08AF92C4801F087F9684602F0B8FF5A
:1056A000304602F0B5FF0028FAD07379DB07F7D453
:1056B0003DB129463046FFF7C3FFFF2801D000283F
:1056C000EED10135142D34D0AB1E112B2ED8DFE8CE
:1056D00003F0090B0D0F11131517191B1D1F2123A3
:1056E0002527292B194C22E0194C20E0194C1EE0EB
:1056F000194C1CE0194C1AE0194C18E0194C16E032
:10570000194C14E0194C12E0194C10E0194C0EE041
:10571000194C0CE0194C0AE0194C08E0194C06E051
:10572000194C04E0194C02E0194C00E0194C063603
:10573000AAE7194804F0F6FB012002B070BD00BFD3
:10574000141B0020D0C700082EBD00085CC600084E
:1057500073C600088AC60008A3C60008BCC60008B5
:10576000CBC60008DAC60008EBC60008FCC6000875
:1057700015C700082EC7000849C7000864C70008FD
:105780007EC7000898C70008B4C7000842C60008D2
:1057900032C6000859C60008DDC7000810B5084C1D
:1057A0002368012B0BD0074B07484FF480721A83F4
:1057B00001F0FAF8054801F0F7F80123236010BD65
:1057C0006400002000080240EAC700082EBD00085F
:1057D000F8B5274E442404FB00630F4619690546BB
:1057E000062936D8DFE801F038040C151D252D00F8
:1057F0003846FFF741FA1F4B04FB0564DB6906E0FE
:105800003846FFF739FA1B4B5B6A04FB056463619A
:1058100022E03846FFF730FA164B04FB0564DB6BD9
:10582000F5E73846FFF728FA124B04FB05641B6CBA
:10583000EDE73846FFF720FA0E4B04FB05645B6C7E
:10584000E5E73846FFF718FA0A4B04FB05649B6C42
:10585000DDE7094801F034FE442303FB05653946C2
:10586000AA696869013AFFF7ABF96864F8BD00BF3F
:1058700090120020901B0020FDC70008F0B51D49C4
:1058800044234343CA188BB0044650688DF8000087
:1058900090688DF80100D0688DF8020010698DF8CD
:1058A000030050698DF80400183392698DF80620C2
:1058B0000B44000A1F1D8DF805000DF10706243367
:1058C0000A463D4603CD9D42306071602F4606F189
:1058D0000806F6D1442101FB0421282202FB04F032
:1058E0000B6C8DF82730694600F2A12004F0D2FE3F
:1058F0000BB0F0BD9012002007B5064B02A91B6843
:1059000001F8013D01224FF4287004F0C3FE03B0FA
:105910005DF804FB901200202DE9F0410D4D80460A
:1059200008270124042618EA040F6E8305D00520F9
:10593000FFF7DCF82E83502004E05020FFF7D6F864
:105940002E830520FFF7D2F86400013FE4B2EAD1CC
:10595000BDE8F081000C024038B5084C0425658391
:105960000520FFF7C3F825830A20FFF7BFF8246955
:105970003220FFF7BBF8C4F3800038BD000C0240B2
:105980002DE9F041054600EB010845450DD00827FB
:1059900001240026FFF7E0FF00B126436400013F29
:1059A000E4B2F7D105F8016BEFE7BDE8F081000044
:1059B00038B51A4D04246420FFF798F86C834FF42F
:1059C0000C70FFF793F82C831420FFF78FF8144A1C
:1059D0003C23136000231C46296949071AD50CB1E2
:1059E00003B9136811680029F6D12CB11BB1E31A71
:1059F00003EB830400E01C463220FFF777F8074BE7
:105A000078201D69FFF772F81E2C8CBFC5F380004B
:105A1000002038BD002CE5D11468E3E7000C0240FB
:105A2000F41B002037B5414D2B68E3B904F032F97F
:105A3000012468462C60FFF7E9FA3D4A136B43F0F6
:105A4000080313638DF804408DF806408DF8074075
:105A5000384C042502236946204600958DF8053010
:105A6000FFF7DDFA2583FFF7A3FF002859D0FFF7E2
:105A70009FFF314C50B13320FFF74EFF08212046E5
:105A8000FFF77EFF0125FFF793FF02E020606060D3
:105A900005462A4A23781360294A0121222B1160E6
:105AA00001D0282B3ED1FFF783FFD8B35520254CDA
:105AB000FFF732FF04F0CAFABE20FFF72DFF0921DD
:105AC0002046FFF75DFF237913F0600F2AD0FFF720
:105AD0006FFF38B35520FFF71FFF04F0B7FA4E20D1
:105AE000FFF71AFF7F20FFF717FF8020FFF714FF53
:105AF0000020FFF711FFFFF75BFFFFF759FF88B1A9
:105B00005520FFF709FF04F0A1FA4820FFF704FF32
:105B1000FA24FFF721FF08B9013CFAD1FFF748FF4B
:105B200000E00546284603B030BD00BF401C002001
:105B300000380240000C02409C470020541C00200A
:105B40003C1C0020581C002010B5FFF731FF58B353
:105B500055201A4CFFF7E0FE04F078FABE20FFF75C
:105B6000DBFE09212046FFF70BFFFFF721FF144B57
:105B70001B68222B224601D0282B10D11379507894
:105B80001278C3F341135C1D0933C109C3F10C033F
:105B900000F00700A04042FA03F3184306E094F92E
:105BA00001102078C90F01E0FF2010BD054B19B985
:105BB0001A68801A586010BDFF20FBE7581C0020AF
:105BC000541C00208000002070B51E4D1E4C002883
:105BD00014BF2046284600F10806483056F8085CF5
:105BE0002C0627D556F8044C9C4223D105F04004DE
:105BF00011B1B4FA84F46409E4B1C5F3C20405F048
:105C00000705AC4203D1A51A6C426C4111E008D2E1
:105C1000944204D8954234BF0024012409E00024B2
:105C200007E0954204D294428CBF0024012400E096
:105C3000012424B908368642D0D1002070BD01204D
:105C400070BD00BFFC1B0020641C002070B51F4B02
:105C5000186886B0B8B30DF101041D4E224600232A
:105C60003C20995902F8011CF11808334D68B5FB26
:105C7000F0F1402B117000FB1151517002F1030241
:105C8000EFD118226946BF2004F004FDD8B1114DB0
:105C900000233C215A5904F8012CEA1808335068B3
:105CA000B0FBF1F2402B227001FB1202627004F192
:105CB0000304EFD11822694640F2D71004F0EAFC41
:105CC000003018BF012006B070BD00BF382500208D
:105CD000FC1B0020641C0020D74B1620F0B5186474
:105CE0003C205864202083F8480083F84B0083F858
:105CF000520083F85300D1489865D148986607212F
:105D0000D048DFF898E3D04F196200220421022422
:105D100001250F26D866C3F87CE00320DFF880E376
:105D200059625F65DC651C6619675967986783E887
:105D300024009A60DD601E615E61DA619A62DA6257
:105D40001D635D639A635A66C3F880E0DFF854E32D
:105D5000C3F890E0DFF850E3C3F894E0DFF84CE3D9
:105D6000C3F8A4E0DFF848E3C3F8A8E0DFF844E3B1
:105D7000C3F8B8E0DFF840E3C3F8BCE0DFF83CE389
:105D8000C3F8CCE0DFF838E3C3F8D0E0DFF834E361
:105D9000C3F8E0E0DFF830E3C3F8E4E0DFF82CE339
:105DA000C3F8F4E0DFF828E3C3F88440C3F8884080
:105DB000C3F88C00C3F89840C3F89C40C3F8A00017
:105DC000C3F8AC40C3F8B040C3F8C040C3F8C44007
:105DD000C3F8C800C3F8D410C3F8D810C3F8DC0067
:105DE000C3F8E840C3F8EC40C3F8F000C3F8F8E0AB
:105DF000C3F8FC00C3F80001C3F8B420C3F80401E1
:105E0000C3F81041C3F81441904CC3F81C41904CA6
:105E1000C3F820418F4CC3F830418F4CC3F8344154
:105E20008E4CC3F844418E4CC3F848418D4CDFF88A
:105E3000A4E2C3F858418C4CC3F808E1C3F85C41B4
:105E4000DFF894E2894CC3F81801C3F82411C3F8B1
:105E50002811C3F82C01C3F83811C3F83C11C3F85A
:105E60004001C3F84C01C3F85001C3F85401C3F812
:105E70006011C3F86411C3F86801C3F86C71C3F80A
:105E80008011C3F88411C3F80CE1C3F87051C3F852
:105E90007451C3F87821C3F87C41C3F88851C3F822
:105EA0009011C3F8D011C3F8D4110821C3F8EC1134
:105EB000C3F8F01109216E4FC3F8F411C3F8F811BB
:105EC0000A21C3F89C71C3F8FC116A4FC3F8001291
:105ED0000B216948C3F8AC71C3F80412C3F8081267
:105EE000664FC3F88C010C21C3F89421C3F89821A4
:105EF000C3F8A021C3F8A421C3F8A821C3F8B02196
:105F0000C3F8B421C3F8B821C3F8BC71C3F8C021E9
:105F1000C3F8C421C3F8C821C3F8CC41C3F8D85191
:105F2000C3F8DC01C3F8E021C3F8E421C3F8E82199
:105F3000C3F80C12C3F810120D21C3F81412C3F8E1
:105F400018120E21C3F81C12C3F8201285B0C3F832
:105F50002462C3F8286203F50A7141F8042F013264
:105F60000F2AFAD1032446494648C3F86822C3F8E9
:105F70006C4205F032F8444B002502A81D60FFF783
:105F800045F8424A136B43F0040313638DF80C5039
:105F900005F18045402305F50235029302A902234D
:105FA00028468DF80F308DF80D40FFF738F80120A6
:105FB000FEF7B4FB2B6913F0400400F00581344870
:105FC00000F0F2FC334800F0EFFC01238DF80E30B6
:105FD000022300248DF80C3002A903232E488DF8EB
:105FE0000D308DF80F40FFF71AF840236B832B6AB2
:105FF00023F070632B622B6A43F000732B62234BF8
:106000001A6C42F002021A641A6B42F400121A630C
:10601000A3F50D3301201A8822F45C721204120CCD
:106020001A807E22DA621C8598821A8C22F0010284
:106030001204120C1A8451E0144400201543000885
:1060400009C90008AD40000804C9000842C9000899
:10605000ED7400084AC90008D978000836C900085C
:106060000180000852C90008997C000857C900083F
:10607000AAC3000868C900085FC900086EC9000803
:1060800075C90008844600203425002000380240ED
:106090007BC900082EBD0008000802400EC9000898
:1060A0009543000815C900087576000897C40008D4
:1060B000417800081DC900080D80000823C90008A8
:1060C000D97500082CC900083D7B000831C90008BB
:1060D000078000083DC90008497900081A8C9D888E
:1060E000198B22F0020221F0730109041204090C39
:1060F000120C41F060010243ADB29D8019835C63D4
:106100001A841A8B354D22F008021204120C42F048
:1061100008021A831A8892B242F080021A80B3F8F9
:1061200044206FEA42426FEA524292B2A3F84420FE
:106130009A8992B242F400729A810F238DF804304A
:106140008DF805408DF8070001A88DF8064003F092
:10615000E3FC234B23491A6822F001021A601A68F3
:1061600022F001021A6021221C605C609C60DC60ED
:106170001C615A611C4AD1601A681C4911401C4AB2
:106180000A431A605A6922F0070242F001025A617A
:1061900030225A60174A9A60174ADA60174B19681A
:1061A00040F6685320465943224600EB40030B4417
:1061B000EC180130B0F58F6FEA546270A270F4D120
:1061C00003F032FB05B0F0BD0D4800F0EDFB0D48CB
:1061D00000F0EAFB8DF80E40FAE600BF44250020EF
:1061E000706002403D000020006002403F801CF0D3
:1061F000402D030A34040040682400203C25002080
:106200009CC900082EBD000807B5074B02A9D3F8AA
:106210006C3201F8013D012240F27F2004F03AFA8D
:1062200003B05DF804FB00BF144400201FB5084B09
:10623000002253F8041F0DF802100132102AF8D181
:10624000694640F2AB7004F025FA05B05DF804FB36
:106250003C4600201FB5084B002253F8041F0DF8E0
:1062600002100132102AF8D1694640F2EF1004F012
:1062700011FA05B05DF804FBFC450020042807B5C1
:1062800011D80F4A02EB001302EB0012D3F8A03131
:10629000D2F8A82103F00F0392078DF8073005D537
:1062A00043F0200300E0FF238DF8073001220DF1B9
:1062B000070100F2351004F0EDF903B05DF804FBBE
:1062C00014440020022807B59BBF0B4B03EB0013BF
:1062D000FF23D3F870314FF0010298BF03F00F0392
:1062E0000DF1070100F225108DF8073004F0D2F906
:1062F00003B05DF804FB00BF144400200D2807B56F
:106300000ED80D4A142303FB0022D36D526E03F006
:106310000F0392078DF8073005D543F0100300E016
:10632000FF238DF8073001220DF10701E53004F05D
:10633000B1F903B05DF804FB1444002007B5064B27
:1063400002A91B6C01F8013D0122DD2004F0A2F935
:1063500003B05DF804FB00BF1444002007B5064BF2
:1063600002A95B6C01F8013D0122DC2004F092F9E6
:1063700003B05DF804FB00BF1444002007B5064BD2
:1063800002A99B6801F8013D0122DB2004F082F99B
:1063900003B05DF804FB00BF1444002007B5064BB2
:1063A00002A95B6901F8013D0122DA2004F072F9CB
:1063B00003B05DF804FB00BF1444002007B50B4B8D
:1063C00093F851208DF8042093F852208DF8052081
:1063D00093F853308DF80630032201A940F2A170E2
:1063E00004F058F903B05DF804FB00BF144400202A
:1063F00007B50A4B93F84B208DF8042093F84C20F6
:106400008DF8052093F84D308DF80630032201A950
:10641000D72004F03FF903B05DF804FB14440020DA
:1064200007B5064B02A9DB6901F8013D0122BE2038
:1064300004F030F903B05DF804FB00BF1444002001
:1064400007B5064B02A91B6901F8013D0122BD20D9
:1064500004F020F903B05DF804FB00BF14440020F1
:1064600007B5064B02A9DB6801F8013D0122A9200E
:1064700004F010F903B05DF804FB00BF14440020E1
:1064800007B5064B02A95B6A01F8013D0122A8206D
:1064900004F000F903B05DF804FB00BF14440020D1
:1064A00007B5064B02A91B6A01F8013D0122BC2079
:1064B00004F0F0F803B05DF804FB00BF14440020C2
:1064C00007B5064B02A91B6801F8013D0122A72070
:1064D00004F0E0F803B05DF804FB00BF14440020B2
:1064E00010B5094C636883420CD92368984209D0DF
:1064F00001232060A36219B10146042003F0D4FAFD
:10650000FFF7DEFF206810BD1444002007B50A4BDA
:1065100093F848208DF8042093F849208DF8052041
:1065200093F84A308DF80630032201A9A42004F024
:10653000B1F803B05DF804FB144400200B4B1A695A
:106540005A6193F8482083F84B2093F8492083F848
:106550004C2093F84A2083F84D20054A054B1178CA
:1065600019705178927859709A70704714440020CD
:10657000440000208800002010B50C4C0C48226913
:1065800004F1480103F0C2FCA368033B012B04D9CA
:10659000236A9B0701D5FFF7D1FF236B23B10120AD
:1065A000BDE81040FDF766BE10BD00BF14440020DA
:1065B000440000200C4A0D49D2F8BC000C4B51F8A5
:1065C000201083F84810D2F8BC000A4951F8201076
:1065D00083F84910D2F8BC10074A52F8212083F8FA
:1065E0004A20FFF7C9BF00BFD446002038CA0008C0
:1065F00014440020D8C90008A4C80008094BDA6870
:10660000012A02D0022A0AD070473F2283F848208C
:10661000002283F8492083F84A20FFF7ADBFFFF737
:10662000C9BF00BF14440020064907484B690F2B1F
:1066300028BF0F2301EB83035131D3F82C22FDF740
:10664000ADBC00BF144400200800002037B5134D36
:10665000134C6B690F2B28BF0F2305EB830305F148
:106660004B01D3F82C222046FDF798FC6B6B9BB1B5
:106670000C4B227833F812208DF80420627833F81E
:1066800012208DF80520A278012133F812308DF800
:10669000063001A8FDF7C6FC03B030BD144400204D
:1066A00088000020B6BE000870B5164C0E46E061AA
:1066B00019B10146082003F0F7F9E269114BE2B97C
:1066C0001A690F2A08D00F221A61FFF755FF0EB181
:1066D000FEF7F0FCFFF7B4FE63690A4D0F2B0CD0F8
:1066E0000F236B61FFF7B2FF1EB169690E2003F043
:1066F000DBF96369A361FFF751FEBDE87040FFF766
:106700008FBE00BF144400200C4A0D49D2F8BC00D3
:106710000C4B51F8201083F84B10D2F8BC000A49FA
:1067200051F8201083F84C10D2F8BC10074A52F8E8
:10673000212083F84D20FFF789BF00BFD4460020F9
:1067400038CA000814440020D8C90008A4C80008AA
:106750000D4B9A68042A16D8DFE802F003060609F2
:106760001300586BFDF780BC002001F0D7BD3F221D
:1067700083F84B20002283F84C2083F84D20FFF74C
:1067800065BFFFF7C1BF704714440020084B9A69EA
:106790005A6193F84E2083F84B2093F84F2083F8EA
:1067A0004C2093F8502083F84D20FFF74FBF00BFD7
:1067B00014440020F0B5064689B00F461446002A5E
:1067C00065D00020FDF756FD20070BD5FEF7E6FF4C
:1067D000C820FDF7A3FF2F4B9B6843B90120FDF7AD
:1067E00043FC04E0E10602D5012001F097FD6207B9
:1067F0004DD5284DFDF7C0FB2B6B002B43D00B2351
:1068000040F2E2722449009302970923019604A8FA
:1068100004F098FB04A800F0C7F8204800F0C4F882
:1068200008240C221E491F4804F0FCFB9DF8182088
:106830000094002302210C2003F050FA9DF8192047
:106840000094214600230C2003F048FA0094002312
:106850003A220E210C2003F041FA9DF81A200094F0
:10686000002313210C2003F039FA9DF81B2000941B
:10687000002319210C2003F031FA0C2204A9084846
:1068800004F0D0FB01E0E30601D50123AB6209B0BF
:10689000F0BD00BF14440020C0C900082EBD000890
:1068A000AC200020B920002010B50B4B0B4C5B6CCA
:1068B0000B4873B1142202FB03F10A4AB2FBF1F256
:1068C0002260094AD2F8C42053433C22B3FBF2F3BE
:1068D00000E02360036010BD14440020E420002089
:1068E00040020020A0BB0D00D446002038B5224C49
:1068F00040F225512046FEF7D1FAB8B14FF6DF73CA
:1069000023801E4BA2881968FF2992B20ED81C4919
:106910001C4D0C68D2B2601C2A55FF2888BF00228B
:10692000086088BF0A601A6801321A60124C40F28F
:1069300027712046FEF7B2FAE8B14FF67F73124A8C
:106940002380136893B11149114C0B68581C80289F
:10695000086008BF0020E35C08BF086011680139C7
:106960001160DBB2044A9BB2938038BD094A1368B8
:1069700023F08003136038BD00440040281000203D
:1069800094220020640E0020D0200020242100202A
:10699000B82200200C440040024A1368002BFCD1AE
:1069A000704700BFD020002010B5441E14F8010F1E
:1069B00010B101F083FDF9E710BD00002DE9F74F9C
:1069C0004FF08043814E824C4FF6FE771F82326932
:1069D00020680196002840F058817E490B6802F437
:1069E00080620D461BBB7C481AB903680133036003
:1069F0004BE102689AB101220A6078490A6078493D
:106A00000B6078490B6078490B6078490B607849D6
:106A10000B60784BFF211960774B1A7035E1774A8C
:106A20001368BB4200F23181013313602DE16B4BDF
:106A3000D3F800909846B9F1000F4DD06E4F5AB17F
:106A40003B780133DBB2E92B3B7040F2E980624BCB
:106A5000086018603870E3E05F4A1368A3F11F0113
:106A60000A29914603D83A78063A042A1DD9A3F197
:106A70005E02532A07D83A78A2F12E012B2916D9A3
:106A8000173A162A15D9A3F13C020F2A03D83A78EF
:106A90003C3A0F2A0FD9283B162B03D83B78133BDF
:106AA0000C2B0AD90021296008E0554906E0554918
:106AB00004E0554902E0554900E055492B681BB1F7
:106AC0004422544804F033FA4A4A00231360012256
:106AD000C9F800203B706FE0414B19681F46002940
:106AE0006DD04C4B002A46D0424A586B1168884200
:106AF00096460DD19A6B012A0AD1374A5969126814
:106B0000914217D899698A4214D8C3F838908AE01C
:106B1000DFF8E4801E6898F80020DFF8F890013272
:106B2000D2B2012E88F8002007D0E92A7BD9421E74
:106B300091421AD000232B60A3E00B2A70D90A29B6
:106B4000F3D929484A1CC9F834200268A1F10B0E78
:106B500042EA0E220260D9F82C20114401310A22A7
:106B6000C9F8301088F8002005E09B6B002BE1D1BC
:106B7000CEF8000057E01968264ADFF85C801E480E
:106B8000032940F0A083DFF86CE0DEF80010102944
:106B900040F09983D8F80030053B072B00F2AD8315
:106BA0000378A3F13C000F2800F2818300233B60AF
:106BB0001123CEF800300123C8F8003030E05ABB72
:106BC000054A1368013313602AE000BF0008024041
:106BD0008422002008210020EC200020A022002098
:106BE000F4200020B022002014210020F0200020FA
:106BF000742200208C220020D8200020FC200020BD
:106C000050CB000898CA0008DCCA000894CB0008E2
:106C1000D8CB00082821002001221A60944B1A705A
:106C20002B68002B31D0934F934B796B1B689942A3
:106C30002BD1BB6B4BBB914B914AD3F800C0106872
:106C400084451E468F4840F06B838F4B1B68B3F51D
:106C5000966F80F065830368013303603B68012B06
:106C600040F0608300680138012800F26983864B98
:106C7000002119602368002B40F0C38300232B60A0
:106C80001360824A13607A4A1370814D23682B681F
:106C9000012B0CD97F4A136840F6A66101338B4261
:106CA000136004D17C4B01211960002313607B4ADF
:106CB00013680133EA2B136004D1794B0121196069
:106CC00000231360774B1B68002B00F0CA81764AC3
:106CD00013680133962B136040F0C38100201060CD
:106CE000724A1168FF2914460CD171490B68642B54
:106CF00005BF01994FF4805301334B8314BF0B60E0
:106D00001060AEE1019B6B4A1B6913F400634FF006
:106D1000200040F0028350830129674A08D003D342
:106D20000229664E16D02CE001212160136098E103
:106D300011688B4200F09581002B1360604B4FF07F
:106D4000FF021A605D4B0CBF02210321002221606B
:106D50001A6086E111688B4202D1336801330EE07C
:106D6000136033680321782B216003D9544B002230
:106D70001A6003E04A2B01D800232360002333600C
:106D80006FE111688B42E8D0136033684C4F9A1F53
:106D90000221122A21600BD9052B94BF49484A4889
:106DA000FFF702FE4948FFF7FFFD002323600FE1D4
:106DB0000F2B3B6840F2F880113B292B00F2088131
:106DC000DFE813F02A000601060106012E0032005A
:106DD0003B003F00430047004B004F008E009200F5
:106DE00096009A009E00A200A800AE00B000B2007B
:106DF000B400B600B800BA00BE00C200C600C800A9
:106E0000CA00CC00CE00D000D200D400D600DA00F8
:106E1000DE00E200E600EC002D4B01221A60D7E014
:106E20002C4A1368013302E02A4A136802331360C4
:106E3000294A136801331360CAE0264A13680433F1
:106E4000F5E7244A13680833F1E7224A13680A3346
:106E5000EDE7204A13681433E9E71E4A1368283324
:106E6000E5E71D4B1B68DA0700F1B2801B4897E786
:106E7000D8200020282100208C220020980000200B
:106E8000B022002070210020FC200020EC200020F7
:106E90004C010020A42200205C010020B42200202C
:106EA000F801002064240020E82000209400002045
:106EB000DC2000200000024010210020F8200020EB
:106EC0008C0000201CCC000839CC00082EBD000826
:106ED0000C2100208C0F00209022002057CC0008AD
:106EE0008F4A1368013312E08D4A136802330EE0B3
:106EF0008B4A136804330AE0894A1368083306E0B2
:106F0000874A13680A3302E0854A13681433136012
:106F1000844A8EE7834B1B68DB0759D482483FE7DE
:106F2000824A0AE0814A0CE0804A0EE07F4A20E073
:106F30007E4A22E07D4A24E07D4A136801332AE03C
:106F40007B4A1368023326E0794A1368043322E04F
:106F5000784AF2E7774AF4E7764AF6E7754A08E0B6
:106F6000744A0AE0744AE8E7734AEAE7724AECE7CF
:106F7000714A136808330EE06F4A13680A330AE057
:106F80006D4A1368143306E06B4A1368283302E035
:106F9000694A136850331360684A4AE7674B1B68B5
:106FA000D80715D46648FBE6232B08D03A2B0BD024
:106FB0001C2B0DD1634B1B68D90709D556E7594BDC
:106FC0001B68DA0704D5A9E75C4B1B68DB07E9D42B
:106FD0003A680F2A0AD15C4B1A68002A00F03982FD
:106FE0005A4A0121116000221A6032E2102A19D196
:106FF000564900230B6054490B6052490B604949C4
:107000000B604E490B6052490B6052490B6044497A
:107010000B6047490B6045490B6046490B60464988
:107020000B6002E0FF2A3FF4A9AE01323B2A3A602E
:1070300014D13B4A484B11681868464C884247486F
:1070400007D1016827680131B94202BF3E490127D3
:107050000F6012681A60236803608FE63FF68CAEFB
:107060008CE63F4A13680133962B136004D13D4BE5
:1070700001211960002313603B4A136801330F2B71
:10708000136004D1394B0121196000231360384982
:107090000B68BBB1374B1A6801321A6018680A686E
:1070A00090420FD3344A0021196013680133142B26
:1070B000136004D131481160036801330360304B21
:1070C00001221A602F4A136843F6982101338B423C
:1070D00001D01360C0E12C4B012018602B68002107
:1070E00003441160294A2B60D2F8C4300344C2F82B
:1070F000C430D2F8C4302D2B13460BD1244BD2F818
:10710000C04019688C4200F0C280D2F8C0201A60DA
:10711000204BBBE0D2F8C440312C3FD11E4BB5E030
:10712000640F0020D420002078CC0008B401002097
:107130006C0F0020A80100203C0200201821002034
:1071400099CC000890220020A822002024020020D0
:107150000C2100208C0F00209C2200200021002008
:10716000E0200020B8010020982200201C210020EF
:10717000E42000202021002088220020400200205E
:1071800010020020AC220020F4010020D446002090
:10719000900000202C100020740F0020D2F8C44072
:1071A000322C01D1AE4B71E0D2F8C440332C01D166
:1071B000AC4B6BE0D2F8C4403C2C62D1C2F8C41096
:1071C000A94A1160A94A1160A94A1160D3F8C020E8
:1071D0000132C3F8C020A74A1060D3F8C0203C2A6F
:1071E00055D1C3F8C010D3F8BC200132C3F8BC207D
:1071F000D3F8BC20182A4AD1C3F8BC10D3F8AC206D
:107200000132C3F8AC20D3F8AC20072A08BFC3F87A
:10721000AC10D3F8B82098490132C3F8B820D3F89D
:10722000B850D3F8B400D3F8B020441E022851F867
:1072300024100FD190070DD16424B2FBF4F004FBAD
:10724000102030B94FF4C874B2FBF4F004FB1022E4
:1072500002B901318D421AD90120C3F8B800D3F820
:10726000B410864A0144C3F8B410D3F8B4300C2BE0
:107270000DD9C2F8B400D2F8B0300344C2F8B0302F
:1072800005E0D2F8C4301E2B01D17D4B18607D4B38
:107290001A68002A00F0E0801A68013A1A601B6838
:1072A000002B40F0D980784B01221A60D4E00F3BCC
:1072B0000A20D1620F2B4FF020011060116351633F
:1072C00015D8012014E0D8F800105E686F4A8E428D
:1072D00017D95B696D4A99420FD3936999420CD8CB
:1072E0000178D369994208D3136A994205D80020DE
:1072F00001F026F900233B605DE400232B6003705E
:1073000059E49668B142E4D890F800C0D668B44514
:10731000DFD312699445DCD8D3E710830123FBE463
:1073200000239AE4052B03D10068012808D19EE4CC
:107330000A2B01D0292B03D10068C0073FF597AC79
:107340000120022B2060DFF86CA15148DFF868E1D2
:10735000504F1DD1DFF86481002972D1DFF85091C0
:10736000D9F80030B3F5E16F0FD2DFF830A1D8F8CB
:1073700000300360DAF80030C2F800C043F00103C7
:10738000CAF80030C9F800105BE0CAF8001058E0F5
:10739000052B2BD1404B93F8008093F801B093F864
:1073A000029008F00F0181EA18180BF00F0188EA2B
:1073B000010181EA1B1B09F00F018B451CBF002155
:1073C000CAF80010D97889EA010919795B7989EA44
:1073D00001094B451CBF002323603049304BD1F8D5
:1073E00000801B6848EA03030B600523CEF80030D9
:1073F00003683B602B4B116819602B4B19682B4BB2
:1074000037E417682A49DFF8B4E0BC45DFF880C0EC
:107410000FD1DEF80000DCF80030984209D10B688B
:1074200040F6C90083429FBF1C48036843F0010334
:107430000360DCF80030CEF80030002337600B60CA
:107440001CE40223CEF8003003683B60C8F800302B
:10745000D0E710233B6091E403B0BDE8F08F00BF9C
:10746000900F00203010002020210020400200203A
:10747000882200205001002020CB0008D4460020A4
:107480005801002010000020D001002028210020F9
:1074900014210020CC2000207C220020C8200020C5
:1074A000F0200020782200207422002004210020F7
:1074B000FC200020842200206C2100209C00002061
:1074C0000FB413B5084C04AB4FF4807153F8042B80
:1074D0000193204603F0E4FD2046FFF765FA02B071
:1074E000BDE8104004B07047742100202DE9F84336
:1074F000364DAB6A23B1364A0023AB62EB621360B0
:10750000EC6A002C60D1324E336893BBDFF8C4C004
:107510001C461A46E1464FEA421E0CEB0E0020279D
:1075200080467B1EC15C11F0010F14D01F2B02D0CE
:10753000C45DE4070ED421F0010108F803103BB14B
:10754000013B03EB0E0149444978C90702D5F6E730
:10755000012403E001240BB11F46E2E70132202A97
:10756000D9D10120FCF7E4FE01230CB9336000E01F
:107570001C463368012B27D1164F002107EB41161B
:1075800000233046C25C02F00A0EBEF1020F0FD19A
:1075900013B112F0080F0BD142F00802C2541F2B96
:1075A00005D05A1CB45CA40701D51346F7E70124A3
:1075B0000133202BE6D101312029DFD10820FCF74F
:1075C000B7FE0CB90123EB62BDE8F8831444002038
:1075D0000C2400201440002038B5214A936A33B1AE
:1075E000204900230B6020499362D3620B60D36A69
:1075F000002B34D11B4C236873B91C4B03F58061FD
:1076000013F8012F22F008028B421A70F8D10820DB
:10761000FCF78EFE012320E0134801680131016070
:10762000C9071CD5013B12489BB2B3F5806F10D23D
:10763000C15C11F0020F03F1010508D00C4A41F0C2
:1076400008010820D154FCF773FE256003E0ABB2BB
:10765000EBE70123D36223680133236038BD38BDD3
:107660001444002048230020102400201340002050
:10767000144000202DE9F04F6E4B9A6A85B022B17C
:107680006D4900229A62DA620A60DB6A002B40F0E0
:10769000CD80694A15680F2D114600F2C480674EEF
:1076A00000229C19A05C654F20F00800A054013214
:1076B000202AF7D12033B3F5806FF1D16A1C0A601C
:1076C000C2F11006002100237C18E05C20F01000BD
:1076D000E0540133202BF8D12031B1F5806FF2D185
:1076E000002407EB441C00201CF800309B071DD52C
:1076F0000F2C04D833190F2B28BF0F2303E0A31B33
:107700000F2B98BF10230F2804D831180F2928BF3A
:107710000F2103E0811B0F2998BF102107EB4313B2
:1077200013F801E04EF0100E03F801E001302028BC
:10773000DAD10134202CD4D105EB4513029300217A
:10774000AB013E48039316460C464FEA450C029B9C
:10775000C3EB010A039B0CEB0A0903EB0908CCEB12
:10776000080301931546002301EB000E1EF8037079
:10777000FF073CD50F2C1DD80F2B0DD8A24236D8B1
:107780009A4234D803EB0A07074417F821BC4BF0A0
:10779000080B07F821BC2AE0A24228D81F2D26D8C2
:1077A00003EB0907074417F81FBC4BF0080B07F859
:1077B0001FBC1CE00F2B0DD81F2E18D89A4216D8CC
:1077C000019FDF19074497F81FB04BF0080B87F8AB
:1077D0001FB00CE01F2E0AD81F2D08D808EB030796
:1077E000074497F821B04BF0080B87F821B01EF83A
:1077F000037017F0100F1CBF47F008070EF8037056
:107800000133202B05F10105B0D12031B1F5806F96
:1078100004F1010406F1010699D1082005B0BDE884
:10782000F04FFCF785BD034B0122DA6205B0BDE8DD
:10783000F08F00BF14440020542400201440002086
:1078400070B5224B9C6A8EB01E4654B3002423466A
:10785000142202FB0361496E890741BF0EA901EBA7
:107860008401013441F8383C01330E2BF1D1184D1D
:107870000CB92C600BE003F0E7F9B0FBF4F303FB69
:1078800014000EAB03EB800050F8383C2B602A68E4
:10789000142303FB02639B6D98470E4B00221A6072
:1078A00011E00B4A0B4812680168142505FB0233EE
:1078B0000131DA6D0160914205D39B6D04600EB019
:1078C000BDE8704018470EB070BD00BF14440020E2
:1078D0004C2300200424002038B5184CA36A23B19F
:1078E000174A0023A362E3621360E36A23BB144DCB
:1078F0002B6801332B6003F0A7F9124B00F007004F
:1079000003F5806101281A7805DD12F0030F02D01B
:1079100042F0080201E022F008021A7001338B42A3
:10792000F0D12B68202B03BF0123E3620220082043
:10793000BDE83840FCF7FCBC38BD00BF1444002053
:10794000FC230020144000202DE9F04F724B9A6A6E
:1079500085B03AB1002271499A62DA6201220A6066
:107960006F490A60DB6A002B40F0D2806B4B1D68C8
:10797000194635B36B4E20256A1E50018719002326
:10798000FC5C04F00A0EBEF1080F0DD165490844F5
:1079900024F008041F2AC4540DD001EB4512D15C19
:1079A00041F00801D15406E00133202BE8D11546FF
:1079B000002AE1D10A60082005B0BDE8F04FFCF7CD
:1079C000B7BC574B03931A68002A00F09980564EB3
:1079D000564833685649574FD3B10268514B09682E
:1079E00003EB421E01321EF80140026024F008043D
:1079F0000EF8014003EB4213585C40F008045C545D
:107A00003C68A242D7D140F0090058543560D2E713
:107A1000494E0268D7F800C0D1F800E0019218463C
:107A20009B461C46984619464FF02009A6F5806AE9
:107A300009F1FF350022002944D1A6F12007BF5CDF
:107A4000029707F00A07022F38D12DB3029C04F0E9
:107A500008072946FFB2013977B1B35CCDF804902D
:107A6000012043F00803B3549646AC4603468346D0
:107A700004468046014621E00029ECD1C3B912F842
:107A80000A10019341F00801012302F80A109646FA
:107A9000AC4618469B460EE012F80A10012441F04D
:107AA000090102F80A109646AC46A046214605E0B8
:107AB0009646AC4601231C46984619460132202AB8
:107AC000B9D100E00121203EA946002DB0D1B8F186
:107AD000000F02D0174AC2F800C014B1144AC2F80D
:107AE00000E0BBF1000F02D0104A019C146008B105
:107AF0000D4A136000297FF45EAF039B19605AE7BB
:107B0000FCF73AFA0820FCF713FC034B0122DA6277
:107B100005B0BDE8F08F00BF144400203C240020D5
:107B200038240020144000204C240020442300204E
:107B300040240020D8230020144400202DE9F843DD
:107B4000524B9A6A22B1524900229A62DA620A6062
:107B5000DB6A002B40F098804D4D2C680F2C3DD8EF
:107B60004C4963016FF01F001A1960430A44C4F1C5
:107B70002006401A00EB020E7645464F05D91778CD
:107B800047F0080702F8017BF4E71B1B621C3B442B
:107B9000C4F11F00824203F120030DD213F814E058
:107BA0004EF0080E03F814E093F81FE04EF0080EB4
:107BB00083F81FE00132EDE704EB40128B186FF001
:107BC0001F0101FB00F2D21B197841F0080103F8F4
:107BD000011BD1188E42F7D89CB119E0102C4BD163
:107BE00016E06FF01F0103EB4E1301FB0EF23B4456
:107BF000921B197821F0080103F8011BD118884263
:107C0000F7D808200134FCF793FB2C60BDE8F8831B
:107C1000631E204F5A016FF01F0E99180EFB03FED2
:107C20003944C3F12000C7EB0E0E0EEB010C60458A
:107C3000184E05D90E7826F0080601F8016BF4E716
:107C400020321A4432442146C3F11F0EC4F1000809
:107C5000714502F12002C4D212F820CCC3EB020914
:107C60002CF0080C02F820CC19F808C02CF0080CF5
:107C700009F808C00131EBE7FCF77EF90820FCF7B2
:107C800057FB024B0122DA62BDE8F883144400205E
:107C900018240020144000202DE9F3412E4B9A6A4D
:107CA00022B12E4900229A62DA620A60D3F82C804F
:107CB000B8F1000F4DD1294B1C680134082C1C6011
:107CC00044DC274F274D7A7A6B7A93420ED00826F0
:107CD000234631460C20009602F000F86A7A0094A0
:107CE00043463146C4F1140001F0F8FFBA7AAB7A8A
:107CF00093420FD008230093132123460C2001F058
:107D0000EDFF184B13219A7A00940023C4F114005C
:107D100001F0E4FFFA7AEB7A93420FD00823009344
:107D2000192123460C2001F0D9FF0E4B1921DA7AD4
:107D300000940023C4F1140001F0D0FFFCF71CF9FB
:107D4000082002B0BDE8F041FCF7F2BA024B012274
:107D5000DA6202B0BDE8F081144400203C23002028
:107D6000B9200020AC2000202DE9F04F994FBB6ACC
:107D700085B08146002B7BD0974B3A69974C984D44
:107D800000264FF03F08694601A81E60BE62FE62F1
:107D90008DF800808DF801808DF8026002F0B6F851
:107DA0009DF804208F4B34F812201A709DF805209E
:107DB00034F812205A709DF8062034F812209A7078
:107DC000B9F1000F0CD010233A698DF80C6003A9AB
:107DD00002A88DF80D808DF80E3002F097F808E0BB
:107DE0002B788DF808306B788DF80930AB788DF8EA
:107DF0000A309DF808207C4B34F812201A709DF848
:107E0000092034F812205A709DF80A2034F8122004
:107E10009A702A78754B34F812201A706A7834F800
:107E200012205A70AA78724D34F812209A700024E9
:107E300014F0010F4FEA84060AD002F005FF6D4BE3
:107E40000340002B10DA013B63F01F0301330BE00A
:107E500002F0FAFE674B0340002BBEBF03F1FF3375
:107E600063F01F03013310330134202CAB51DFD1F9
:107E7000FC6A002C40F0AB80574F3B685F2B00F250
:107E80009E80594DDFF874812B788DF80C306B781B
:107E90008DF80D30554EAB788DF80E3058F8040F34
:107EA00030280DD8D8F8003001340133202CC8F820
:107EB0000030F3D1FCF7F6F83B6801333B6086E015
:107EC000A0F1300BBBF1010F05D1464904EB4B107B
:107ED00002F002F80EE0A0F132031F2B07D800F1E8
:107EE00000603238404904EB401001F0F5FFBBF16F
:107EF0001F0FEAD94FF0010A0BF1FF39B9F11F0F3B
:107F000007D9ABF10209ABF1030BBBF11E0F29D965
:107F10004DE0394B4FEA49101A18125D92070AD505
:107F2000BAF1050F07D932788DF80C2072788DF8E8
:107F30000D20B2780CE02A78B2FBFAF28DF80C2012
:107F40006A78B2FBFAF28DF80D20AA78B2FBFAF249
:107F500003A920448DF80E2001F0BEFFB9F1000FF7
:107F600025D0CEE7244B4FEA49101A18125D93072B
:107F70000AD5BAF1050F07D932788DF80C2072783E
:107F80008DF80D20B2780CE02A78B2FBFAF28DF869
:107F90000C206A78B2FBFAF28DF80D20AA78B2FBB9
:107FA000FAF203A920448DF80E2001F095FF0AF1A2
:107FB000010AB9F1000F3FF475AFCB469CE7FBF720
:107FC000DBFF0820FCF7B4F9024B0122DA6205B0AE
:107FD000BDE8F08F1444002008240020B6BE00083D
:107FE000440000203823002058240020D4230020FF
:107FF000542300201F000080144000205023002044
:108000000020FFF7B1BE0120FFF7AEBE2DE9F74F0C
:108010009848836ADBB1984A984900231360984ACC
:108020000C781360974A83621360974AC3621360A7
:10803000964A1360964A974B32F814401C704C785D
:10804000897832F8144032F811205C709A70C36A53
:10805000884E002B40F00A81874D894F2C68002CF8
:108060004CD196F848301F2B05D83F238DF80030AF
:108070008DF8014008E096F849301F2B07D83F23C0
:108080008DF800408DF801308DF802400DE096F833
:108090004A308DF800401F2B4FF03F0394BF8DF8FE
:1080A00001408DF801308DF802300269694601A85F
:1080B00001F02CFF764B9DF80420774933F812200D
:1080C0000A709DF805203E6833F812204A709DF82A
:1080D000062033F812308B70704B00221A705A70E1
:1080E0009A70684B1C6804EB461001F0F5FE6C4B6F
:1080F0001E706C4B1C7001232B60AFE03A683A2A6B
:1081000007D9FBF739FF0820FCF712F90123F362C6
:10811000ACE05D4B5B4E1968DFF870918A429C467B
:108120004BD13168D9F80030994246D1D30702D5F6
:1081300031B1013902E01E2902D80131924601E035
:1081400002F1010A584BD64603EB4A18BEF11F0F45
:1081500030D8F2450EF0010B04D0BBF1000F03D074
:108160001F2303E00B4601E05B4615E0BBF1000F67
:1081700012D00133002B74D0013B18F803B00BF080
:108180000A0BBBF1020F10D0BBF1080FF2D10CE0CB
:10819000BBF1080F09D001331F2B62D818F803B0C8
:1081A0000BF00A0BBBF1020FF2D1CCF800E0C9F8DA
:1081B000003002E03B23CCF8003012F0010F3368AE
:1081C000D9F8001003D08B4207D9013B02E08B4263
:1081D00003D201332B4A136007E0DCF800309A42E7
:1081E00035BF013201233A60C362D7F80080B8F18D
:1081F0001F0F05D83068284900EB481001F06CFECD
:108200001B2C274F274C1ED13B781F2B0ED82649FD
:10821000227801EB43112020895C11F0020F14BF7A
:108220001C491E4900FB032001F056FE00230133C8
:10823000FA18F95C02F8011CE218E15C02F8011C72
:108240001A2BF4D12B602B683268E2541A2B98BF9A
:10825000094A07F803809CBF01331360FBF722FF34
:1082600004E00EF1010E08F120086FE703B0BDE84D
:10827000F08F00BF144400200024002044000020A0
:108280004824002014240020F8230020502300203C
:10829000B6BE0008402300205024002044240020C3
:1082A0001C240020DC23002014400020F8B5194DC8
:1082B000194F2E683C68317800232246184601F099
:1082C00069FDC4F1060416F8011F91B11F2C06D8F0
:1082D000002320461A4601F05DFD0634F3E708202E
:1082E000FCF726F83B680C4A0133062B0BD01360D1
:1082F000F8BD1F2CF3D8002320461A46202101F098
:1083000049FD0634F5E7002313602B6801332B6029
:10831000F8BD00BFB4000020D046002007B5002300
:10832000014601A88DF804308DF805308DF806302F
:10833000FBF778FE03B05DF804FB000038B5054696
:10834000064C28B101236363BDE83840FBF760BEEB
:108350000120FFF7E3FF656338BD00BF1444002030
:108360002DE9F0411E4D14462A8892B242F48072E3
:1083700007462A801B480E46984601F077FC18B342
:108380002B88B8F1000F04D023F480631B041B0C6E
:1083900002E09BB243F480632B80114D124807F03A
:1083A000FE072F8201F062FC90B110482B8B01F088
:1083B0005DFC88B1F3B214B1C6F307262E829BB2DE
:1083C0002B820020BDE8F0814FF0FF30BDE8F08146
:1083D0006FF00100BDE8F0816FF00200BDE8F081B0
:1083E000005C00400100001002000010800000103E
:1083F000F0B52E4D2E4F85B001F0B6FBAC882D4B5D
:1084000024F03F04684624041E68240CFCF7BAFDDF
:10841000029AB2FBF7F7B8B20443AC802988264B26
:1084200021F001010904090C9E4229804FEA46030C
:1084300009D8B2FBF3F301309BB2032B80B298BF93
:108440000423288416E03344B2FBF3F39BB2C3F356
:108450000B020AB943F001034FF4967101FB07F2D6
:108460004FF47A7192FBF1F21049013292B243F467
:1084700000430A840D4A938313889BB243F001039F
:108480001380138823F4816323F002031B041B0C65
:1084900043F4806313804FF48043138113889BB2AD
:1084A00043F00103138005B0F0BD00BF005C004045
:1084B00040420F005C240020A086010030B50E4928
:1084C0000B680D4A7F2BFBD80C4B0D4D1C68611CB3
:1084D0007F291960C0B288BF0021285588BF196064
:1084E00072B613680133136062B6064A136843F02C
:1084F0008003136030BD00BFD02000206024002026
:10850000B82200200C44004008B50A4B1B680BB988
:10851000002008BD02220849E12002F0BBF8002833
:10852000F6D002220549E32002F0B4F8003018BF6B
:10853000012008BD382500201C0000201E0000205E
:1085400070B52C4A2C4C516A2368994205D8956A1B
:10855000AB4202D2D66B294D08E0D16A254D8B4241
:108560000FD32E6BB3420CD2EE6B254D2EB1591AA0
:108570002E6800FA01F1314302E0296840EA410126
:1085800029601268032A09D1A3F11102032A2DD808
:108590001C4990400A681043086027E0052A25D14D
:1085A000A3F11402032A06D8154DA3F1080200FA1C
:1085B00002F12A6807E0A3F11801032906D8124D39
:1085C000296800FA02F20A432A6001E02F2B0DD835
:1085D00003F007060122D9080C4DB24010B1685CC7
:1085E000024302E0685C20EA02026A54013323601D
:1085F00070BD00BF282100208C2200201421002003
:10860000B022002074220020F02000207C220020D4
:1086100070B5254C2368002B31D0244A244B1168B7
:10862000022911D003292CD11D681968C943C9B288
:10863000B1EB152F1FD11968C9B219601D490D681A
:10864000196841EA052114E01D681968C943C9B2D7
:10865000B1EB152F0BD0184D2E6848F2EE718E42FB
:1086600009D10B2111601968C1F30721296019682C
:10867000C9B2196005E000200023236070BD1846D0
:1086800070BD12680C4D02702A68A0F801201A68AB
:108690000A49A0F803200A68427100221A600120EA
:1086A0002A600A60E8E700BF842200206C210020D5
:1086B0007822002004210020CC200020C8200020A7
:1086C000564B2DE9F7431860064601F04DFA544B1E
:1086D0001A6B42F001021A631A6B42F004021A6329
:1086E0006846FCF793FC0024694601254D488DF847
:1086F00007404FF480778DF805408DF804508DF8D1
:1087000006500097FCF78BFC6846FCF77FFC8DF861
:1087100004408DF807408DF8054004F1804404F5CD
:1087200002344FF40073694620460093FCF777FC4F
:10873000236999055DD54FF480783A4F0925C146E4
:10874000A7F818900120FBF7E9FF23699A0555D592
:10875000344B4FF480721A830120FBF7DFFF23694B
:108760009B0553D52E4D6846FCF750FC2B6B2D48CE
:1087700043F001032B632B6B43F004032B632B6A41
:1087800043F400032B622B6A23F400032B62436A39
:1087900023F00F034362436A43F004034362636AB6
:1087A00023F0F0036362636A43F0400363620223D1
:1087B0008DF804308DF8053001238DF806308DF8E2
:1087C000073069464FF480730093FCF728FC4FF4A0
:1087D0000073694614480093FCF721FC2B6C43F4AA
:1087E00000032B64114B1E60FFF702FE03B0BDE8CF
:1087F000F08367832846FBF791FF9CE7A7F81A8070
:108800000120FBF78BFF013D9AD1A1E70848FEF755
:10881000CBF80848FEF7C8F8A4E700BFA41C002066
:108820000038024000000240000802405C240020A2
:10883000BACC00082EBD000808B50B4A13889BB2BD
:1088400043F40073138013886FEA43436FEA534382
:108850009BB213801388C3F30E03138001F084F9D5
:10886000BDE80840FFF7C4BD005C004070B5064697
:108870000D460624304601F083F940B9013C03D08F
:108880000120FBF74BFFF5E7FFF7D6FF05E0284691
:1088900001F076F90028F1D00124204670BD0000D7
:1088A00070B51C460023FFF75BFD20BB124801F0AA
:1088B000DDF9E8B1049B114EE518AC420F4A0BD02C
:1088C00014F8013B33820E490B48FFF7CFFF002815
:1088D000F3D16FF003000EE013889BB243F40073F2
:1088E00013804FF4003001F04BF90028F9D170BD2E
:1088F0006FF0020070BD70BD80000010005C004091
:10890000040000102DE9F041069F7C1E1E466342C4
:1089100063418046FFF724FD0546002845D12C49D8
:108920002C48FFF7A3FF002841D02B4C2B4823886D
:108930009BB243F48073238001F098F900283AD069
:1089400048F001085FFA88F8A4F81080244801F084
:108950008DF9002833D0238B013EAF421CD0013566
:10896000AF4207D01F4801F081F960B3238A06F8AF
:10897000013FF2E7228822F480621204120C228066
:10898000228892B242F4007222804FF4003001F04B
:10899000F7F80028F9D1E5E70F4A13889BB243F4B2
:1089A000806313800020BDE8F081BDE8F0816FF0A6
:1089B0000300BDE8F0816FF00400BDE8F0816FF0C6
:1089C0000500BDE8F0816FF00600BDE8F08100BF52
:1089D0000400001080000010005C00400100001046
:1089E0000200001040000010F7B505460C46002AB2
:1089F00043D02E48FDF7D8FF284602F0F6FA2E465F
:108A00002F18BE4211D016F8012BA2F120035E2BC5
:108A100003D81046FFF752FDF3E72549684602F0F8
:108A200091FA6846FDF7C0FFEBE70CB32020FFF793
:108A300045FD2220FFF742FD204602F0D6FA2646E9
:108A40002718BE4211D016F8012BA2F120035E2B8D
:108A500003D81046FFF732FDF3E71549684602F0E8
:108A600071FA6846FDF7A0FFEBE72220FFF726FD2D
:108A70001048FDF799FFFDF78FFF284601F0E6FD4E
:108A80005CB1202001F0BCFD222001F0B9FD2046A0
:108A900001F0DCFD222001F0B3FD074801F0D6FD16
:108AA000064A1368002BFCD103B0F0BDD6CC0008F9
:108AB000DBCC0008E2CC00082EBD0008A820002076
:108AC00038B50E4C206309B1FFF738FC0C4B216B15
:108AD0005B68002914BF0C25142513B1032000F096
:108AE000E3FF226B074B12B9044A526B0AB1002212
:108AF00000E001221A60284638BD00BF144400205F
:108B0000980F00206424002001460148FEF7D8BCDD
:108B1000F0CC0008044B186828B14022034940F209
:108B2000FF1001F0B7BD7047382500200047002036
:108B300010B50B4C23680BB9002010BDFFF7EAFFFE
:108B40000028F9D02368002BF6D04022054940F2D6
:108B50003F2001F09FFD003018BF012010BD00BF75
:108B600038250020404700202DE9F04FD04D2B68DC
:108B70009BB0002B00F0D584CE48FDF715FFCE4802
:108B8000FDF712FF2B6823B10422CC49002001F02D
:108B9000B1FDCA4ECA483168FEF792FC336823F42F
:108BA0007F0424F47F44002C40F0CC84A3F582326F
:108BB000A2F58072B2F5823F00F2C484C14FC24870
:108BC0003C711A0C30321B0A30333A702E22BB70C3
:108BD0007A70FDF7E9FEB848FDF7E6FE2B681BB397
:108BE000DFF8108304EB8400052210A9043001F0A3
:108BF00081FD062363439DF8401003F8081003EB42
:108C000008029DF842109DF8413043EA0123A2F882
:108C100001309DF844109DF84330013443EA0123AC
:108C2000142CA2F80330DDD12B68002B00F0388221
:108C30003F238DF81C30A54BD6F800801A889B780E
:108C40008DF8223008238DF80E303C238DF80F303C
:108C500016238DF810304FF0030907230024ADF8D8
:108C600020208DF813304A460F2306A9A4208DF842
:108C700015308DF80A408DF81D408DF81E408DF896
:108C80000B408DF80C408DF811408DF812408DF896
:108C9000179001F02FFD01220DF10D01A72001F029
:108CA00029FD01220DF11101A82001F023FD01226F
:108CB00005A9BD2001F01EFD01220DF11601BE2007
:108CC00001F018FDB8F5843FC0F0168101220DF1C6
:108CD0001201A92001F00EFD7D4B984540F20C8158
:108CE00001220DF11301BC2001F004FD4A4607A941
:108CF000D72001F0FFFC01220DF11501DA2001F06F
:108D0000F9FC01220DF10E01DB2001F0F3FCB8F5B6
:108D1000003FC0F0F18001220DF10F01DC2001F0D5
:108D2000E9FC012204A9DD2001F0E4FC694B98452F
:108D300040F2E2800DF1300B0E225946E5200DF194
:108D4000240A01F0D7FC4A46514640F225100DF1A5
:108D5000280901F0CFFC0522494640F2351001F008
:108D6000C9FC5D4A11461BF80430FF2B0BD013F0F1
:108D7000100F03F00F00536ED06514BF43F00203D1
:108D800023F00203536601340E2C02F11402EAD1DF
:108D900000231AF80320FF2A1CBF01EB031002F086
:108DA0000F0203F1010318BFC0F87021032BF0D1AB
:108DB0000020D1F8B821DFF82CE1034619F8034070
:108DC000FF2C10D001EB031C04F00F0AF045CCF887
:108DD000A0A108D9012B06D1A40601D40223EDE7F6
:108DE00042F0020218460133052BE7D108B1C1F861
:108DF000B8213A4B98457FD901220DF10A0140F282
:108E0000451001F077FC01220DF10B014FF4A37026
:108E100001F070FCB8F5013F6ED90DF140094946EB
:108E2000102240F2EF1001F065FC2D4B00240F21C1
:108E300019F8042001340F2A8CBF19601A60102C15
:108E400003F10403F4D1274B984555D901220DF1C4
:108E5000170140F27F2001F04DFC234B98454BD980
:108E6000032208A940F2A17001F044FC012203A9E9
:108E70004FF4A37001F03EFC06221C4940F2A5709D
:108E800001F038FC2246494640F2AB7001F032FC5A
:108E9000174A00230F2019F8031001330F298CBF44
:108EA00010601160102B02F10402F4D12CE000BF1D
:108EB0003825002022B900082EBD0008340000200B
:108EC0000ECD0008D446002035CD0008EDCC0008BA
:108ED000FF080100FF00020014440020FF0102000F
:108EE00000460020FF050200FF0802008446002023
:108EF00040460020141B0020C14B03F1400253F8F0
:108F0000041F19649A42FAD19DF80E30BD4C042B0F
:108F100084BF00238DF80E309DF811300D2B84BFD7
:108F200000238DF811309DF81230022B84BF0023EE
:108F30008DF812309DF818303F2B84BF3F238DF8F9
:108F400018309DF819303F2B84BF3F238DF819301E
:108F50009DF81A303F2B84BF3F238DF81A309DF8BF
:108F60001C303F2B84BF3F238DF81C309DF81D30F3
:108F70003F2B84BF3F238DF81D309DF81E303F2BC3
:108F800084BF3F238DF81E309DF814300F2B84BF13
:108F90000F238DF814309DF815300F2B84BF0F234D
:108FA0008DF815309DF81630012B1CBF00238DF86D
:108FB00016309DF80F30782B84BF78238DF80F3052
:108FC0009DF81030772B84BF16238DF810309DF854
:108FD0001730102B84BF03238DF817309DF80D3008
:108FE00023609DF80E30A3609DF8133023629DF836
:108FF000113063629DF81230E3609DF8183084F8F8
:1090000048309DF8193084F849309DF81A3084F8BA
:109010004A309DF8203084F851309DF8213084F892
:1090200052309DF8223084F853309DF814309DF86A
:109030001C009DF81D109DF81E2023619DF816E070
:109040009DF8153084F84B0084F84C1084F84D20BE
:109050006361C4F81CE09DF80FE0C4F844E09DF89B
:1090600010E0C4F840E04FF0000E84F84E0084F8A1
:109070004F1084F85020A361D4F83080C4F830E059
:10908000FDF7E4FAFDF7D0FAFDF776FA9DF8173010
:10909000C4F86C32C4F83080FDF7B0FAFDF758FB25
:1090A0002B68594CA3B110222146AA2001F022FBC3
:1090B00070B1022210A9BA2001F01CFB40B19DF84A
:1090C00040209DF8413063612D2A08D15B4205E0C4
:1090D00010224E494C4801F0A5FF012363612B6823
:1090E000002B59D03368B3F5023F55D31AA9002499
:1090F00001F8384D01224FF4287001F0FBFA9DF879
:1091000030301F2B88BF8DF83040414C9DF83030F7
:1091100023604FF00009A2464FF0280B0DF16703C2
:10912000DAF80020914504F1440835D20BFB09F030
:10913000282210A900F2A120019301F0DBFA9DF88A
:10914000402048F8402C9DF8412048F83C2C9DF8E0
:10915000422048F8382C9DF8432048F8342CBDF8BC
:10916000442048F8302C019B9DF8462048F82C2CD0
:109170001C340DF1470252F8041B44F8041B9A42B8
:10918000F9D1002208F8082C9DF8672048F8042C33
:1091900009F101094446C3E72B68002B6ED0D6F8CD
:1091A00000901C4B994569D910AC18222146BF206C
:1091B00001F0A0FAA0B34FF00008174A43464FF061
:1091C0003C0E4046E15C42F8041CE118033304EB1A
:1091D000030C49781CF801CC1EFB01C1B1F5B46F3A
:1091E000116082BF42F8040C10604FF00108182B88
:1091F00002F10802E6D1094B99453AD914E000BFC3
:10920000FC450020144400206800002046CD0008E2
:1092100090120020FF060100001C0020FF04020045
:109220009C4B99452AD980461822214640F2D710F6
:1092300001F060FAE8B10023974A4FF03C0E18465F
:10924000E15C42F8041CE118033304EB030C497899
:109250001CF801CC1EFB01C1B1F5B46F116082BFD7
:1092600042F8040C10604FF00108182B02F10802BC
:10927000E6D1B8F1000F01D0FCF7E8FC2B686BB326
:109280003268864B9A4229D910AC182221464FF4F5
:10929000227001F02FFA08B30021814A0B464FF0EB
:1092A0003C0C8E46E05C42F8040CE018033304EBFF
:1092B0000308407818F8018C1CFB0080B0F5B46FEF
:1092C000106082BF42F804ECC2F800E00121182BC4
:1092D00002F10802E6D109B1FBF7A2FD3268714B39
:1092E0009A4259D92B687BB1012210A9DF2001F0E5
:1092F00001FA9DF840300A2B84BF00238DF84030DE
:10930000694B9DF840201A602B689BB13268654B11
:109310009A4208D9012210A9DE2001F0EBF99DF84C
:1093200040300A2B02D900238DF840305F4B9DF866
:1093300040205A602B68002B2ED03268594B9A423D
:109340002AD902225A49E12001F0D4F902225949CE
:10935000E32001F0CFF9584B9A88D988B2F5805FA5
:109360004FF0000224BF9A800122B1F5805F22BF36
:10937000514A40F6FF71D180D8889B884E4928BF5A
:109380000122984205D800238B8040F6FF73CB80E2
:1093900000E00AB1FFF7B8F83268484B9A423AD970
:1093A0002B68C3B3464C2022214640F2471001F0FF
:1093B000A1F980B3202204F1210140F2671001F0ED
:1093C00099F940B3082204F1420140F2871001F0FC
:1093D00091F900B3082204F14B0140F28F1001F023
:1093E00089F9C0B12378FF2B0BD094F82130FF2BE3
:1093F00007D094F84230FF2B03D094F84B30FF2B6A
:1094000009D10023237084F8213084F8423084F895
:109410004B3000F009FB2B68002B5FD032681F4BEC
:10942000284C9A4250D9012207A94FF4207001F02C
:1094300061F902220CA940F2812001F05BF90222BD
:1094400010A940F2832001F055F9012208A940F249
:10945000852001F04FF9012209A940F2862001F090
:1094600049F901220AA940F2872001F043F99DF849
:109470001C30A360BDF83030E360BDF8403023619C
:109480009DF8203063619DF82430A3619DF8283059
:1094900023E000BFFF040200681C0020FF0602005A
:1094A0006C010020FF00020080000020A4000020CA
:1094B0001C0000201E00002018000020FF010200F8
:1094C000D0240020D40100201E23A3600023E360E9
:1094D000236163610723A3610523E3612B683BB329
:1094E00032681A4B9A4223D94022194940F2FF10A0
:1094F00001F000F9E0B1174B1B68CBB140221649CF
:1095000040F23F2001F0F6F890B197F82C30613B23
:10951000192B0DD8114B93F86C30613B192B11D9D5
:1095200006E00F48FDF740FA0E48FDF73DFA09E066
:109530000D49074801F051FD0C49074801F04DFD68
:10954000FFF7F6FA1BB0BDE8F08F00BFFF05020081
:10955000004700203825002040470020D446002046
:1095600039B900082EBD0008E3B70008EDB70008C0
:10957000044B186820B104220349002001F08AB886
:10958000704700BF3825002034000020F0B5364B6E
:10959000364E374D3468A3F13002002814BF184608
:1095A0001046344B2A681B689A4243D2324B1968E2
:1095B0002A68324B40F6685707FB013302EB420240
:1095C000134400F110010246802793F801E01EEADF
:1095D000070F14BF4FF04F0E4FF02F0EA2F800E010
:1095E00002328A424FEA5707EFD100F1200280276A
:1095F00093F800E01EEA070F14BF4FF04F0E4FF034
:109600002F0EA1F800E002318A424FEA5707EFD14E
:10961000303080219F780F4214BF4F272F271780AB
:10962000023282424FEA5101F4D12B6801331834DF
:109630002B6016E01249182300250A68A24208D9B7
:10964000013B00F10202058004F1010409D010463B
:10965000F3E700EB43030022834202D00280023092
:10966000FAE73460F0BD00BF98240020CC2400202D
:10967000282500202C250020C82400204425002077
:10968000302500202DE9F041414B1A68B2F5E13F49
:1096900088B07AD04FF4E13802A8C3F80080FBF715
:1096A000B5FC4FF41653049300243A4BADF8144024
:1096B0000C27ADF81640ADF81840ADF81A70ADF8AB
:1096C0001C401A6B344D42F001021A631A6B42F0CF
:1096D00001021A631A6C42F400321A642B6A23F4F2
:1096E00070632B622B6A43F4E0632B622B6A23F4D2
:1096F00070432B622B6A43F4E0432B6202238DF804
:109700000C30032328468DF80D300126042302A9CE
:1097100002938DF80E408DF80F60FBF780FC082354
:109720002846A5F5DE350DEB03010293FBF777FC28
:10973000AB896FEA43436FEA53439BB2AB81284640
:1097400004A9CDF81080ADF81440ADF81640ADF87E
:109750001840ADF81C40ADF81A7000F02FFAAB8934
:109760000E4A9BB243F40053AB81136843F02003CD
:10977000136001A826238DF804308DF805408DF87C
:1097800006408DF8076000F0C7F908B0BDE8F08129
:109790002425002000380240000002400C44004014
:1097A00013B5072269460020FBF79EFEB8B39DF86B
:1097B00000200A23140902F00F011A4A13FB0411B6
:1097C00091609DF801100C0901F00F0113FB0411C9
:1097D000D1609DF802100C0901F00F0113FB041178
:1097E00011619DF80310013911629DF804100C09F4
:1097F00001F00F0113FB041151619DF805100C09D4
:1098000001F00F0113FB0411013991619DF806105D
:109810000C0901F00F0113FB04136433D36102B090
:1098200010BD00BFD4460020F8B5B0F58F6F2B4BAC
:1098300028BF4FF48F601C68002CFCD1284D294EA6
:109840002B683360B3FA83F35B092B60264B274AFE
:109850001C60274B1C6018234343ED331360254BDA
:1098600018602046FFF792FE0120FFF78FFE1B4B8A
:1098700001221A60204A138823F001031B041B0CE9
:1098800013801E4B196821F00101196030215960C5
:10989000196841F018011960196841F00101196057
:1098A000138817499BB243F00103138040F66857B1
:1098B00033682A6804EB440007FB03030B4407FBEF
:1098C00002021888885201EB020E01349B788EF850
:1098D0000230B4F58F6FEBD1F8BD00BF3425002006
:1098E0003C250020C8240020CC2400203025002066
:1098F000282500202C250020000400407060024034
:109900004425002038B5174B174C1A68616811F0D0
:10991000100F1D4601D0100707D42B686168114A4B
:1099200089061ED5DB061CD505E01023E360002068
:10993000FFF72CFEF1E70C4B2021D9600B4B196887
:109940000B4B1B68994204D20120BDE83840FFF759
:109950001DBE136823F001031360064B00221A603A
:1099600038BD38BD7060024000600240CC24002049
:10997000302500203425002030B5244C227895B0C5
:1099800005462346002A3FD094F84220B2B194F80D
:109990004B209AB12146684601F01FFB1C496846DE
:1099A00001F0F4FA04F14201684601F0EFFA1849B7
:1099B000684601F0EBFA04F14B010BE093F821301B
:1099C00013B31249684601F008FB1149684601F0DB
:1099D000DDFA1049684601F0D9FA032D14D8DFE802
:1099E00005F002060A0E012269460B480AE0012230
:1099F00069460A4806E001226946094802E009482A
:109A000001226946FEF7F0FF15B030BDD0240020DA
:109A100055CD0008F124002059CD00085FCD000885
:109A2000F9BC000868CD000808B52022114940F2B1
:109A3000471000F02FFED0B10F4B1B68BBB12022A6
:109A40000E4940F2671000F025FE80B108220C4953
:109A500040F2871000F01EFE48B10822094940F28A
:109A60008F1000F017FE003018BF012008BD002045
:109A700008BD00BFD024002038250020F12400209C
:109A8000122500201B25002000B591B00B46024690
:109A90000449684601F056FA6846FBF713FB11B01B
:109AA0005DF804FB73CD000800B58BB0C1F307234C
:109AB0000246009302A8CBB2044901F043FA02A87F
:109AC000FBF700FB0BB05DF804FB00BF7BCD00088B
:109AD00001490020FBF710BB5C44002000B50C4B93
:109AE0000C499A688FB006A80492DA6803921A6942
:109AF00002925A6901929A690092DB69002201F090
:109B000021FA06A8FBF7DEFA0FB05DF804FB00BFF0
:109B1000D446002089CD000810B5114B4478DA688E
:109B2000D243C2F30222C2F10403DBB204FA03F30C
:109B3000D9B20F231341827813400B4302780949AD
:109B40001B010A44DBB282F8003303780122580972
:109B500003F01F0302FA03F341F8203010BD00BFE9
:109B600000ED00E000E100E0044B1A6A42F400025C
:109B70001A621A6A22F400021A6270470038024020
:109B800082B00023009301930B4B0193030F0093CA
:109B9000009B20F07F4013B1019B143302E0019B36
:109BA000000C18330193019B1B68034214BF012072
:109BB000002002B0704700BF005C00407FB5038A00
:109BC00023F440531B041B0C038283890E469BB273
:109BD00023F4B053898823F00C0233890B43718935
:109BE0000B439BB213438381838AB2899BB223F4D4
:109BF00040731343838204466846FBF7C3F91A4B4C
:109C00009C4203D003F580639C4201D1039D00E098
:109C1000029DA389316813F4004F4FF0190202FB33
:109C200005F214BF4D008D00B2FBF5F5A289642644
:109C3000B5FBF6F000010109120406FB115307D52C
:109C4000D9003231B1FBF6F202F00702104306E010
:109C50001A013232B2FBF6F303F00F03184380B25D
:109C6000208104B070BD00BF0010014038B505462A
:109C700006242846FFF784FF40B9013C03D00120A9
:109C8000FAF74CFDF5E7FEF7D7FD00E0012420468A
:109C900038BD00000B4BC8221A600B4B0B4A1B68E7
:109CA000B3FBF2F30A4A013B53600A4BF02183F8FD
:109CB00023100023936007231360074B05221A60CB
:109CC000704700BFA0000020B8000020400D030036
:109CD00010E000E000ED00E0B00000202DE9F042CF
:109CE000140622D5DC2A1BD007D8C42A1CD0D62AB9
:109CF00012D0B02A16D1012217E0E42A0AD003D8E4
:109D0000DF2A0FD1082210E0F62A07D0FC2A09D159
:109D100007220AE0052208E0032206E0062204E00A
:109D2000042202E0202200E00222C0EB030E174CC6
:109D3000174E0EEBC2022244069D0EEB0004AC420D
:109D400021D201EB40143444002503EB000C6345A1
:109D500012D81F2810D84F191F2F0DD8175CC5F126
:109D6000040947FA09F717F0010F277814BF47F0E5
:109D7000020727F0020727700135052D04F10104C1
:109D8000E5D10130D8E7BDE8F08200BFA7CD0008DB
:109D9000144000202DE9F74F00930B0622D5DC2953
:109DA0001BD007D8C4291CD0D62912D0B02916D16F
:109DB000012117E0E4290AD003D8DF290FD10821B7
:109DC00010E0F62907D0FC2909D107210AE0052176
:109DD00008E0032106E0062104E0042102E020213E
:109DE00000E00221284C019400F5C0762644C90009
:109DF00000274FF001094FF0080B244B02F1010C32
:109E0000C2F1040E3546002403EB070ABCF1050F2E
:109E100022D804EB0008B8F11F0F16D81AF80180F9
:109E2000009B48FA0EF84BB118F0010F0DD095F8D1
:109E3000008048F0020885F8008006E018F0010F65
:109E400014BF85F800B085F8009001340CF1010CC6
:109E500001350EF1FF3ED9E7009B3BB10137082FDA
:109E600006F12006C9D103B0BDE8F08F04444FEAE3
:109E7000471E1F2CF2D8019B04EB0E051D44013434
:109E800085F88091F5E700BF14400020A7CD0008B9
:109E900030B50E4A136C1844536C984200D3C01A64
:109EA000772812D80A4B0B4A1B680C7800F58060A3
:109EB00000EB400040F6685505FB030013181454EE
:109EC0004A785A708A789A7030BD30BD14440020A8
:109ED0003C25002044250020B0F5806F30B50FD21E
:109EE000084B094A1B680C7800EB400040F66855A7
:109EF00005FB0300131814544A785A708A789A7034
:109F000030BD00BF3C250020442500200F2A044B13
:109F100028BF0F2203EB8202D2F8EC21FAF73EB8F9
:109F20001444002070B5114B1A6B01461E46E2B175
:109F30000F4D104C20233E22A81C2B706B7001F09B
:109F400071F80D4B256000221A60FAF74DF84FF4B6
:109F50007A7523681B7843B1FEF7A8F9D6F86C022E
:109F600068438009FAF7DAFBF3E770BD1444002078
:109F70008C460020B4000020D046002007B5254BB9
:109F80001868002842D024498A680A2392FBF3F01B
:109F900003FB102202EB00128DF80020CA6892FB2E
:109FA000F3F003FB102202EB00128DF801200A6986
:109FB00092FBF3F003FB102202EB00128DF802205B
:109FC0000A6A01328DF803204A6992FBF3F003FB21
:109FD000102202EB00128DF804208A69013292FBF4
:109FE000F3F003FB102202EB00128DF80520CA6982
:109FF000643A92FBF3F103FB112303EB01130722F5
:10A00000694600208DF80630FBF760FA03B05DF872
:10A0100004FB00BFA4000020D446002070B5054614
:10A020008AB00E46002456F8243000932A46234670
:10A03000054902A800F086FF013402A8FBF742F8A8
:10A04000402CF0D10AB070BDA7D1000838B5044D3E
:10A050000024285D0134FBF75FFC082CF9D138BDE2
:10A060009C4700202DE9F041404B414D88B04FF412
:10A07000E13802A8C3F80080FAF7C8FF4FF416537E
:10A08000049300243B4BADF814400C27ADF8164068
:10A09000ADF81840ADF81A70ADF81C401A6B42F0DC
:10A0A00002021A631A6B42F002021A631A6C42F43B
:10A0B00080221A646B6A23F470636B626B6A43F4E8
:10A0C000E0636B626B6A23F470436B626B6A43F408
:10A0D000E0436B6202238DF80C3003238DF80D30C2
:10A0E00001264FF4806302A9284602938DF80E40A2
:10A0F0008DF80F60FAF793FF2846A5F5DE354FF48B
:10A10000006302A90293FAF78AFFAB896FEA43431F
:10A110006FEA53439BB2AB8104A92846CDF8108067
:10A12000ADF81440ADF81640ADF81840ADF81C403D
:10A13000ADF81A70FFF742FDAB890F4A9BB243F4AA
:10A140000053AB81136843F02003136001A8272359
:10A150008DF804308DF805408DF806408DF80760C5
:10A16000FFF7DAFC08B0BDE8F08100BF4025002011
:10A1700000040240003802400C4800402DE9F7433B
:10A18000234E244D6846FAF741FF336B43F0010339
:10A190000024336301274FF0800869462846CDF834
:10A1A00000808DF805408DF804708DF806408DF81C
:10A1B0000740FAF734FF336B3B4333634FF04009FA
:10A1C00069462846CDF800908DF805408DF804705A
:10A1D0008DF806408DF80740FAF721FF336B3B43BB
:10A1E000336369461026284600968DF805408DF8A1
:10A1F00004708DF806408DF80740FAF710FFA5F8B7
:10A200001880A5F818902E8303B0BDE8F08300BF36
:10A21000003802400000024010B50A4A0A4C136898
:10A22000591CB1F5807FE35C116004BF002111600F
:10A23000DBB272B605490A68013A0A6062B6036089
:10A24000012010BD2C4800203C4900202410002093
:10A250002DE9F341FCF7A0FB994A1368002BFCD1D0
:10A26000984E3368002B00F01E81DFF86082964F15
:10A270003368002B00F0178101A8FFF7CDFF0028FD
:10A2800000F01181019A914D01230A2AC8F800308B
:10A2900040F0FD803A688E4C0023A354002A00F061
:10A2A000F380894A136023782E2B03D16378002B27
:10A2B00000F0FB8005228749854800F09EFE30B9FA
:10A2C0003F228549854800F0ADFE0D20F2E00522D1
:10A2D00083497F4800F091FE30B93F227E497F4894
:10A2E00000F0A0FE0F20E5E07E48FCF75DFB78481B
:10A2F000FCF75AFB7C48FCF757FBFCF74DFB0222AE
:10A300007A49734800F079FE002800F0CE800522DB
:10A3100077496F4800F071FE002800F0C8800222E3
:10A3200074496B4800F069FE002800F0C2800A22E0
:10A330007149674800F061FE40B90F226F497048CB
:10A3400000F070FE01236B600420B3E003226D492E
:10A350005F4800F052FE30B91F226B496B4800F095
:10A3600061FE0520A6E005226949594800F045FE36
:10A3700058B902226749584800F03FFE08B9022345
:10A3800000E00123AB60062094E0052262495048BA
:10A3900000F033FE30B90F224F49504800F042FE22
:10A3A000072087E008225D49494800F026FE30B9C1
:10A3B0003F225B49494800F035FE0A207AE00B2233
:10A3C0005849434800F019FE30B93F2256494348E6
:10A3D00000F028FE15206DE0062254493C4800F0AC
:10A3E0000CFE064640B9022251493C4800F01AFED4
:10A3F00085F84E600B205DE009224E49344800F09C
:10A40000FCFD064640B902224B49344800F00AFEE2
:10A4100085F84E6016204DE0092248492C4800F08E
:10A42000ECFD30B90F224449454800F0FBFD0820FF
:10A4300040E004224349264800F0DFFD30B93F22C6
:10A440004149264800F0EEFD092033E005223F494E
:10A450001F4800F0D2FD30B93F221F491F4800F0CD
:10A46000E1FD0C2026E005221A49194800F0C5FD3F
:10A4700000283FF425AF3649154800F0A4FD002818
:10A480000CBF0E20FF2015E0FCF786FAF0E60D2A3F
:10A490003FF4EEAE3B68FF2B3FF6EAAE591C396045
:10A4A0000B49CA54E4E6002006E0012002E0022045
:10A4B00000E003200023237002B0BDE8F08100BF5C
:10A4C000A82000202410002030480020980F0020F1
:10A4D00034480020B5D1000839480020E40F00209E
:10A4E00001D20008BBD10008BDD10008C1D10008CD
:10A4F000C4D10008CAD10008CDD100083E480020D0
:10A50000D40F0020D8D1000837480020B40F002015
:10A51000DCD10008E2D10008E5D10008EBD1000849
:10A520003C480020F4D100083F48002000D2000839
:10A530003A48002007D200083D48002011D2000808
:10A54000A40F00201BD200083848002020D20008A9
:10A5500026D2000838B5224C40F225512046FAF7A1
:10A560009DFCB8B14FF6DF7323801E4BA28819689B
:10A57000FF2992B20ED81C491C4D0C68D2B2601C47
:10A580002A55FF2888BF0022086088BF0A601A6821
:10A5900001321A60124C40F227712046FAF77EFC15
:10A5A000E8B14FF67F73124A2380136893B11149C3
:10A5B000114C0B68581C8028086008BF0020E35C21
:10A5C00008BF0860116801391160DBB2044A9BB210
:10A5D000938038BD094A136823F08003136038BDA7
:10A5E0000048004024100020384900203C49002049
:10A5F000A8200020A4470020A84700200C480040C5
:10A6000030B50E490B680D4A7F2BFBD80C4B0D4D16
:10A610001C68611C7F291960C0B288BF00212855C1
:10A6200088BF196072B613680133136062B6064AB8
:10A63000136843F08003136030BD00BFA8200020E2
:10A640003C4A0020A84700200C48004010B5441E9A
:10A6500014F8010F10B1FFF7D3FFF9E710BD0000A8
:10A6600000B591B00B4602460749684600F06AFC07
:10A67000012269460548FEF7B7F9054B00221A602A
:10A6800011B05DF804FB00BF2CD20008CEBC00085E
:10A69000741000202DE9F743134B1B6880460E46CB
:10A6A0000BB900201DE0114F8D180C46B946C6EBC2
:10A6B0000801AC4221444FF0010211D00C48009235
:10A6C00023460068FEF7ECF80028EAD110233A6828
:10A6D000002AFCD0013BC9F80000F8D10134E6E7BC
:10A6E000104603B0BDE8F083382500201C2100206F
:10A6F0002848002013B50B4608490C6854B10146A0
:10A700000748009200680122FEF7FCF8B0FA80F0DA
:10A71000400900E0204602B010BD00BF38250020EF
:10A7200028480020F0B5104B1B68984285B001D036
:10A73000FDF7C6FF0D4E002401276000012540F003
:10A74000A00000970DF10F032A4600213060FEF7AC
:10A75000D9F810B9064B1D6002E00134082CECD189
:10A76000034B186805B0F0BDA41C00202848002049
:10A77000382500201FB5C3074CBF0F490F494208B9
:10A78000684600F0DFFB0020F9F774FDF9F72CFCB8
:10A7900000229DF8001010460123FFF7FBFA012369
:10A7A00000229DF801100620FFF7F4FA044B012265
:10A7B0009A6205B05DF804FB34D2000839D2000873
:10A7C000144400200B4AD3681269934206D2834294
:10A7D0000CD882422CBF00200120704706D982424B
:10A7E00006D2834294BF00200120704701207047A9
:10A7F00000207047D40100200649074A074B9A42BF
:10A80000BEBF51F8040B42F8040BF8E70448804738
:10A810000448004780D30008000000202C010020DD
:10A820008D530008E50100083349344A002301E054
:10A8300041F8043B9142FBD3F5F70EFDFEE7FEE73E
:10A84000FEE7FEE7FEE7FEE7FEE7FEE7FEE7FEE7E0
:10A85000FEE7FEE7FEE7FEE7FEE7FEE7FEE7FEE7D0
:10A86000FEE7FEE7FEE7FEE7FEE7FEE7FEE7FEE7C0
:10A87000FEE7FEE7FEE7FEE7FEE7FEE7FEE7FEE7B0
:10A88000FEE7FEE7FEE7FEE7FEE7FEE7FEE7FEE7A0
:10A89000FEE7FEE7FEE7FEE7FEE7FEE7FEE7FEE790
:10A8A000FEE7FEE7FEE7FEE7FEE7FEE7FEE7FEE780
:10A8B000FEE7FEE7FEE7FEE7FEE7FEE7FEE7FEE770
:10A8C000FEE7FEE7FEE7FEE7FEE7FEE7FEE7FEE760
:10A8D000FEE7FEE7FEE7FEE7FEE7FEE7FEE7FEE750
:10A8E000FEE7FEE7FEE7FEE7FEE7FEE7FEE7FEE740
:10A8F000FEE7FEE7FEE700002C010020504A0020A2
:10A900000A22002100F070BA08B5074B044613B1C3
:10A910000021AFF30080054B1868836A03B19847A4
:10A92000204600F003FB00BF000000003CD20008FE
:10A9300038B5074B1C68E36B05461BB9242000F0B3
:10A94000C7F8E063E16B2846BDE8384000F002B884
:10A950001C0100200268474BF0B592FBF3F403FBA7
:10A960001422002ABCBF02F5A83202F5C0724FF4CF
:10A97000616004F52F2492FBF0F300FB13224FF0EB
:10A980003C00ACBF04F66C2404F66B248B6092FB95
:10A99000F0F300FB13224B600A600723E21C92FBDA
:10A9A000F3F3C3EBC303D31A8B61334B334D94FBE7
:10A9B000F5F503FB054448F6AC62B4FBF2F2224421
:10A9C00040F2B457B4FBF7F3D21A2D48B4FBF0F0C1
:10A9D00048F69466131AB3FBF6F6344440F26D124F
:10A9E000B3FBF2F0B3FBF7F3E31A02FB1033992445
:10A9F00003EB83020232B2FBF4F20A2A04FB02F4F4
:10AA000004F102064FF00504B6FBF4F434BF02264D
:10AA10006FF0090616444FF4C87202FB05055F1C6F
:10AA2000012E98BF0135B3F5997FA7EB040702D338
:10AA3000A3F5997214E0820705D16424B0FBF4F207
:10AA400004FB12024AB94FF4C872B0FBF2F402FBE5
:10AA50001400B0FA80F2520900E001223B331A449C
:10AA6000A5F26C750023CA614D610E61CF600B6267
:10AA70000846F0BD805101004FC5FDFFB13A02000C
:10AA8000B03A020070B50E4B0E4CE41AA41000252B
:10AA90001E46A54204D056F8253098470135F8E700
:10AAA00000F092FE084C094BE41AA41000251E4643
:10AAB000A54204D056F8253098470135F8E770BD17
:10AAC000240100202401002028010020240100206E
:10AAD000024B0146186800F059B800BF1C01002065
:10AAE00002440346934202D003F8011BFAE7704781
:10AAF00038B50546002946D051F8043C0C1F002B00
:10AB0000B8BFE41800F002FA1F4A1368114613B9DF
:10AB10006360146032E0A3420ED92268A018834219
:10AB200004BF18685B68636004BF121822600C6081
:10AB300024E0A24203D813465A68002AF9D11868C3
:10AB40001918A1420BD1216801445818824219609A
:10AB500014D1106852685A60014419600EE002D99D
:10AB60000C232B600AE021686018824204BF106841
:10AB70005268626004BF091821605C602846BDE825
:10AB8000384000F0C4B938BD444A002070B5CD1C2F
:10AB900025F0030508350C2D38BF0C25002D064681
:10ABA00001DBA94202D90C23336046E000F0AEF984
:10ABB000234B1C681A462146A1B10B685B1B0ED4BF
:10ABC0000B2B03D90B60CC18CD501EE08C420DBF6F
:10ABD00063684B686360136018BF0C4615E00C4651
:10ABE0004968E9E7174C23681BB9304600F066F85E
:10ABF00020602946304600F061F8431C18D0C41C80
:10AC000024F00304A0420DD12560304600F07FF906
:10AC100004F10B00231D20F00700C31A0ED05A4286
:10AC2000E25070BD211A304600F048F80130EBD1F7
:10AC30000C233360304600F06AF9002070BD00BF7D
:10AC4000444A0020404A0020194B10B51C68A36BF1
:10AC5000D3B91820FFF73CFF43F20E33A063038003
:10AC60004AF6CD33438041F2342383804EF26D6344
:10AC7000C3804DF6EC630381052343810B2383815D
:10AC800001220023C0E90423A16B0A4C0B69486927
:10AC9000094A5C4302FB0040A3FB02230132034448
:10ACA00043F10003C1E9042323F0004010BD00BFBD
:10ACB0001C0100202DF451582D7F954C38B5064CC1
:10ACC000002305460846236000F022F9431C02D108
:10ACD000236803B12B6038BD4C4A00202DE9F047B2
:10ACE00080464048D0F800900F463D4615F8014B8D
:10ACF00009EB0400407800F0080000F0FF0608B1FE
:10AD00002F46F2E72D2C03D1BD1C7C78012603E0F1
:10AD10002B2C04BF7C78BD1C13B1102B0AD15BE037
:10AD2000302C57D1287800F0DF0058284DD16C78AE
:10AD300010230235002E14BF4FF0004C6FF0004C72
:10AD40000027BCFBF3FA384603FB1ACC09EB040ED0
:10AD50009EF801E01EF0040F01D0303C0BE01EF025
:10AD6000030E1BD0BEF1010F0CBF4FF0370E4FF09A
:10AD7000570ECEEB0404A34210DDB7F1FF3F0AD01B
:10AD8000504506D801D1644503DC03FB0040012790
:10AD900001E04FF0FF3715F8014BD7E77B1C0CD1D2
:10ADA000002E4FF0220314BF4FF000406FF0004020
:10ADB000C8F800302AB9BDE8F08706B1404272B148
:10ADC00007B1691E1160BDE8F0873024002BB1D1B6
:10ADD0000823AFE70A23ADE7302CA3D0AAE7BDE8EC
:10ADE000F08700BF2001002013460A4601460248B2
:10ADF0000068FFF773BF00BF1C0100202DE9F0477A
:10AE000080463C48D0F800900E46354615F8014B78
:10AE100009EB0400407800F0080000F0FF0708B1DB
:10AE20002E46F2E72D2C03D1B51C7478012703E0E0
:10AE30002B2C04BF7478B51C13B1102B0AD153E02E
:10AE4000302C4FD1287800F0DF00582845D16C789D
:10AE5000102302354FF0FF3C0026BCFBF3FC03FB44
:10AE60000CFA6FEA0A0A304609EB040E9EF801E07C
:10AE70001EF0040F01D0303C0BE01EF0030E1AD080
:10AE8000BEF1010F0CBF4FF0370E4FF0570ECEEB57
:10AE90000404A3420FDD002E08DB604506D801D173
:10AEA000544503DC03FB0040012601E04FF0FF3670
:10AEB00015F8014BD8E7002E07DA2223C8F8003036
:10AEC0004FF0FF302AB9BDE8F08707B1404272B1B8
:10AED00006B1691E1160BDE8F0873024002BB9D19E
:10AEE0000823B7E70A23B5E7302CABD0B2E7BDE8BB
:10AEF000F08700BF2001002013460A4601460248A1
:10AF00000068FFF77BBF00BF1C010020704770473F
:10AF1000044B1968024609B90349196018680244CC
:10AF20001A607047484A0020504A0020FEE710B5DA
:10AF3000431E0A44914204D011F8014B03F8014F1B
:10AF4000F8E710BD0EB400B59CB04FF402711DAB14
:10AF5000ADF81410029006906FF000410A48049179
:10AF600007914FF6FF7153F8042BADF816100068E7
:10AF7000019302A900F0FCF8029B00221A701CB099
:10AF80005DF804EB03B070471C01002010B50246C9
:10AF9000134601321C78002CFAD1013B11F8012B29
:10AFA00003F8012F002AF9D110BDC9B2034610F8E9
:10AFB000012B1AB19142F9D11846704700290CBFF4
:10AFC00018460020704710F8012B11F8013B012AA8
:10AFD00028BF9A42F7D0D01A7047034611F8012BC8
:10AFE00003F8012B002AF9D17047034613F8012B0F
:10AFF000002AFBD1181A0138704730B582B1451EBE
:10B00000013915F8013F11F8014FA34206D1EC4375
:10B010001444E04201D0002BF3D11C46181B30BD74
:10B02000104630BD10B5034642B111F8014B03F88C
:10B03000014B013A002CF7D11A4400E010BD9342B5
:10B0400002D003F8014BFAE710BD30B5141E0546D7
:10B050009BB0184604DA8B232B604FF0FF301DE0C5
:10B060004FF40273ADF80C3014BF04F1FF332346E4
:10B07000029305934FF6FF7300910491ADF80E30E3
:10B0800002461E9B6946284600F072F8431CBCBF6E
:10B090008B232B6014B1009B00221A701BB030BDB3
:10B0A00007B5009313460A46014603480068FFF7B8
:10B0B000CCFF03B05DF804FB1C0100202DE9F04734
:10B0C0008E689E4282460C46914698463ED88A89B2
:10B0D00012F4906F3AD0256809696F1A65690223E6
:10B0E00005EB450595FBF3F57B1C43449D4238BFBA
:10B0F0001D4653050FD52946FFF748FD064698B172
:10B100003A462169FFF713FFA38923F4906343F0C4
:10B110008003A38113E02A4600F025FB064670B9A0
:10B1200021695046FFF7E4FC0C23CAF80030A389DC
:10B1300043F04003A3814FF0FF30BDE8F087266164
:10B1400065613E44ED1B2660A5604646464528BF26
:10B15000464632464946206800F0EAFAA3689B1B3F
:10B16000A36023681E4426600020BDE8F08700002D
:10B170002DE9F04F9DB0804603938B891C060D4648
:10B1800016460DD50B695BB94021FFF7FFFC28601F
:10B19000286118B90C23C8F80030CDE040236B615A
:10B1A0000023099320238DF82930DFF89CB1302348
:10B1B0008DF82A3037463C4614F8013B1BB9B7EBF3
:10B1C000060910D003E0252BF9D02746F3E74B46BC
:10B1D000324629464046FFF771FF013000F0A78054
:10B1E000099B4B4409933B78002B00F0A08000237F
:10B1F0004FF0FF3204930793059206938DF8533076
:10B200001A930126052221784E4800F041FA671C66
:10B21000049B38B14B4A801A06FA00F01843049098
:10B220003C46EFE7D90644BF20228DF853201A0789
:10B2300044BF2B228DF8532022782A2A03D0079A64
:10B2400000210A200BE0039A111D12680391002AC5
:10B2500010DA524243F00200079204900BE02746B6
:10B2600001343B78303B092B03D800FB023201212B
:10B27000F5E701B107923B782E2B1ED17B782A2B64
:10B280000AD1039B1A1D1B680392002BB8BF4FF015
:10B29000FF330237059310E000230593781C19460D
:10B2A0000A24074601303A78303A092A03D804FBC9
:10B2B00001210123F5E703B10591032239782248E2
:10B2C00000F0E6F940B14023CBEB000003FA00F0B8
:10B2D000049B18430490013739781C488DF82810D6
:10B2E00006227E1C00F0D4F988B1194B33B9039BB8
:10B2F000073323F007030833039314E003AB0093F1
:10B300002A46144B04A94046AFF3008007E003AB84
:10B3100000932A460F4B04A9404600F093F8B0F181
:10B32000FF3F824603D0099B5344099342E7AB8910
:10B330005B0601D4099801E04FF0FF301DB0BDE875
:10B34000F08F00BF41D3000847D300084BD300085B
:10B3500000000000BDB000082DE9F04791461F46EF
:10B360000A698B68DDF820809342B8BF1346C9F89C
:10B37000003091F8432006460C4612B10133C9F85B
:10B3800000302368990642BFD9F800300233C9F86B
:10B390000030256815F0060510D104F1190A07E000
:10B3A0000123524639463046C04701301AD0013594
:10B3B000E368D9F800209B1A9D42F1DB94F84330F2
:10B3C0002268003318BF012392060FD5E1185A1CDA
:10B3D000302081F84300224494F8451082F843104D
:10B3E000023303E04FF0FF30BDE8F08704F1430281
:10B3F00039463046C0470130F4D02268D9F80050B1
:10B40000E36802F00602042A08BF5D1B2269A368F4
:10B410000CBF25EAE57500259342C4BF9B1AED18C1
:10B420004FF000091A344D4509D001232246394610
:10B430003046C0470130D5D009F10109F3E70020BB
:10B44000BDE8F0872DE9F04317460A7E85B06E2AE5
:10B45000984606460C460C9B01F1430E00F0AE8068
:10B4600011D8632A22D009D8002A00F0BB80582ABC
:10B4700040F0CA8081F84520834955E0642A1ED0F7
:10B48000692A1CD0C0E0732A00F0B08009D86F2A66
:10B490002ED0702A40F0B8800A6842F020020A607C
:10B4A0003EE0752A24D0782A3AD0ADE01A6801F13E
:10B4B0004205111D1960136884F84230A8E0216824
:10B4C0001A6811F0800F02D0111D196008E011F008
:10B4D000400F02F10401196002D0B2F9003000E01F
:10B4E0001368002B3CDA2D225B4284F8432037E0BE
:10B4F00021681A6811F0800F02D0111D196007E051
:10B5000011F0400F02F10401196001D0138800E02E
:10B510001368227E5C496F2A14BF0A2208221BE0AE
:10B5200078225A4984F845202268186812F0800F62
:10B5300000F104051D6003D1550601D5038800E024
:10B540000368D00744BF42F0200222601BB9226882
:10B5500022F0200222601022002084F8430001E043
:10B5600049490A226568A560002D08DB206820F0A3
:10B57000040020602BB9002D7DD175460CE0002B16
:10B5800079D07546B3FBF2F002FB1033CB5C05F8C3
:10B59000013D03460028F5D1082A0BD12368DA07BC
:10B5A00008D5236962689A42DEBF302305F8013C62
:10B5B00005F1FF35C5EB0E0323612EE008681A681C
:10B5C000496910F0800F03D0101D1860136808E05F
:10B5D00010F0400F02F104001860136801D01980C8
:10B5E00000E0196000232361754616E01A68111DFA
:10B5F0001960156862680021284600F049F808B112
:10B60000401B6060636804E004F1420584F8422056
:10B6100001232361002384F84330CDF800803B46AA
:10B6200003AA21463046FFF797FE013002D14FF0C2
:10B63000FF3026E023692A4639463046C0470130AC
:10B64000F5D023689B0710D5002504F1190907E000
:10B6500001234A4639463046C0470130E7D001351C
:10B66000E368039A9B1A9D42F2DBE068039B9842D1
:10B67000B8BF184605E00B7884F8423004F1420563
:10B680008AE705B0BDE8F08352D3000863D3000811
:10B6900001F0FF01102A2BDB10F0070F08D010F883
:10B6A000013B013A8B422DD010F0070F42B3F6D187
:10B6B000F0B441EA012141EA014122F007047FF0A0
:10B6C00000070023F0E80256083C85EA010586EAF7
:10B6D000010685FA47F5A3FA87F586FA47F6A5FA33
:10B6E00087F68EB9EED1F0BC01F0FF0102F007023F
:10B6F00032B110F8013B013A83EA010313B1F8D1EA
:10B700000020704701387047002D06BF35460338CA
:10B71000073815F0010F07D1013015F4807F02BF03
:10B72000013015F4C03F0130F0BC0138704700BF54
:10B73000884210B501EB020301D8421E0BE098428B
:10B74000FBD28118D21AD34204D013F8014D01F86C
:10B75000014DF8E710BD994204D011F8014B02F8F1
:10B76000014FF8E710BDF8B5074615460E4621B95A
:10B770001146BDE8F840FFF709BA1AB9FFF7B8F962
:10B780002846F8BD00F015F885420ED929463846FE
:10B79000FFF7FCF9044650B131462A46FFF7C7FBD4
:10B7A00031463846FFF7A4F901E03046F8BD20469F
:10B7B000F8BD51F8040C0028BEBF091851F8043C2C
:10B7C000C018043870470000F8B500BFF8BC08BCCA
:10B7D0009E467047F8B500BFF8BC08BC9E4670474F
:10B7E0002E350075636C6F636B2E64650075706435
:10B7F000617465000D0A57656C636F6D6520746F29
:10B8000020576F7264436C6F636B204C6F67676582
:10B810007221002D2D2D2D2D2D2D2D2D2D2D2D2D4C
:10B820002D2D2D2D2D2D2D2D2D2D2D2D2D2D2D0075
:10B8300069726D705F696E69742E2E2E00706F775D
:10B8400065725F696E69742E2E2E00706F77657257
:10B850005F696E697428292063616C6C656400708F
:10B860006F7765725F6F6E2E2E2E0064656C617946
:10B870005F696E69742E2E2E00626F6172645F6C58
:10B8800065645F696E69742E2E2E0074696D657231
:10B89000325F696E69742E2E2E0077707362757434
:10B8A000746F6E5F696E69742E2E2E00566572730A
:10B8B000696F6E3A2000332E302E305431004861CB
:10B8C0007264776172653A2053544D333246343195
:10B8D000315245004C4544733A2057533238313287
:10B8E00020475242005359533A256C7520483A2557
:10B8F0006C752C2050313A256C752C2050323A252D
:10B900006C750D0A00727463206973206F6E6C6928
:10B910006E6500727463206973206F66666C696E71
:10B920006500656570726F6D2F666C617368206964
:10B9300073206F6E6C696E6500656570726F6D2F38
:10B94000666C617368206973206F66666C696E65EA
:10B9500000747279696E6720746F20726564756314
:10B96000652049324320636C6F636B20737065659B
:10B97000642E2E2E00727463206973206E6F772000
:10B980006F6E6C696E65007274632072656D6169BB
:10B990006E73206F66666C696E6500656570726FA8
:10B9A0006D206973206E6F77206F6E6C696E650015
:10B9B000656570726F6D2072656D61696E73206F61
:10B9C0006666696E65007570646174696E672045AE
:10B9D0004550524F4D20746F2076657273696F6EBB
:10B9E000203078253038782E2E2E200049522063C2
:10B9F0006F646573006E696768742074696D652093
:10BA0000636F6E66696775726174696F6E00616CF1
:10BA100061726D2074696D6520636F6E666967750C
:10BA2000726174696F6E0074656D706572617475B2
:10BA3000726520636F6E66696775726174696F6E97
:10BA40000052544320636F6E666967757261746952
:10BA50006F6E004C445220636F6E66696775726149
:10BA600074696F6E007765617468657220636F6ECC
:10BA700066696775726174696F6E00757064617470
:10BA800065206D61696E20706172616D65746572AB
:10BA90007320636F6E66696775726174696F6E009B
:10BAA000646F6E65004446504C41594552204C4FDE
:10BAB000474745520D0A0045535038323636204C20
:10BAC0004F474745520D0A007265616420727463E6
:10BAD0003A202573202534642D253032642D2530FD
:10BAE000326420253032643A253032643A253032CF
:10BAF000640D0A007573657220627574746F6E2030
:10BB0000707265737365643A20636F6E66696775FA
:10BB100072696E6720657370383236362061732023
:10BB200061636365737320706F696E7400313233C3
:10BB30003435363738393000776F7264636C6F6331
:10BB40006B00617020222573222C2225732200773E
:10BB5000707320627574746F6E2070726573736594
:10BB6000643A2073656E64696E672065737038325D
:10BB700036362077707320636F6D6D616E64007769
:10BB800070730065737038323636206E6F772075AB
:10BB9000700065737038323636206E6F77206F6EA6
:10BBA0006C696E650064636637373A20257320251B
:10BBB00034642D253032642D253032642025303216
:10BBC000643A253032643A253032640D0A007469D3
:10BBD0006D6500466F756E642054696D65723A201C
:10BBE000257320617420253032643A253032640D8B
:10BBF0000A00466F756E642054696D65723A206163
:10BC00006D62696C696768742025732061742025F2
:10BC10003032643A253032640D0A006E65745F7408
:10BC2000696D655F636F756E74646F776E203D201C
:10BC300025642C20646F6E277420636865636B2015
:10BC40006F7665726C6179730D0A004453313878F0
:10BC500078782074656D70657261747572653A20CC
:10BC6000256425730D0A005254432074656D706578
:10BC70007261747572653A20256425730D0A006F30
:10BC80007665726C61792069636F6E2025730D0A89
:10BC90000075632D69636F6E2E747874006F76651E
:10BCA000726C61792064617465006F7665726C6195
:10BCB000792074656D7065726174757265006F7658
:10BCC00065726C617920776561746865722069635B
:10BCD0006F6E006F7665726C61792077656174684C
:10BCE000657220666F7265636173742069636F6E3D
:10BCF000006F7665726C6179207765617468657232
:10BD0000006F7665726C6179207765617468657221
:10BD100020666F726563617374006F7665726C6123
:10BD200079207469636B65723A20272573270D0AA1
:10BD3000006F7665726C6179206D70333A20253022
:10BD400032642F253033640D0A006F7665726C61A2
:10BD500079206D70333A20696E76616C6964206673
:10BD60006F726D61743A2025730D0A00676F74203D
:10BD700074656D70657261747572652066726F6D41
:10BD800020445331387878783A20256425730D0A99
:10BD900000676F742074656D70657261747572658B
:10BDA0002066726F6D205254433A20256425730D2E
:10BDB0000A00737769746368696E6720706F7765CE
:10BDC00072206F6666006466706C617965722069C6
:10BDD00073206F6E6C696E650025642025303264B7
:10BDE0003A2530326420616C61726D5F696478203D
:10BDF0003D2025640D0A00737065616B3A20253083
:10BE000032643A253032640D0A00646973706C61E3
:10BE10007920636F6E66696775726174696F6E0011
:10BE20006F7665726C617920636F6E666967757293
:10BE30006174696F6E0074696D65736572766572A1
:10BE400020636F6E66696775726174696F6E0064F6
:10BE500066706C6179657220636F6E666967757272
:10BE60006174696F6E005375004D6F005475005713
:10BE700065005468004672005361000066BE000809
:10BE800069BE00086CBE00086FBE000872BE0008E4
:10BE900075BE000878BE00080000003F0000003FAB
:10BEA000003F3F0000003F3F003F003F3F3F3F3F1C
:10BEB00020200020202000000100010002000200DC
:10BEC000030003000400040005000500060007004D
:10BED000080009000B000D000E00100012001400F5
:10BEE000170019001C001F002100240028002B004F
:10BEF0002E003200360039003D00420046004A0064
:10BF00004F00540059005E00630069006E00740029
:10BF10007A00800086008C0093009900A000A700A2
:10BF2000AE00B600BD00C500CD00D500DD00E500C7
:10BF3000EE00F600FF003F3F3F3F00000403030315
:10BF40000303034E65772074696D657A6F6E653AF9
:10BF50002025640D0A004446506C617965723A20D0
:10BF600073657420766F6C756D652025640D0A000D
:10BF7000636D643A2073657420756E6B6E6F776EB7
:10BF8000206E756D20766172206964782025643A90
:10BF90002025640D0A0050756E6B74653A20256C7F
:10BFA0006400495020257300696E666F3A206970FD
:10BFB0002061646472657373203D2025730D0A004F
:10BFC000414E00414400414500414600434E00437C
:10BFD00044004345004346004D4E004D44004D454E
:10BFE000004D46004F54004F49004F44004F43005E
:10BFF0004F530025732530327825303478004F595F
:10C00000004F4E004F46007425303278253032788C
:10C01000253032782530327800612530327825306D
:10C0200032782530327825303278006C25303278FD
:10C0300025303278253032782530327800696E66C6
:10C040006F3A2077656174686572203D2025730D15
:10C050000A00696E666F3A207765617468657220C0
:10C06000666F726563617374203D2025730D0A004D
:10C07000696E666F3A2077656174686572206963DE
:10C080006F6E2025730D0A0075632D7765617468E6
:10C0900065722E74787400696E666F3A20776561F8
:10C0A0007468657220666F7265636173742069637A
:10C0B0006F6E2025730D0A0063616E6E6F742072BF
:10C0C0006561642069636F6E0D0A0050756E6B7454
:10C0D000653A20256400003F00003F3F00003F20FC
:10C0E00020203F3F00003F003F003F3F000044460C
:10C0F000506C617965723A2077726F6E6720636861
:10C1000065636B73756D0D0A004446506C6179650B
:10C11000723A20696E7365727465642055534220CB
:10C12000737469636B004446506C617965723A20A0
:10C13000696E736572746564205344206361726430
:10C14000004446506C617965723A20696E7365727D
:10C1500074656420756E6B6E6F776E2064657669AA
:10C160006365004446506C617965723A2072656D72
:10C170006F7665642055534220737469636B004485
:10C1800046506C617965723A2072656D6F766564B0
:10C190002053442063617264004446506C617965A9
:10C1A000723A204446506C617965722072656D6FF9
:10C1B00076656420756E6B6E6F776E206465766948
:10C1C0006365004446506C617965723A207472610F
:10C1D000636B202564206F6E205553422073746971
:10C1E000636B2066696E69736865642E0D0A00448E
:10C1F00046506C617965723A20747261636B2025D8
:10C2000064206F6E20534420636172642066696EFF
:10C2100069736865642E0D0A004446506C61796547
:10C22000723A20747261636B202564206F6E204621
:10C230006C6173682066696E69736865642E0D0AA7
:10C24000004446506C617965723A204E6F206D65EE
:10C250006D6F727920666F756E64004446506C6134
:10C260007965723A2055534220737469636B206F6D
:10C270006E6C696E65004446506C617965723A2057
:10C2800053442063617264206F6E6C696E65004474
:10C2900046506C617965723A2050432028415558C8
:10C2A00029206F6E6C696E65004446506C6179653B
:10C2B000723A20466C617368206F6E6C696E65001F
:10C2C0004446506C617965723A204D6F64756C65B7
:10C2D0002069732062757379004446506C617965FA
:10C2E000723A204672616D65206461746120696EE6
:10C2F000636F6D706C657465004446506C61796560
:10C30000723A20566572696669636174696F6E205E
:10C310006572726F72004446506C617965723A20A2
:10C3200046696C65206E6F7420666F756E6400449C
:10C3300046506C617965723A20556E6B6E6F776E00
:10C34000206572726F723A20307825303258203072
:10C3500078253032580D0A004446506C6179657278
:10C360003A205265706C793F3F004446506C6179C9
:10C3700065723A20537461747573202530325820E9
:10C38000253032580D0A004446506C617965723A86
:10C3900020566F6C756D652025640D0A004446506B
:10C3A0006C617965723A204551204E6F726D616CF7
:10C3B000004446506C617965723A20455120506FB7
:10C3C00070004446506C617965723A2045512052A4
:10C3D0006F636B004446506C617965723A20455139
:10C3E000204A617A7A004446506C617965723A203D
:10C3F000455120436C6173736963004446506C611E
:10C400007965723A20455120426173730044465069
:10C410006C617965723A20455120756E6B6E6F774D
:10C420006E004446506C617965723A20506C6179B7
:10C430006261636B206D6F6465204E6F726D616C1D
:10C44000004446506C617965723A20506C617962A3
:10C4500061636B206D6F646520466F6C646572006C
:10C460004446506C617965723A20506C6179626122
:10C47000636B206D6F64652053696E676C65004463
:10C4800046506C617965723A20506C6179626163E3
:10C490006B206D6F64652052616E646F6D00444661
:10C4A000506C617965723A20506C61796261636B9E
:10C4B000206D6F646520756E6B6E6F776E004446FD
:10C4C000506C617965723A2056657273696F6E209F
:10C4D000253034580D0A004446506C617965723A33
:10C4E00020534420636172642066696C6573202563
:10C4F000640D0A004446506C617965723A205553C8
:10C500004220737469636B2066696C6573202564CF
:10C510000D0A004446506C617965723A20466C61A0
:10C5200073682066696C65732025640D0A004446B3
:10C53000506C617965723A204B656570206F6E3F73
:10C540003F3F0D0A004446506C617965723A2053B2
:10C5500044206361726420747261636B2025640DF2
:10C560000A004446506C617965723A205553422066
:10C57000737469636B20747261636B2025640D0AA8
:10C58000004446506C617965723A20466C6173686C
:10C5900020747261636B2025640D0A004446506C60
:10C5A000617965723A20717565727920736F66746E
:10C5B000776172652076657273696F6E00444650CC
:10C5C0006C617965723A2073657420736F7572635C
:10C5D00065206465766963653A2025640D0A004428
:10C5E00046506C617965723A2073657420657120DC
:10C5F00025640D0A004446506C61796572206973A8
:10C600002075700076617220004443253032782511
:10C61000303278253032782530327830300025734A
:10C620002530327825730025732530327825303255
:10C6300078006765742074656D70657261747572D9
:10C640006500746F67676C65206175746F20627236
:10C65000696768746E657373006F6B0064656372FD
:10C66000656D656E7420646973706C6179206D6F9F
:10C67000646500696E6372656D656E7420646973CC
:10C68000706C6179206D6F64650064656372656DBF
:10C69000656E7420616E696D6174696F6E206D6F77
:10C6A000646500696E6372656D656E7420616E69A4
:10C6B0006D6174696F6E206D6F646500646563728F
:10C6C000656D656E7420686F757200696E63726562
:10C6D0006D656E7420686F75720064656372656D58
:10C6E000656E74206D696E75746500696E63726540
:10C6F0006D656E74206D696E757465006465637236
:10C70000656D656E74207265642062726967687415
:10C710006E65737300696E6372656D656E74207209
:10C720006564206272696768746E6573730064651E
:10C730006372656D656E7420677265656E206272E6
:10C74000696768746E65737300696E6372656D65A1
:10C750006E7420677265656E206272696768746EB8
:10C760006573730064656372656D656E7420626CD9
:10C770007565206272696768746E65737300696EAF
:10C780006372656D656E7420626C75652062726996
:10C790006768746E6573730064656372656D656E5A
:10C7A0007420676C6F62616C206272696768746E76
:10C7B00065737300696E6372656D656E7420676C76
:10C7C0006F62616C206272696768746E6573730072
:10C7D000706F776572206F66662F6F6E0020205431
:10C7E00068616E6B20796F75210073776974636877
:10C7F000696E6720706F776572206F6E006F766567
:10C80000726C61795F63616C635F6F7665726C6196
:10C81000795F64617465733A20696E76616C6964EE
:10C8200020646174655F636F64653A2025640D0A56
:10C8300000000F00000202020200000F00040404C6
:10C8400004080E000006040400000E020004040C9C
:10C8500000020E000004040600000E08000C040490
:10C860000006060000060600000606000006060098
:10C8700000060C00000406020000060C00080C0470
:10C8800000040E000004060400000E0400040C0462
:10C89000000C06000002060400000C0600040C0850
:10C8A000000000003F0000002F0000001F000000FB
:10C8B0000F00000000000000000000000000000069
:10C8C0000000000000000000000000000000000068
:10C8D0000000000000000000000000000000000058
:10C8E0000F0000001F0000002F0000003F000000AC
:10C8F0003F0000003F0000003F0000003F0000003C
:10C900003F0000004E6F6E65004661646500536332
:10C91000726F6C6C004578706C6F646500536E616B
:10C920006B650054656C657479706500437562656C
:10C9300000477265656E4D61747269780044726F6C
:10C94000700053717565657A6500466C69636B6547
:10C950007200526F6C6C005261696E626F770044B6
:10C9600061796C6967687400436C6F636B00436C3A
:10C970006F636B3200442E4D2E590077733238317D
:10C98000323A2065787465726E616C2070756C6CDB
:10C9900075702064657465637465640077733238FC
:10C9A00031323A206E6F2065787465726E616C204A
:10C9B00070756C6C75702064657465637465640073
:10C9C00025303464253032642530326425303264B9
:10C9D000253032640000000000000000000000006C
:10C9E0000000000000000000000000000000000047
:10C9F0000000000000000000000000000F00000028
:10CA00001F0000002F0000003F0000002F0000006A
:10CA10001F0000000F0000000000000000000000E8
:10CA20000000000000000000000000000000000006
:10CA300000000000000000000000000000000000F6
:10CA4000000000000F0000001F0000002F00000089
:10CA50003F0000003F0000003F0000003F000000DA
:10CA60003F0000003F0000003F0000003F000000CA
:10CA70003F0000003F0000003F0000003F000000BA
:10CA80003F0000002F0000001F0000000F0000000A
:10CA9000000000000000000002000000050000008F
:10CAA0000C00000011000000220000000500000042
:10CAB0000C000000050000000C0000000000000059
:10CAC0001000000010000000200000002000000006
:10CAD0000100000001000000000000000200000052
:10CAE000050000000C000000110000002200000002
:10CAF000050000000C000000050000000C00000014
:10CB00000000000000000000000000000000000025
:10CB10000000000001000000010000000000000013
:10CB20001F0000001C0000001F0000001E0000008D
:10CB30001F0000001E0000001F0000001F0000007A
:10CB40001E0000001F0000001E0000001F0000006B
:10CB5000010000000F0000001500000007000000A9
:10CB60000B000000070000000B00000007000000A1
:10CB70000B0000000F000000140000000000000087
:10CB80000F00000014000000000000000100000081
:10CB90000000000003000000050000000C00000081
:10CBA0000F0000001E000000050000000C00000047
:10CBB000040000000B000000000000001000000056
:10CBC0001500000025000000250000000100000005
:10CBD000010000000000000005000000020000004D
:10CBE0000B0000000C0000001A0000000200000012
:10CBF0000B000000020000000B000000000000001D
:10CC0000100000001C0000002800000030000000A0
:10CC1000010000000100000000000000444346370E
:10CC200037204572726F723A2048696768207075C4
:10CC30006C7365203C3D2035004443463737204522
:10CC400072726F723A20486967682070756C7365FC
:10CC5000203E3D203235004443463737204572722E
:10CC60006F723A2070617269747920503120696E58
:10CC7000636F7272656374004443463737204572B0
:10CC8000726F723A20706172697479205032206933
:10CC90006E636F7272656374004443463737204594
:10CCA00072726F723A207061726974792050332009
:10CCB000696E636F7272656374006572726F723A47
:10CCC0002063616E6E6F74207265736574204932E3
:10CCD0004320627573002D2D3E20003C25303278B4
:10CCE0003E003C30643E3C30613E0D0A00003F3F58
:10CCF00057726974696E6720257320746F204545EB
:10CD000050524F4D206661696C65640D0A00637571
:10CD10007272656E7420656570726F6D2F666C61DE
:10CD200073682076657273696F6E3A2030782530AB
:10CD300038780D0A0072656164696E672069722037
:10CD4000636F646573003139322E35332E313033E1
:10CD50002E31303300222C22007769636F6E00770A
:10CD600069636F6E5F666300776561746865725FA3
:10CD700066630053253032782573004E25303278B3
:10CD800025303278253032780054253032782530FD
:10CD900034642530326425303264253032642530E5
:10CDA0003264253032640000000000000000000CF6
:10CDB00012120C000000000A00040A111F110012D8
:10CDC0000C121212120C000A00121212120C000A9B
:10CDD000000E010F110F000A000C1212120C0012AB
:10CDE00000121212160A00001C121C12121C100053
:10CDF0000000000000000000000000000000000033
:10CE00000000000000000000000000000000000022
:10CE10000000000000000000000000000000000012
:10CE20000000000000000000000000000000000002
:10CE300000000000000000000000000000000000F2
:10CE400000000000000000000000000000000000E2
:10CE500000000000000000000000000000000000D2
:10CE600000000000000000000000000000000000C2
:10CE700000000000000000000000000000000000B2
:10CE800000000000000000000000000000000000A2
:10CE90000000000000000000000000000000000092
:10CEA000000000000000000000000000000000047E
:10CEB0000E0E04040004001B1B1200000000000002
:10CEC0000A1F0A0A1F0A00080E100C021C0400198F
:10CED000190204081313000814140815120D000C8D
:10CEE0000C080000000000040808080808040008F6
:10CEF00004040404040800000A0E1F0E0A000000C7
:10CF000004041F0404000000000000000C0C0800D2
:10CF100000001F0000000000000000000C0C0000DA
:10CF2000010204081000000E11111111110E00046D
:10CF30000C040404040E000E11010608101F000E5C
:10CF400011010E01110E0002060A121F0202001F3B
:10CF500010101E01110E000608101E11110E001FE8
:10CF6000010204080808000E11110E11110E000E26
:10CF700011110F01020C00000C0C000C0C00000041
:10CF8000000C0C000C0C080204081008040200003D
:10CF9000001F00001F000008040201020408000E28
:10CFA000110106040004000E11171517100E000ED3
:10CFB0001111111F1111001E11111E11111E000E51
:10CFC00011101010110E001E11111111111E001F51
:10CFD00010101E10101F001F10101E101010000E39
:10CFE00011101711110F001111111F111111000E45
:10CFF00004040404040E000101010111110E0011CA
:10D00000121418141211001010101010101F00111B
:10D010001B15111111110011191513111111000E09
:10D0200011111111110E001E11111E101010000E01
:10D0300011111115120D001E11111E121111000EE9
:10D0400011100E01110E001F040404040404001149
:10D0500011111111110E0011111111110A040011F9
:10D0600011151515150A0011110A040A11110011E4
:10D0700011110A040404001E02040810101E000E00
:10D0800008080808080E0000100804020100000E3D
:10D0900002020202020E00040A1100000000000059
:10D0A0000000000000003F0C0C0400000000000025
:10D0B000000E010F110F0010101E1111111E0000A3
:10D0C000000E1110110E0001010F1111110F0000BF
:10D0D000000E111E100E000608081E0808080000A9
:10D0E000000F11110F010E10101C12121212000469
:10D0F00000040404040600020006020202120C10DE
:10D10000101214181412000404040404040600008D
:10D11000001A151511110000001C12121212000045
:10D12000000E1111110E0000001E1111111E100031
:10D13000000F1111110F010000160908081C000052
:10D14000000E100E010E0000081E08080A04000060
:10D1500000121212160A0000001111110A04000038
:10D16000001111151F0A00000012120C121200000B
:10D17000001212120E041800001E020C101E0006EF
:10D180000808180808060004040400040404000C3D
:10D1900002020302020C000A14000000000000005A
:10D1A000000000000000006E253032782530327813
:10D1B000253032780046494C4520002800290D0AC8
:10D1C000004F4B004552524F52002D200049504114
:10D1D0004444524553532000415020004D4F444594
:10D1E000200061700054494D452000574541544886
:10D1F00045522000574541544845525F4643200060
:10D200005749434F4E20005749434F4E5F464320F6
:10D21000004649524D574152452000434D4420009D
:10D220004F50454E2000434C4F5345002573222C50
:10D230002225730025752C3500257500BC000020C3
:10D2400000202020202020202020282828282820D6
:10D2500020202020202020202020202020202020CE
:10D260002088101010101010101010101010101036
:10D270001004040404040404040404101010101026
:10D2800010104141414141410101010101010101F0
:10D290000101010101010101010101011010101042
:10D2A00010104242424242420202020202020202C2
:10D2B0000202020202020202020202021010101016
:10D2C000200000000000000000000000000000003E
:10D2D000000000000000000000000000000000004E
:10D2E000000000000000000000000000000000003E
:10D2F000000000000000000000000000000000002E
:10D30000000000000000000000000000000000001D
:10D31000000000000000000000000000000000000D
:10D3200000000000000000000000000000000000FD
:10D3300000000000000000000000000000000000ED
:10D3400000232D302B2000686C4C00656667454635
:10D35000470030313233343536373839414243446F
:10D3600045460030313233343536373839616263FF
:08D37000646566000000000086
:08D378006C2EFF7F0100000094
:10D380000500000020000000003F3F00FF000000FB
:10D39000D80E0000FF0000001F0000000000FF0F7B
:10D3A000FF00000000000000000000000102030474
:10D3B00006070809FFFFFFFF04000000FF00000050
:10D3C000FFFF00002000000005000000000000003A
:10D3D000010203040102030406070809FF0000001C
:10D3E000FFFF0000FF0000003139322E35332E31AF
:10D3F00030332E3130330000000000000100000007
:10D4000000000000FF00000020000000FF000000FE
:10D41000FF000000FF000000FFFF0000FFFF000012
:10D420000A0000000000000000000000FF000000F3
:10D43000640000008C460020007A030A000000000F
:10D4400000000000000000000000000000000000DC
:10D45000000000000000000000000000EEBF000817
:10D4600000000000000000000000000000000000BC
:10D4700000000000000000000000000000000000AC
:10D48000000000000000000000000000000000009C
:10D49000000000000000000000000000BC000020B0
:0CD4A00040D20008AD010008890100081E
:0400000508000000EF
:00000001FF
